:020000040800F2
:100000001840002039030008E93A0008753A000852
:10001000E53A0008551700081573000800000000B5
:10002000000000000000000000000000955A0008D9
:10003000051B0008000000004D4A0008995A0008FE
:100040005303000853030008530300085303000838
:100050005303000853030008530300085303000828
:10006000211B000853030008530300085303000832
:100070005303000853030008530300085303000808
:1000800053030008530300085303000853030008F8
:1000900053030008530300085303000853030008E8
:1000A000530300085303000853030008BD5A000817
:1000B000CD5A0008DD5A0008ED5A00085303000825
:1000C00053030008530300085303000853030008B8
:1000D00053030008530300085303000853030008A8
:1000E000091B0008530300085303000853030008CA
:1000F000815F000853030008715F00085303000884
:100100005303000853030008FD5A00085303000876
:1001100053030008530300080D5B0008615B0008EF
:100120005303000853030008530300085303000857
:100130005303000853030008530300085303000847
:10014000530300085303000853030008653B0008ED
:100150005303000853030008530300085303000827
:100160005303000853030008530300085303000817
:100170005303000853030008530300080000000065
:10018000530300085303000800F002F800F0AAF837
:1001900014A696E8000CB244B344DA4501D100F04D
:1001A000A1F8BAE80F000FA696E83000A5EB040509
:1001B00004EB0607AAEB0704A7F101074FEA1515A0
:1001C0004FEA3414A4F10104AC4201D300F08AF8E0
:1001D00013F0010F18BFFB1A43F0010300F001F800
:1001E000DBE7184700E2000020E20000103A24BFDD
:1001F00078C878C1FAD8520724BF30C830C144BF8C
:1002000004680C6070470000704700000023002461
:1002100000250026103A28BF78C1FBD8520728BF16
:1002200030C148BF0B6070476E2900F0958170297E
:1002300000F0D78266290DF00A8765290DF007873F
:1002400067290DF0048761290DF0038703681B0AF5
:1002500028BF41F08001692900F04281642900F043
:100260003F81752900F03C816F2900F06582782973
:1002700000F0A382E92900F0FF81E42900F0FC816D
:10028000F52900F0F981EF2900F06282F82900F0E9
:10029000A2820368DB0928BF41F08001632900F0D6
:1002A000A387732900F0A887E32900F0B387F32917
:1002B00000F0B887002070471FB50DF0B6FE00F0C3
:1002C00082F801F005F80400002000210DF030FA5A
:1002D000401C6060002000210DF014FAE0601FBD9A
:1002E00010B510BD00F0C6FF1146FFF7E5FF07F09F
:1002F000CBFA01F0A3F803B4FFF7F2FF03BC01F05F
:10030000EBF800000B49D1F800C04A685CF8043BE8
:100310001068184442F8040B8C4528BFA1F1DC0C8E
:100320008A4228BFA1F1DC02C1F800C04A6020F077
:1003300000407047CC010020094880470948004729
:10034000FEE7FEE7FEE7FEE7FEE7FEE7FEE7FEE785
:10035000FEE7FEE704480549054A064B70470000E2
:10036000A95A00088901000818340020184000200C
:1003700018380020183800201CB50C46064B7B446A
:1003800069460090204600F000F9044600206946C6
:1003900000F00EF920461CBD2F0200000B4910B5DD
:1003A000A1F17C020A4CC2E93712372106E000EBCA
:1003B000104342F82130074B00FB03400B1EA1F114
:1003C0000101F4DC10BD0120E8E700006C01002011
:1003D000E119D666CD0D010010B5431C02E010F8FE
:1003E000011B71B18107FAD14FF0013202C88C1A9A
:1003F0008C4314EAC211F9D0C01A0A0603D0C01EF9
:1004000010BDC01A10BD0A0401D0801E10BD090223
:10041000FCD0401E10BD70477047704770B5044651
:1004200085690068C10601D5302600E02026C00796
:1004300007D070BDD4E9012130469047206A401CA6
:1004400020626D1EF6D570BD70B5044685690078D2
:10045000C00707D170BDD4E9012120209047206A50
:10046000401C20626D1EF6D570BD09684A0501D595
:1004700040B27047C905FCD500B2704709684A050B
:1004800001D5C0B27047C905FCD580B2704770B5C0
:100490000C460546012A05D02878800600D5EA6971
:1004A000002302E0012305E05B1C934202D2E05CE2
:1004B0000028F9D1A869E618C01AA861286A18446A
:1004C00028622846FFF7AAFF04E0D5E9012114F8C5
:1004D000010B9047B442F8D32846FFF7B5FF70BD33
:1004E0002DE9F0410646002410687529314616A50D
:1004F00010D0FFF7BAFF002802DA404213A507E048
:1005000031688A0701D512A502E0490704D511A573
:10051000012401E0FFF7B2FF00210A2206F12407BF
:1005200009E0B0FBF2FCB0FBF2F302FB1C00303040
:1005300078541846491C0028F3D123462A463046F1
:10054000BDE8F04100F061BA000000002D0000009D
:100550002B0000002000000011680268006A5305AB
:1005600001D508700AE0D30501D5088006E013061E
:1005700003D5C217C1E9000200E0086001207047FE
:1005800001694A1C02610878704700B58FB0CDE957
:1005900001310021059105497944CDE90310114647
:1005A000684600F029F90FB000BD0000E5FFFFFF2D
:1005B0000A6802F8010B0A60704700002DE9FF5F2E
:1005C00015468A460446DFF8AC80F8440027D8E98F
:1005D00000103E46CDE9001010E03AF816106A46C9
:1005E00002A800F023FE411C07D02178890603D51C
:1005F000E269391891420DD80744761C20788006AC
:1006000002D5E069B84205DDAE42E6DB3AF81600F5
:100610000028E2D1A069C01BA0612046FFF7FEFEC2
:10062000D8E90010CDE90010002017E03AF81810C2
:100630006A4602A800F0FAFDB0F1FF3F81460BD0F8
:1006400000250DF1080B05E0D4E901211BF8050098
:1006500090476D1C4D45F7D308F10100B04280462C
:10066000E4DB206A384420622046FFF7EDFEBDE857
:10067000FF9F00008ADA00002DE9F0418046D21D7C
:1006800022F007020025D2E90002F52915A614D0B0
:10069000011E72F1000106DA0023D0EB030063EBC8
:1006A000020211A608E0D8F800108B0701D50FA6AA
:1006B00002E0490701D50EA601251146002408F1E4
:1006C000240704E000F05CF930323A55641C50EA2B
:1006D0000102F7D12B46324621464046BDE8F041A3
:1006E00000F093B9000000002D0000002B00000076
:1006F0002000000030B4002100F1240408E002F0E2
:100700000705D208303542EA4372DB086554491CBC
:1007100052EA0305F3D10468002310A2250708D587
:1007200004F020040C4304D0C46901230CA2641E0D
:10073000C46130BC00F069B910B5044621461068A8
:10074000FFF79CFE02462046BDE810400023D1E79B
:10075000D21D22F00701D1E90023CBE70000000001
:1007600030000000F0B40D460188090502D5214C87
:100770007C4402E01F4C7C440E34002100F124062E
:1007800008E002F00F071209E75D42EA03721B0955
:100790007754491C52EA0307F3D102780023120769
:1007A00004D5702D06D009B1022311342246F0BCC5
:1007B00000F02BB901231034F8E770B504460D465C
:1007C00021461068FFF75AFE024629462046BDE83A
:1007D00070400023C6E7D21D22F00703D3E90023AF
:1007E000C0E70368126843F0200303600823C36175
:1007F0000023B7E7ECD800002DE9F05F89460446F6
:100800004FF0000ADFF874B1FB44C0F820A0204686
:10081000E1688847002874D0252806D0D4E9012152
:100820009047206A401C2062F1E700265F46204680
:10083000E16888472028054607DB312D05D2781965
:1008400010F8200C08B10643F1E7B00701D526F0F7
:100850000406C4F81CA00027C4F818A02A2D09D04B
:1008600028460CF047FF38B304EB8708303DC8F842
:10087000185019E059F8041B204604EB87029161D7
:10088000E1688847012F054618D1E069002820DA81
:1008900026F020061DE0D8F8180000EB800005EBDC
:1008A00040003038C8F818002046E16888470546FF
:1008B0000CF020FF0028EED1012F0AD02E2D08D1F8
:1008C0002046E16888477F1C0546022F46F0200637
:1008D000C4DBA069002803DA404246F00106A061AB
:1008E000F00701D026F010066C2D0BD0682D09D032
:1008F0004C2D39D06A2D35D0742D35D07A2D33D08A
:1009000016E038E0E1682F4620468847B8420546A1
:1009100009D16C2F26D04FF48060E1680643204651
:100920008847054604E06C2F1AD04FF480700643C8
:100930000DB3A5F14100192802D8203546F4006610
:100940004A462946204626604E46FFF76DFC80B198
:1009500001280BD0F61D26F0070000F1080956E724
:100960004020E4E78020D8E70020D6E706F104091C
:100970004DE7284652E7206ABDE8F09F7CD800008A
:1009800030B5B0F10A0271F100034FEA900E4EEA61
:10099000817EB0EB0E0061EB91014FEA101E4EEA32
:1009A000017E10EB0E0041EB11114FEA102E4EEAC2
:1009B000016E10EB0E0041EB11214FEA104E4EEA92
:1009C000014E10EB0E0041EB1141401841F10001C6
:1009D0004FEAD00040EA41704FEAD1014FEA81046A
:1009E00044EA907410EB800544EB01046D1944EB6C
:1009F0000404521BA3414FF0000348BF0A3200D544
:100A000030BD401C41F1000130BD2DE9F0470D46DD
:100A100099469246044600F124080168880604D5E8
:100A2000E06921F01001216000E00120A84201DD11
:100A3000471B00E00027A1697A1902EB0900081A98
:100A4000A0612078C00602D42046FFF7E7FC00260C
:100A500008E0D4E901211AF806009047206A401CFA
:100A6000761C20624E45F4DB2078C0060AD520466D
:100A7000FFF7D4FC06E0D4E9012130209047206A3A
:100A8000401C2062381EA7F10107F4DC07E0D4E91E
:100A9000012118F805009047206A401C2062281E9A
:100AA000A5F10105F3DC2046FFF7CEFC2078000617
:100AB00002D50220BDE8F0870120FBE72DE9FF4FBA
:100AC0000C461E464FF0FF378BB0D2E90001DDF82F
:100AD00060800A908A46C1F30A5505B93D46002157
:100AE00008464FF00000BAF1000F00F4400005DAAC
:100AF00000EB80004FF4400101EA50004FEA9059AA
:100B0000B9F1010F00DDB9460A9850EA4A000ED04B
:100B100044F61050A5F2FF3545432F14B8F1000FED
:100B20001ED07542291E1EDDC9F100021CE0B8F17D
:100B3000010F4FF0000001D0302103E0F24305E047
:100B40002154401CB042FBDB3046002200212154DE
:100B50000B99C1F80880C1E900200FB0BDE8F08F03
:100B6000BD1B6D1CDEE74A4600DA694206A800F0AC
:100B7000F3FB06AB93E8070003AB83E8070050469E
:100B80000A990CF0D6F98DE80700A0F500501F383F
:100B900000900398002D0ADD42F21F014A460844E6
:100BA000002303A9039068460CF040FC09E0A0F57F
:100BB00000504A461F38002303A9039068460CF0F2
:100BC0004AFC8DE807000004000C03D04FF0FF3012
:100BD000410800E01046B8F1000F03D00022009257
:100BE00015461EE0751E05D4FFF7CAFE3032625569
:100BF0006D1EF9D5B3460122084302D000227F1CA6
:100C000004E02078302801D100227F1E002A0997B5
:100C100084D01DE0112D07DAFFF7B2FE30326255A5
:100C20006D1C50EA0102F5D1084302D00098C8B10A
:100C30000EE00021681E05E0235C625C63542254D0
:100C4000401E491C8142F7DBAB46A81B401E0990A1
:100C5000002004F80B000B98099AC0F80880C0E93E
:100C6000002B7AE711264FF0000857E72DE9F04FE7
:100C700088460446D21D22F0070191B0D1E9000157
:100C8000CDE90A010CF01EFD02460B98C00F01D001
:100C90002D2007E02068810701D52B2002E02021CC
:100CA00001EAC000032A099001D0072A05DB0346A8
:100CB0004146204600F010FB0BE12078800601D56C
:100CC000E06900E00620B8F1650F814606D0B8F172
:100CD000660F18D0B8F1670F70D131E00020B9F17C
:100CE000110F009001DB112301E009F101030AAAB1
:100CF00001A90CA8FFF7E2FEDDE90C70002609F15E
:100D00000105834647E001204B4600904FF0004725
:100D10000AAA01A90CA8FFF7D1FEDDE90DB00C99D4
:100D20005D46002610B909F101000D18B9EB050068
:100D300003D4C0F1FF3609F10105A5EB09002BE052
:100D4000B9F1010F01DA4FF001090020B9F1110FDB
:100D50000090484601DD112300E003460AAA01A9DC
:100D60000CA8FFF7ABFEDDE90C704D46002683466C
:100D7000207800070AD4AB4500DA5D4601A8012DB2
:100D800004DD411911F8011C302907D04F4502DA62
:100D900017F1040F04DA012082460FE06D1EEEE722
:100DA000002F02DCED1B3E4403E0781CA84200DD6E
:100DB0007D1CB81B00F1010A4FF0004720780007A6
:100DC00003D4AA4501DB4FF0FF3A0021B7F1004FF1
:100DD0000DF143088DF8431024D002202B23002F5F
:100DE00001DA7F422D230A21021EA0F1010000DC5E
:100DF0005FB197FBF1FC97FBF1F201FB1C7C1746FE
:100E00000CF1300C08F801CDEEE7A8F101000370F9
:100E10002188090501D5452100E06521A0F10108DF
:100E200000F8011C09980FA9A1EB0807FF1D00B1EC
:100E30000120411901EBEA70A1693844081A401EEB
:100E4000A0612078C00602D42046FFF7E7FA09988F
:100E500028B1D4E901219047206A401C2062207803
:100E6000C00622D52046FFF7D9FA1EE0002E04DB8B
:100E7000B34502DD01A8805D00E03020D4E9012106
:100E80009047206A401C2062761CAAF101005FEAAC
:100E9000000A0AD100F01CFAC0680168405CD4E97D
:100EA00001219047206A401C2062281EA5F10105FF
:100EB000DCDC07E0D4E9012118F8010B9047206A37
:100EC000401C2062381EA7F10107F3DC2046FFF723
:100ED000BBFA032011B041E62DE9F04F04460D4660
:100EE000D21D22F0070089B0D0E900974846394664
:100EF0000CF0E8FB0246F80F01D02D2307E0206834
:100F0000810701D52B2302E0202101EAC0038DF8DF
:100F100020300BB1012000E00020032A824601D0DE
:100F2000072A04DB2946204600F0D6F93FE1207865
:100F3000800601D40D2500E0E569C7F30A560D2DA2
:100F400049DA00214FEA175B08464FF00000002FF6
:100F500000F4400007DA00EB80004FF4400100EBA2
:100F6000D07001EA60008115012901DD4FF0FF31E9
:100F700000224FEA850CBCF1180F06D31346ACF1E2
:100F800018004FF08052C24003E04FF4801323FA60
:100F90000CF30CF10C0CBCF1200F04D3ACF1200CC1
:100FA00009FA0CF001E007FA0CF000294FF00048B4
:100FB00001DD18B90FE00ED140450CD319EB020941
:100FC0005F4121B9404502D19F4329EA0209BBEBA9
:100FD000175F00D0761C2088000502D57B48784436
:100FE00002E07A487844193808AA302302F80A3017
:100FF000037C0AF10101002E0AF1020A53546A46E9
:1010000002DC4FF0300101E04FF031014FF00108F8
:101010008DF8001002D0A6F2FF3603E059EA47012E
:1010200000D06B4E002D02DC2178090704D54FF06B
:1010300002082E218DF80110C44600210BE0C7F3F1
:1010400003433F01C35C491C6D1E02F808300529AB
:1010500008F1010801DA002DF1DC00210CE000EBC1
:101060001973491C1B786D1E082902F808304FEAD5
:10107000091908F1010801DA002DF0DC21688B065E
:1010800002D516E0A8F10108E04505DD02EB0803F2
:1010900013F8013C302BF5D0B8F1000F09DD02EB5D
:1010A000080313F8013C2E2B03D1090701D4A8F142
:1010B0000108002D05DD3E2102F808106D1E08F123
:1010C0000108407C002E02F8080008F1010804DA4B
:1010D0002D20764202F8080002E02B2002F80800DA
:1010E0000A214FF47A70864208F101080BDB96FB67
:1010F000F0F3303302F8083096FBF0F308F1010802
:1011000000FB136601E0642E0CDB642096FBF0F319
:10111000303302F8083096FBF0F308F1010800FBC9
:10112000136601E00A2E06DB96FBF1F0303002F880
:10113000080008F1010896FBF1F001FB1060303067
:1011400002F80800A16908F1010808EB050202EBAA
:101150000A00081AA0612078C00602D42046FFF7D2
:101160005DF9216A08AE01EB0A00206204E0D4E9CF
:10117000012116F8010B9047BAF1010AF7D2207845
:10118000C00602D52046FFF749F96E4609E016F879
:10119000010B3E280FD0D4E901219047206A401C62
:1011A0002062B8F10108F2D22046FFF74DF909B0EC
:1011B0000320BDE8F08F206A2844206203E0D4E9D0
:1011C0000121302090476D1EEBD3F8E7CAD0000014
:1011D00002FCFFFF10B5436913B1AFF3008001E0DB
:1011E000FFF755F9012010BD127800F124010A70B3
:1011F00000224A700122EDE711684FF0FF32E9E763
:1012000010B5436913B1AFF3008001E0FFF7D6F9E1
:10121000012010BD128800F1240182840022C284C2
:101220000122EDE711684FF0FF32E9E72DE9F041C7
:1012300016460C46054600F043F8036893F8010192
:10124000012807D0FF2C12D8185D80B101202C7026
:10125000BDE8F081D3F807013246214603F20713B7
:10126000C7182846BC46BDE8F041002360474FF050
:10127000FF30EDE7754600F0EBF8AE460500694635
:10128000534620F00700854618B020B5FFF762F8F6
:10129000BDE820404FF000064FF000074FF0000877
:1012A0004FF0000BAC46ACE8C009ACE8C009ACE8B4
:1012B000C009ACE8C00921F007018D467047000065
:1012C00010B500F005F8001D10BD00BF65C400009A
:1012D00000487047F40100202DE9F0411F46044604
:1012E00003260168072A01F4006004DB08B116A593
:1012F00005E016A503E008B115A500E015A521F04D
:1013000010002060A069C01EA0610FB1401EA06146
:101310002046FFF783F84FB1D4E9012138469047C2
:10132000206A401C2062C01C206206E0206AFAE7A6
:10133000D4E9012115F8010B9047761EF8D220461A
:10134000FFF782F8BDE8F0814E414E006E616E00FD
:10135000494E4600696E66002DE9F0478146164603
:101360008AB0354878440DC88DE80D00324878447D
:10137000801C03AC0DC884E80D0041F69B30084486
:10138000372190FBF1F290FBF1F5A5F1800501FB0F
:1013900012041B3C02D56442012000E00020DFF86B
:1013A00098A080460027FA44AAF1BE0A0EE0E007A2
:1013B0000AD03246684607EB470101230AEB810158
:1013C0000CF049F88DE8070064107F1C002CEED16A
:1013D000194F7F44AE3F19E0E80715D007EB041022
:1013E0000DF1180A90E80E008AE80E00C068F0427D
:1013F00001D1981908903246012306A903A80CF0E0
:101400002AF803AB83E807006D10641C002DE3D1BC
:101410004FF0010332466946B8F1000F03A802D02D
:101420000CF004F801E00CF016F8C9E90001C9F865
:1014300008200AB0BDE8F087D4CD000010B50446FE
:10144000AFF300802046BDE81040FEF754BF000017
:1014500000487047D401002030B44FF0013C50F8F0
:10146000042B51F8043BCCFA52F4D51A20D1FCB924
:1014700050F8042B51F8043BCCFA52F4D51A17D18A
:10148000B4B950F8042B51F8043BCCFA52F4D51AF5
:101490000ED16CB950F8042B51F8043BCCFA52F43D
:1014A000D51A05D1002CDAD030BC4FF000007047BF
:1014B00029BAB1FA81F111F01801D1F1200084406C
:1014C000F2D1CA40CB4012F0FF0213F0FF0330BC50
:1014D000D01A70477047000001491820ABBEFEE7E4
:1014E0002600020053EA020C00F069802DE9F04B5F
:1014F0004FF00006002B1FBFB3FA83F503FA05F483
:1015000024FA05F65E4012BF1643B2FA82F502FADB
:1015100005F4C5F120051EBF22FA05FC44EA0C04BF
:10152000203556EA044C4FEA144418BF641C4FF0AF
:1015300000084FF00009904271EB030C39D30029E9
:1015400019BFB1FA81F701FA07F6B0FA80F700FA8D
:1015500007F6C7F120071EBF20FA07FC46EA0C0673
:101560002037B6FBF4FCA7EB0507103F07F01F0B75
:10157000CBF120062CFA06F60CFA0BFB44BFB3465F
:101580000026202FA4BF5E464FF0000B5BEA060C3E
:1015900008BF4FF0010B19EB0B0948EB0608ABFB3A
:1015A000027C06FB02CC0BFB03CCC01B71EB0C01D5
:1015B000C1E70B46024641464846BDE8F08B13B5ED
:1015C000084318BF4FF0FF300146AFF30080BDE87D
:1015D0001C407047032A40F2308010F0030C00F0EA
:1015E000158011F8013BBCF1020F624498BF11F85D
:1015F00001CB00F8013B38BF11F8013BA2F1040216
:1016000098BF00F801CB38BF00F8013B11F003038D
:1016100000F02580083AC0F0088051F8043B083AF1
:1016200051F804CBA0E80810F5E7121D5CBF51F893
:10163000043B40F8043BAFF30080D20724BF11F80D
:10164000013B11F801CB48BF11F8012B24BF00F872
:10165000013B00F801CB48BF00F8012B704710B5E3
:10166000203AC0F00B80B1E81850A0E81850B1E85B
:101670001850A0E81850203ABFF4F5AF5FEA027C9A
:1016800024BFB1E81850A0E8185044BF18C918C0CA
:10169000BDE810405FEA827C24BF51F8043B40F86B
:1016A000043B08BF7047D20728BF31F8023B48BF50
:1016B00011F8012B28BF20F8023B48BF00F8012B8E
:1016C00070474FF000020429C0F0128010F0030CA4
:1016D00000F01B80CCF1040CBCF1020F18BF00F825
:1016E000012BA8BF20F8022BA1EB0C0100F00DB8D4
:1016F0005FEAC17C24BF00F8012B00F8012B48BF32
:1017000000F8012B70474FF0000200B513469446D5
:101710009646203922BFA0E80C50A0E80C50B1F149
:101720002001BFF4F7AF090728BFA0E80C5048BF5D
:101730000CC05DF804EB890028BF40F8042B08BFFB
:10174000704748BF20F8022B11F0804F18BF00F8F7
:10175000012B7047FEE70000002070470020704713
:1017600041F66830C2F20000D0F8D41200EB8101DB
:10177000D1F8C00298B140F65862C2F2000201F5F9
:101780003071C0F80822096800220029C0F8102230
:101790001EBF40F25860C2F20000C1F804020020EF
:1017A000704700002DE9F04188B004460E684FF6FE
:1017B000FC6576A0CFF6FC6506F022F82068A8420A
:1017C00066D1082E67D3E088864264D1A1880029BB
:1017D00000F09480022940F0D480102E5BD3207B4F
:1017E00041F65835C2F200052871A068617B286077
:1017F00042F2EC60C2F200004FF0010840F61846D9
:1018000080F80080C4F202064FF400306971306045
:1018100025208DF80C008DF818104FF4803703A8A0
:101820000121376001F096FB06A8012101F092FB2F
:101830003020C6F800808DF80C0003A80121376025
:1018400001F088FB2846052101F084FB2A20C6F818
:1018500000808DF80C0003A80121376001F07AFBAD
:101860002846052101F076FBC6F80080E8782F793C
:1018700029786A78AB786D79CDE900074EF2BD30F2
:10188000C0F60000029505F0BBFF0220306002E0C8
:1018900043A005F0B5FF41F66830C2F20000D0F871
:1018A000D41200EB8102D2F8C01219B302F53072E3
:1018B000C1F804421168E9B1027CD0F8C802D1F83D
:1018C00004324027002A4FF0000208BF4FF400778F
:1018D000C0F88C228279C0E9A1370127012AA0F83B
:1018E000787204BFC0F89432012200F51E710068BE
:1018F00005F030FB002008B0BDE8F0811028CAD107
:10190000208961890130A289484380B282423AD15C
:1019100047F61820C1F6FF70006847F610210590C1
:1019200047F61420C1F6FF70C1F6FF710068096820
:101930004022CDE9031003A806A903F0E5FF43F216
:101940000C46C2F20006308801097E2911D842F601
:101950000C420699C2F20002131815500122996038
:101960000121C0F210029981002110305A60997350
:10197000308080B200F03CF800288CD1002030800C
:1019800089E713A085E70CA083E700BF5365726960
:10199000616C206D7367206465636F64652E0A0057
:1019A0004D6573736167652070726566697820653F
:1019B00072722E0A00000000496E76616C69642024
:1019C00072657175657374206D73672E0A0000006F
:1019D0004D6573736167652074797065206F7574E8
:1019E000206F662072616E67652E0A0000207047C6
:1019F00041F66831C2F20001D1F8BC22D2F81422BB
:101A0000002A1CBF01207047D1F8D42201EB8202CA
:101A1000D2F8C032A3B302F5307C42F60C42C2F2D7
:101A20000002C3F80822DCF80020C3F810023AB321
:101A3000D2F8140200284FF0010018BF7047C2F816
:101A40001402D2F81032D1F8C802D2F808C28B6260
:101A500040F20112014621F8382F0022C264827937
:101A6000C0F844C0012A836404BFC0F854C00122F6
:101A700080B5006805F06EFA0020BDE88040704730
:101A800003207047F0B581B0044600680D46C66873
:101A90000769BA070AD516F0020107D0406B29463C
:101AA0000BF05CF920686FF00201016179070BD53A
:101AB00016F0040108D0806B691CC9B20BF04EF916
:101AC00020686FF00401016139070BD516F0080199
:101AD00008D0C06BA91CC9B20BF040F920686FF0A8
:101AE00008010161F9060BD516F0100108D0006C51
:101AF000E91CC9B20BF032F920686FF010010161E6
:101B000001B0F0BD7047000080B54FF4804000F098
:101B1000A5F94FF40040BDE8804000F09FB90000F7
:101B200043F61440C4F201000168490744BF042190
:101B30000160704770B581B00022009290F83C209F
:101B4000012A01D102218FE00E6801220A2E80F8BD
:101B50003C2009D3B2B25200D0F800E012FA86F26B
:101B60001E3A0EF10C0305E0D0F800E006EB460249
:101B70000EF110034FF0070C1D680CFA02F4A54398
:101B80001D608D681C6805FA02F222431A604968DC
:101B900006290ED801EB81014A1F71461F2351F817
:101BA000345F934025EA03030B60B3B203FA02F2F9
:101BB00013E001EB81030C29B2B204D8714651F84D
:101BC000304F233B03E0714651F82C4F413B1F251A
:101BD0009D4024EA05059A400D600B6842F2043CE2
:101BE000C4F2010C1A43ACF541739E450A6038D12A
:101BF000122E06D1DCF8001041F48001CCF8001060
:101C00002FE026F0010110292BD1DCF80010102E56
:101C100041F40001CCF8001023D140F21C01C2F2C3
:101C2000000109684DF68362C4F21B32A1FB021267
:101C3000910C01EB810149000091009989B1009953
:101C400001390091009961B1009901390091009921
:101C500039B1009901390091009911B10099013908
:101C6000EAE7002180F83C10084601B070BD000092
:101C7000002804BF0120704710B586B00446006CF0
:101C8000002853D1216842F20012C4F20102002060
:101C900091420590049020D042F20000C4F201006D
:101CA00081423FD1002043F630010090C4F202018E
:101CB0004A6942F480724A614A6902F48072009271
:101CC000009A0090086840F004000860086800F07E
:101CD000040000900098072018E043F630010090BF
:101CE000C4F202014A6942F400724A614A6902F48C
:101CF00000720092009A0090086840F004000860AA
:101D0000086800F00400009000980620019003206D
:101D100002900020039040F60000C4F2020001A9E6
:101D200000F046FA0020606484F83C00206CC00695
:101D30003AD4206C41F202118843023042F204315D
:101D40002064C4F20101086820F4403008600A6889
:101D500094E809101A43D4F810E00A60416801239E
:101D600021F4807141604168C0F6007341EA0E21A0
:101D70004160416821F040714160416841EA0C01D5
:101D80004160816821F400618160E16882681143EB
:101D90008160A16A8268994222F0706282608268E2
:101DA00004D122F040510AE0012052E01143816049
:101DB000816821F040518160E16A8268114381604D
:101DC000816821F0020181608168227E94F82030D0
:101DD00041EA42018160416883B141F400614160A0
:101DE00041684EF2000221F460414160616ACFF621
:101DF000FF72436802EB4131194301E021F40061B5
:101E00004160C16A40F2000C21F47001C162E269D4
:101E10006169CFF6F07CC36A0CEB02521A43C262CE
:101E2000826822F40072826094F83020836843EA6A
:101E300042228260826822F480628260826842EA82
:101E40008121816000206064216C012262F3010124
:101E50002164002184F83C1006B010BD2DE9F04F3C
:101E60008DB043F61441C4F201010A68024200F049
:101E70007D81B0F5804F086000F09080B0F5004F94
:101E800040F07481762040F618448DF80400002755
:101E9000C4F202044FF4801501A801218DF82470CA
:101EA000256001F057F809A8012101F053F8102628
:101EB000AD20266025608DF8040001A8012101F005
:101EC00049F809A8012100F0ABFE02202660CDE907
:101ED0000177ADF804009F208DF830000CA8012197
:101EE000CDE90777CDE90577CDE90377256001F0E6
:101EF00031F809A80C2100F093FE2660BDF82400FB
:101F00009FEDA71AC0BA00EE100ABDF82600B8EE81
:101F1000C00AC0BA02EE100ABDF82800B8EEC22A04
:101F2000C0BA20EE010A22EE011A02EE100ABDF834
:101F30002A009FED9C3AC0BA8DED040A00EE100A0B
:101F4000BDF82C00B8EEC22ABDF82E108DED021A95
:101F500022EE031AC0BA8DED031A01EE100AC8BAB8
:101F600002EE100A9FED903AB8EEC22A22EE032A42
:101F70009FED8E3AB8EEC00AB8EEC11A21EE031AF0
:101F800020EE030A01A88DED051A8DED062A8DEDD0
:101F9000070A01F0ABFD0DB0BDE8F08F40F6184721
:101FA000C4F202074FF400303860072001AC8DF80E
:101FB00004004FF48036204601213E60012500F0E8
:101FC000C9FF09A8012100F02BFE3D609DF8248087
:101FD0005FEAC86006D45FEA886016D45FEA4860AA
:101FE0002AD4C1E027208DF8040010208DF82400A9
:101FF00001A801213E6000F0ADFF09A8012100F019
:10200000A9FF3D605FEA8860E8D527208DF80400CD
:1020100020208DF824004FF48030386001A8012181
:10202000012500F097FF09A8012100F093FF3D6012
:102030005FEA486040F1988042F2EF6B261D4FF452
:1020400080394FF0010A09ADC2F2000B5FEA486027
:1020500055D500BF61208DF8040020460121C7F846
:10206000009000F077FF5846202100F0D9FDC7F816
:1020700000A09BF800103FA005F0C2FB9BF80010E9
:1020800021B141A005F0BCFB27E000BF47F61820B6
:10209000C1F6FF70006800210B9047F61420C1F6CE
:1020A000FF700068C6E900110A9047F61020C1F6DB
:1020B000FF700068C6E9021131617161B1614FF0D2
:1020C00001110191099028460CA9202203F01CFC63
:1020D0000C980390204601F009FD27208DF804009C
:1020E00040208DF8240020460121C7F8009000F020
:1020F00031FF2846012100F02DFFC7F800A017206E
:102100008DF8040020460121C7F8009000F022FF5E
:102110002846012100F084FDC7F800A09DF82400A6
:10212000C00715D107208DF8040020460121C7F80B
:10213000009000F00FFF2846012100F071FDC7F864
:1021400000A09DF824805FEA48603FF583AFD6E7A2
:10215000E2208DF804004FF48030386001A801219E
:10216000012400F0F7FE3C60022038600DB0BDE8AD
:10217000F08F00BF4D6173736167652020636F64EA
:10218000653A25752E0A0000496E76616C696420F7
:10219000574C20636F64653A25752E0A00000000D5
:1021A00000000039000000B958A08B3958A08BB945
:1021B0002DE9F04F82B000F13E4707F1FF77860529
:1021C00046EA972741F60046C4F20206082243F683
:1021D000004EB04208BF0722C4F2010E072F38BFDD
:1021E0003A46002600274FF00008009209E000BFA1
:1021F00008F101080437B8F1100F06F1020600F0EB
:10220000A3800D68012202FA08F415EA0409EFD050
:10221000D1F804B003220BF0030CACF10105B2407D
:10222000012D6FEA020A0FD88268CD6802EA0A021D
:10223000B5402A4382604268A243CBF3001404FAFB
:1022400008F42243426005E0BCF1030F02D14FF0D5
:10225000030C1EE0C2688C6802EA0A02B440224302
:10226000BCF1020FC26014D16FF0030202EA5802FF
:102270000244D2F820C007F01C040F230D69A340CC
:102280002CEA0303A5402B431362D1F804B00BF0F2
:10229000030C02680CFA06F302EA0A021A431BF462
:1022A000403F0260A4D0002243F644030192C4F2EE
:1022B00002031A684FF6084C42F480421A601A680A
:1022C000CFF6FF7C02F480420192019A28F00302CB
:1022D000724452F80C3007F00C050F24AC40A343B5
:1022E000009C04FA05F52B4342F80C30DEF8082078
:1022F0004B6842EA090543F60C4CDC0258BF22EA5F
:102300000905CEF80850C4F2010CDCF800209C024C
:1023100042EA090558BF22EA0905CCF80050DEF868
:1023200004209C0342EA090558BF22EA0905CEF8B9
:102330000450DEF80020DB0342EA090558BF22EA18
:102340000905CEF8005053E702B0BDE8F08F000059
:1023500010B5014641F62870C2F20000D0F8E04402
:1023600079B194F89C02032818BF10BDD4F8B802C4
:10237000826992B300232046C4F8D432BDE81040ED
:102380001047D4F89402032827D1D4F85811B4F890
:102390006001814222D9D4F86421D4F8C832091AE4
:1023A00002EB000CC4F85811C4F864C1814288BF24
:1023B00008469A7903F515710024012AC3E998C0EB
:1023C000C3F86842A3F854422DD118680122C3F81B
:1023D00070C2BDE8104004F0BDBD10BD94F89C0271
:1023E000032808D1D4F8B802016921B10020C4F84B
:1023F000D402204688470420C4F89402D4F8C83296
:102400004FF480709A79194621F8140F0024012A9C
:102410001C625C629C6206D1186801221C63BDE8E4
:10242000104004F097BD1868BDE8104004F092BD5C
:102430002DE9F04782B041F62870C2F20000D0F8D2
:10244000E09490F89C4409F2AA2889F8AA4290F8EE
:102450009D5489F8AB5290F89EA490F89F144AEAD4
:102460000122A9F8AC2290F9A0C490F8A1745FFAF7
:102470008CF141EA0726A9F8AE62B0F8A234012037
:10248000A9F8B032C9F8940204F01F000228C9F874
:10249000983211D0012825D0C8BB14F0600042D07A
:1024A000402801D020284CD1D9F8D40209EB800073
:1024B000D0F8B80282680FE014F060006BD04028BA
:1024C00001D020283DD1D9F8B80282680020002A26
:1024D000C9F8D40200F0A0834846414602B0BDE8E6
:1024E000F047104714F0600018BF402818D199F841
:1024F0009C020138022898BFBCF1010F5FD920E08F
:10250000802104F0A5FCD9F8C802002103E0D9F825
:10251000C80204F0800102B0BDE8F04704F098BCA6
:102520002028E4D00DE0092D0BD8DFE815F00D00D0
:10253000AD000A00CD000A00D8001D010A003601D6
:102540005E01D9F8C802DBE799F89C02013802283D
:10255000F7D8022BF5D1D9F8A4020321002808BF2F
:10256000012149F80C1F0220C9F88802D9F8BC32B1
:102570004FF480721946C9F81890C9E9020021F891
:10258000142F9A790027012A5862C3F820909F627D
:1025900000F0268183E2E5B3012D62D0032DD0D176
:1025A00099F89C02032861D110041CD111F07F001E
:1025B00019D0C3B9D9F8C80204F04AFC13E0D9F81D
:1025C000B8028268002A00F027830020C9F8D402EC
:1025D000484641469047B9F8B012002940F01C83A4
:1025E000002840F019830420C9F89402D9F8C832B1
:1025F0004FF480701946002721F8140F1F629A7952
:102600005F62012A9F6240F04A82186801221F63BC
:1026100046E299F89C02032800F01781022808BFBF
:102620005FEA41607FF48DAF022049F8140F4B46FA
:10263000BCF1000F58BF03F5A073002603F80E6F1E
:10264000C9F88002D9F8B4724FF480723946C9F8DB
:102650001030C9F8040021F8142FBA793B6278626F
:1026600066E199F89C02032800F0218102287FF49A
:1026700068AFD9F8C8024A063FF442AF04F0E8FB5D
:10268000D9F8C802802146E799F89C02013802284F
:102690003FF657AF90B2012840F0BE8200230420DD
:1026A000C9F8A432C9F89402D9F8C8724FF48070FE
:1026B000BA79394621F8140F012A3B627B62BB626A
:1026C00000F03A813868EBE190B2022800F00B810B
:1026D00001287FF436AF0120C9F8A40283E7002E59
:1026E00008BF002B7FF42DAF90B27F283FF629AFB3
:1026F00099F89C0203283FF424AFD9F8C80289F85E
:102700009EA290F89414012913D080F811A00168BA
:102710000AF07F03D1F8002822F4FE62C1F80028F5
:10272000D1F8002842EA0312C1F80028002180F8FD
:1027300094140421C9F894124FF48072014621F8D0
:10274000142F11F80E2C0023CB600B61012A4B6172
:1027500004BF03630122006804F0FCFBBAF1000F20
:102760000CBF0120022075E10020ADF80600B9F889
:10277000AC024FF0FF3101EB1021062900F2F2818B
:10278000DFE811F00700DE00EB00F001F001F800D7
:102790000401D9F8B4020268BBE1012B7FF4D1AE89
:1027A00099F89C02411E022980F0A880002049F877
:1027B000080F0221C9F88C12D9F8C03201274FF452
:1027C00080721946C9F81C90C9E9037721F8142FC3
:1027D0009A79C3F82090012A5F62986240F05F8185
:1027E00018680122C3F830905AE140F23425C2F251
:1027F0000005BAF1020F85F800A0BFF4A2AE99F867
:102800009C02032800F0D080022840F0FC80BAF13E
:10281000000F3FF4E8AED9F8B802C9F804A00028C8
:1028200000F001810268484651469047002800F0B8
:10283000FA80D9F8C802802104F00AFBD9F8C8024E
:10284000002104F005FB022004E101F00F0000EB81
:102850008000BCF1FF3F09EB8000D4BF90F823005B
:1028600090F8630100283FF46CAE01F07F0000EBAC
:10287000800009EB800000F11402BCF1FF3FC8BFEB
:1028800000F5AA72480631D0D9F8C8020CF07F01D1
:1028900001EBC10100EB810000F25621BCF1000FF9
:1028A00048BF00F11601087800B301201FE01004B2
:1028B00040F0B281480600F09181D9F8C8120CF0BE
:1028C0000F020879824200F2898102EBC20001EB1B
:1028D0008003BCF1FF3F40F3E88003F5157000274B
:1028E00083F85572E5E089F8A0727CE600209073C9
:1028F000022002F10E03C9F8940208E003287FF4D5
:1029000020AE022009F10403C9F894020120D9F88D
:10291000C8724FF480723946C9F82430C9F81400DF
:10292000C9F8180021F8142FBA79002678623B62A2
:10293000012ABE627FF4C6AE386801223B63AFE075
:1029400099F81010D9F8B80200290CBF816AC16A41
:102950000DF106008847022124E0C0B2052800F2EC
:102960000181DFE800F003C2C6CACED2D9F8B402B2
:102970004268CDE099F81000002840F0F380D9F8C3
:10298000B802416B0DF106008847C7E099F81000C6
:10299000002840F0E780D9F8B802016B0DF106007D
:1029A000884707214170B9E0BAF1000F57D0D9F834
:1029B000040050453FF417AED9F8B8124A68C1B2C6
:1029C00048469047D9F8B80229780028C9F8041079
:1029D0003FF409AE02684846904700283FF403AE32
:1029E000D9F8C802802104F033FAD9F8C8020021CE
:1029F00004F02EFAD9F8B80299F804104268484653
:102A00009047022026E0D9F8C802802104F020FA7D
:102A1000D9F8C802002104F01BFAD9F8B8022978C5
:102A2000426848465AE50420C9F89402D9F8C80219
:102A30004FF48072014621F8142F8279002303623B
:102A40004362012A836204BF03630122006804F029
:102A500081FA032089F89C0202B0BDE8F0870220C9
:102A600089F89C02D9F8B802002142684846C9F8A2
:102A700004A0002490470420C9F89402D9F8C83271
:102A80004FF480709A79194621F8140F012A1C62BC
:102A90005C629C6203D1186801221C6300E0186824
:102AA00002B0BDE8F04704F055BA012703F1140065
:102AB0005F7591F894740023012F8370027000F009
:102AC0008D8047780B685201012F1A4472D1D2F8D9
:102AD000003923F40013C2F80039007900F0FE0039
:102AE000022878D102F5106071E0D9F8B40282684A
:102AF0000EE0D9F8B402C2680AE0D9F8B40202695B
:102B000006E0D9F8B402426902E0D9F8B402826959
:102B100042B399F810000DF106019047B9F8B022C0
:102B20006AB3BDF80610E9B1914238BF0A460221E6
:102B3000ADF80620C9F89412D9F8C832C9E90522BF
:102B40005A629A794FF480771946C9F8240021F81F
:102B5000147F0027012A18629F6225D11A68186322
:102B600010461FE0D9F8C802802104F071F9D9F8A5
:102B7000C802002104F06CF902B0BDE8F08704201F
:102B8000C9F89402D9F8C8324FF480709A7919467E
:102B900021F8140F0027012A1F625F629F6203D190
:102BA00018681F63012200E0186804F0D3F902B02E
:102BB000BDE8F087D2F8003B23F40013C2F8003BD5
:102BC000007900F0FE00022805D102F530600268AD
:102BD00042F080520260002081F894040420C9F879
:102BE0009402D9F8C8024FF48072014621F8142FDC
:102BF0008279002404624462012A846204BF04636F
:102C00000122006804F0A6F9D9F8B802C9F8D44244
:102C10008268002A7FF460AC02B0BDE8F087000053
:102C200070B582B042F20C45C2F2000595F8512011
:102C3000012A40F03281002800F02F816C6843F2B5
:102C4000104EB4F5827FC2F2000E6DD1AA68002A40
:102C50006AD1042285F85120DEF8004095F8512011
:102C6000042A02D0012A40F0188195F85020012A48
:102C700000F01381012285F8502095F8512000239F
:102C8000042A1CBF052285F851206B65A863E987DB
:102C9000A9872863E9862A68A9862B646B64136870
:102CA0005B0603D4136843F040031360EB68B3F58D
:102CB000006F40F0A2800129844608D184463CF888
:102CC000023BD360C5F830C0EB8E013BEB8601239D
:102CD00005E000BFDEF80010A14240F0C480E98E9C
:102CE00019B9E98F002900F0DA80916889070CD5BD
:102CF000E98E51B1012B08D13CF8021B0023D160B1
:102D0000C5F830C0E98E0139E9869168C907E1D07C
:102D1000E98F0029DED0D168012320F8021BA863C7
:102D2000E98F0139E987D5E7DEF8002095F85030C2
:102D3000012B00F0B280012385F85030042385F880
:102D4000513000236B65A863A987E9872B63AB86A5
:102D5000EB86D5F808C02968BCF5004F2B646B647E
:102D600007D10B6823F040030B600B6823F480430A
:102D70000B600B685B0603D40B6843F040030B60E9
:102D8000EE68EB8F46B91BE0CB6820F8023BA863E6
:102D9000EB8F013BEB87EB8FEBB18B68DB07F3D15C
:102DA000DEF8003093425ED1EB8F002BF5D112E0BC
:102DB0000B7B00F8013BA863EB8F013BEB87EB8FAC
:102DC0004BB18B68DB07F3D1DEF8003093424AD178
:102DD000EB8F002BF5D1B4F5827F0CD1BCF5004F01
:102DE00002D0BCF5806F46D10868BCF5806F20F03A
:102DF000400008603FD101203EE00129844608D10F
:102E000084461CF8013B1373C5F830C0EB8E013BC0
:102E1000EB86012304E000BFDEF80010A14222D1BE
:102E2000E98E09B9E98FD1B3916889070CD5E98E8C
:102E300051B1012B08D11CF8011B00231173C5F8F7
:102E400030C0E98E0139E9869168C907E4D0E98F7D
:102E50000029E1D0D168012300F8011BA863E98FA4
:102E60000139E987D8E7012085F85100002085F86D
:102E7000500002B070BD8020002102F0A9FD28B1F1
:102E8000686D40F02000686520206865012085F8A5
:102E90005100002085F85000686D02B070BD02201E
:102EA0000121224602F094FD30B1686D40F020000F
:102EB000686520206865D9E740F21C00C2F2000076
:102EC000006849F68171C1F25E61A0FB0101480D05
:102ED0004FF47A71484301906868B0F5827F12D14F
:102EE00080200021224602F073FD0028DDD1A86871
:102EF0000028CBD1002000902868C168009180682C
:102F000000900098C2E7286801990029EFD0019944
:102F10000139019181680906E9D501990029E6D0B6
:102F200001990139019181680906E0D501990029CB
:102F3000DDD001990139019181680906D7D5019940
:102F40000029D4D001990139019181680906DBD4A7
:102F5000CDE7000070B582B043F2104C42F20C4550
:102F6000C2F2000CC2F20005DCF8006095F85130A6
:102F7000012B40F0808000287DD095F85030012B47
:102F800079D0012385F850300323002285F8513091
:102F90006A652863A986E986AA63AA87EA87AB6877
:102FA0002A64B3F5004F2B686A6407D11A6822F0CF
:102FB00040021A601A6842F480421A601A68520687
:102FC00003D41A6842F040021A606A680139EC685A
:102FD000B2FA82F2B1FA81F152094909B4F5006FEF
:102FE00041EA020111D131B130F8021BD9602863E6
:102FF000E98E0139E986E98E01B399688907F3D42E
:10300000DCF80010B142F6D010E031B110F8011B2D
:1030100019732863E98E0139E986E98E71B19968DF
:103020008907F3D4DCF80010B142F6D0012085F80E
:103030005100002085F8500002B070BD022001212F
:10304000324602F0C5FCC0B1686D40F020006865F2
:1030500020206865A86838B9002000902868C168F9
:103060000091806800900098012085F851000020B0
:1030700085F85000686D02B070BD40F21C00C2F2CD
:103080000000006849F68171C1F25E61A0FB010198
:10309000480D4FF47A71484301906868B0F5827F1B
:1030A00007D180200021324602F092FC0028CBD1CB
:1030B000D0E7286801990029CCD001990139019104
:1030C00081680906C6D501990029C3D00199013943
:1030D000019181680906BDD501990029BAD00199ED
:1030E0000139019181680906B4D501990029B1D04F
:1030F00001990139019181680906DBD4AAE7000032
:10310000002804BF012070472DE9F04387B0044632
:1031100090F83D00F8B1022084F83D002068211DA0
:1031200002F048FF012084F8460084F83E0084F84D
:103130003F0084F8400084F8410084F8420084F89D
:10314000430084F8440084F8450084F83D000020E2
:1031500007B0BDE8F083206840F6FF71C4F20001BB
:1031600088424FF0000184F83C100691CDE904112B
:10317000CDE9021179DC40F2FF71C4F2000188420E
:1031800000F3BB80B0F1804F00F0778140F2004146
:10319000C4F200018842BED1002743F630000197F7
:1031A000C4F202000169002541F0020101610169D8
:1031B000C4F2020501F00201019101990197016831
:1031C0000DF1080841F0010101600168022601F0DB
:1031D0000101019101990197016841F0020101602B
:1031E0000068414600F0020001900198C020029062
:1031F0002846CDE90367CDE90576FEF7D9FF032020
:1032000002A9C1C105F580604146CDE90576FEF70A
:10321000CFFF4EF60C50CEF2000000684FF0FF32A8
:10322000C0F3022080F00701042928BF04210338DD
:1032300002FA01F14FF0010338BF384623EA0101D9
:10324000814002FA00F023EA000008434EF21B41DD
:103250000001CEF2000188704EF20410CEF20000A0
:103260004FF0005140F8041C55E74FF6FF71C4F2CF
:103270000001884200F3A08041F20001C4F2000185
:10328000884200F0658141F20041C4F200018842A9
:103290007FF441AF002043F630010190C4F20201F7
:1032A0000A6942F020020A61096901F020010191D6
:1032B00001994EF60C51CEF200010968C1F30221CA
:1032C00081F00702042A28BF0422033938BF0146CF
:1032D0004FF0FF309040022222EA000088404EF278
:1032E0001B410001CEF2000108774EF20410CEF22D
:1032F00000004FF4000101600DE740F60001C4F248
:103300000001884200F0578140F60041C4F20001FC
:1033100088427FF400AF002543F630000195C4F2E7
:103320000200016941F008010161016901F0080131
:10333000019101990195016841F001010160006866
:1033400002A900F00100019001980F2002900220D4
:10335000CDE90305CDE905500020C4F20200FEF7D7
:1033600027FF4EF60C50CEF2000000684FF0FF32FF
:10337000C0F3022080F00701042928BF042103388C
:1033800002FA01F14FF0010338BF284623EA010198
:10339000814002FA00F023EA000008434EF21B418C
:1033A0000001CEF20001C8754EF20410CEF200000A
:1033B0004FF480210160AEE640F20041C4F2010109
:1033C000884200F04D810021C4F2010188427FF45F
:1033D000A2AE002543F630000195C4F20200416917
:1033E000012641F001014161416901F001010191B2
:1033F00001990195016841F010010160006802A97E
:1034000000F01000019001984FF4D4400290022087
:10341000CDE903050020C4F2020000F580500595B7
:103420000696FEF7C5FE4EF60C50CEF20000006880
:103430004FF0FF32C0F3022080F00701042928BFBB
:103440000421033802FA01F138BF284626EA0101B7
:10345000814002FA00F026EA000008434EF21B41C8
:103460000001CEF2000108704EF20410CEF200000E
:103470004FF0006140F8041C4DE6002743F6300091
:103480000197C4F202000169002541F001010161C8
:103490000169C4F2020501F001010191019901974E
:1034A00001680DF1080841F00101016001684FF069
:1034B000020901F0010101910199019701680126BA
:1034C00041F0020101600068414600F002000190F5
:1034D0000198202002902846CDE90397059706968B
:1034E000FEF766FE40F60840CDE9020905F580606A
:1034F0004146CDE904770696FEF75AFE4EF60C508B
:10350000CEF2000000684FF0FF32C0F3022080F0DE
:103510000701042928BF0421033802FA01F138BF4A
:10352000384626EA0101814002FA00F026EA00004E
:1035300008434EF21B410001CEF2000148704EF2EA
:103540000410CEF200004FF0805140F8041CE2E578
:10355000002043F630010190C4F202010A6942F0F2
:1035600010020A61096901F01001019101994EF6FA
:103570000C51CEF200010968C1F3022181F007026B
:10358000042A28BF0422033938BF01464FF0FF3018
:103590009040022222EA000088404EF21B410001C6
:1035A000CEF20001C8764EF20410CEF200004FF4C5
:1035B00080010160AFE5002543F630000195C4F2BB
:1035C0000200016941F004010161016901F0040197
:1035D000019101990195016841F0080101600068BD
:1035E00002A900F00800019001984FF47040029089
:1035F0000220CDE90305CDE905500020C4F2020008
:1036000000F54060FEF7D4FD4EF60C50CEF20000FF
:1036100000684FF0FF32C0F3022080F00701042958
:1036200028BF0421033802FA01F14FF0010338BF2B
:10363000284623EA0101814002FA00F023EA000053
:1036400008434EF21B410001CEF20001C8704EF259
:103650000410CEF200004FF0804140F8041C5AE5FF
:10366000002543F630000195C4F20200416941F0A3
:1036700002014161416901F0020101910199019545
:10368000016841F004010160006802A900F0040033
:10369000019001984FF4707002900220CDE903056B
:1036A000032006900020C4F2020000F5006005959A
:1036B000FEF77EFD4EF60C5CCEF2000CDCF800004E
:1036C0004FF0FF37C0F3022282F007030420042BDF
:1036D00028BF0346033A07FA03F34FF0010638BF49
:1036E0002A4626EA030303FA02F24EF21B431201B2
:1036F000CEF200034EF2041E5A74CEF2000E4FF4C6
:103700008051CEF80010DCF80010C1F3022181F0E6
:103710000702042A38BF1046033907FA00F038BF01
:10372000294626EA0000884007FA01F126EA01014D
:1037300008430001D8744FF48040CEF80000EAE45A
:1037400090F83C20012A4FF0020200F0C38080B5BF
:1037500080F83D20D0F800C04FF67772DCF80830D2
:1037600023EA0202CCF808200B684F2B28DC1F2B21
:1037700044DD202B45D0302B43D0402B40F0AC8093
:10378000D1F804E0C968DCF82030DCF8202022F011
:103790000102CCF82020DCF8182022F0F00242EAE6
:1037A000011123F00A0242EA0E02CCF81810CCF8FC
:1037B0002020DCF8081041F0470121F030017EE0C4
:1037C0006F2B26DDB3F5005F47D0B3F5805F78D06F
:1037D000702B40F08180D1E901E3C968DCF8082052
:1037E00043EA0E0322F47F4243EA01211143CCF85D
:1037F0000810DCF8081041F0770160E00BB1102BE5
:103800006AD1DCF8081021F07001194341F007017A
:1038100055E0502B34D0602B5ED1D1F804E0C9685C
:10382000DCF82030DCF8202022F01002CCF8202038
:10383000DCF8182022F4704242EA013123F0A002A1
:1038400042EA0E12CCF81810CCF82020DCF8081050
:1038500041F0670121F0100131E0D1E901E3C968CD
:10386000DCF8082043EA0E0322F47F4243EA0121F8
:103870001143CCF80810DCF8081041F480411EE038
:10388000D1F804E0C968DCF82030DCF8202022F010
:103890000102CCF82020DCF8182022F0F00242EAE5
:1038A000011123F00A0242EA0E02CCF81810CCF8FB
:1038B0002020DCF8081041F0570121F02001CCF85D
:1038C00008100022012180F83D10002180F83C10F2
:1038D000BDE88040104670470122F3E70168D1F847
:1038E0000CC00B699A0708D51CF0020205D06FF0D6
:1038F00002020A618A69002202775A0708D51CF081
:10390000040205D06FF004020A618A69002202777E
:103910001A0708D51CF0080205D06FF008020A61EA
:10392000CA6900220277DA0608D51CF0100205D019
:103930006FF010020A61CA6900220277D8071EBF21
:103940001CF001006FF001000861180605D51CF09D
:1039500080001CBF6FF080000861580605D51CF080
:1039600040001CBF6FF040000861980658BF7047C8
:103970001CF020001CBF6FF02000086170470000A1
:1039800090F83C20012A4FF0020200F0708010B540
:1039900080F83D200268D2F808C0D1E900E32CF09D
:1039A000770C23F0070444EA0C044FEA331344EA8B
:1039B0000E04072B4FF0010C946008D8DFE803F0E9
:1039C0004747474704091B2DBEF1050F32D101229D
:1039D00046E0D1F808E00969146A136A23F001038C
:1039E0001362936923F0F00343EA011124F00A0300
:1039F00043EA0E0329E0D1F808E00969146A136A62
:103A000023F010031362936923F4704343EA0131F6
:103A100024F0A00343EA0E1317E0D1E902E4096998
:103A2000936844EA0E0423F47F4344EA01211943D6
:103A300091600CE0136A146A24F001041462946922
:103A4000096924F0F00444EA011191611362D1681C
:103A500021F04001D160D16821F48041D160002281
:103A6000002180F83DC080F83C10BDE810401046B1
:103A700070470000FEE7000041F6D460C2F200008B
:103A800001684A6992072AD44A69520511D44A69E1
:103A9000920724D44A6952050BD44A6992071ED46E
:103AA0004A69520505D44A69920718D44A695205F1
:103AB000E7D50A6842F400720A606FF480624A61D6
:103AC00000212022016380F83D2080F83E10026C26
:103AD00042F00402026480F83C100120704700208C
:103AE00070470000FEE70000FEE70000F0B581B07F
:103AF00040F618450446C4F202054FF40030286031
:103B000007208DF801004FF480370DF101000121ED
:103B10002F600126FFF71EFA68460121FFF780F8A3
:103B20002E609DF80000C00709D0E1208DF802004A
:103B30000DF1020001212F60FFF70CFA2E60A0208A
:103B40008DF803000DF1030001212F60FFF702FA49
:103B500020462021FFF7FEF902202E60286001B0E8
:103B6000F0BD00002DE9F04F89B041F6287EC2F289
:103B7000000EDEF800B0DBF81400C00740F06287EA
:103B8000DBF81400DBF81810014200F05B87DBF86B
:103B90000808C0F30D20CEF8D404DBF81400DBF8DD
:103BA00018100840800705D5DBF8140000F002006B
:103BB000CBF81400DBF81400DBF818100BF50069E3
:103BC0000840C006584640F18C80DBF8180020F011
:103BD0001000CBF81800DBF82020C2F34340062881
:103BE00002F00F0141D00228584676D147F6F07016
:103BF00012EA0005584670D001EBC1000EEB8000C0
:103C000000F51873D0F860022A09042AC5F30117D9
:103C100047D34FF0FF3606EB9516032EC5F3811CF4
:103C200014D3AD0925F003054FF480545BF804600C
:103C3000043D06605BF8046046605BF804608660E3
:103C40005BF80460C66000F11000EFD1BCF1000F1A
:103C500027D04FF480555BF805600446BCF1010F96
:103C600044F8046B0FD120461BE04FF480505BF802
:103C70000030C2F30A12CEF89C345BF80000CEF894
:103C8000A004584620E05BF80560BCF1020F4660D6
:103C900001D1083005E04FF480565BF8066086607D
:103CA0000C3067B14FF480565BF80660012F067048
:103CB00005D0350A022F45701CBF370C8770186875
:103CC0008718DEF800001F6001EBC1010EEB8101D7
:103CD000D1F868321A44C1F86822816941F01001B4
:103CE000816141698269CDF818B011400903CDF8AE
:103CF000109040F16F81D0F81818D0F81C281140AE
:103D00000D0C00F0678143F20A090EF51D764FF4A1
:103D10003067C4F654794FF000081BE00BEB070046
:103D2000022181605FEA8A6042BF0BEB070020211D
:103D300081605FEA8A4042BF0BEB07004FF40051FD
:103D4000816008F101086D0807F1200706F12406DB
:103D500000F03C81E807F4D0DEF8000039188A68EA
:103D6000D0F8143803EA020A5FEACA726ED00BEB8D
:103D7000070201239360036C8A689EF80640012CB9
:103D800024D114072DD4940600F1BA8012F0280F24
:103D90005CD109F10104A34202D312F4004227D1FD
:103DA00032680969B7F5306F6FF3DF41A2EB0101AB
:103DB00046F80C1C41D1DEF86422002A00F0DE80B7
:103DC000DEF860020844CEF8600236E009F580743F
:103DD000A34210D110040BD4900644BF2020886069
:103DE0002BE009F10100834230D312F400402DD0C2
:103DF0004FF4004085E0B7F5306F1ED1DEF8641255
:103E0000D9B9016C494503D9D0F8001B002914D455
:103E10000021C0F8101BD0F8101B41F40021C0F89D
:103E2000101BD0F8101B41F01801C0F8101BD0F87F
:103E3000101B41F0C041C0F8101B5FFA88F0FEF77C
:103E400087FA41F6287EC2F2000E00BF5FEA0A70D0
:103E50005CD50BEB070008218160DEF8000009F15A
:103E6000010B046C384481685C4512D311F40041A5
:103E70000FD04FF400418160FEF7DAFA41F6287E58
:103E8000C2F2000E9EF80600DDF818B001280ED030
:103E90003CE0FEF7CDFA5C4541F6287EDDF818B02F
:103EA000C2F2000E32D39EF8060001282ED1DEF8B1
:103EB0000000016C494503D9D0F8001B002925D426
:103EC0000021C0F8101BD0F8101B41F40021C0F8ED
:103ED000101BD0F8101B41F01801C0F8101BD0F8CF
:103EE000101B41F0C041C0F8101B0EF29C41C0F8FD
:103EF000141BD0F8001B41F08021C0F8001B05E026
:103F0000202088605FEA0A70A3D400BF5FEACA601D
:103F100042BF0BEB0700102181605FEA8A707FF5DA
:103F200001AFDBF81400000604D50499486840F49A
:103F30008060486016F81D0C01287FF4EFAEDEF8B3
:103F4000E0040022D0F8D41206F81D2C00EB810109
:103F5000D1F8B81200293FF4E1AE90F89C22032A70
:103F60007FF4DCAE4A6A002A3FF4D8AE5FFA88F1EB
:103F7000904741F6287EC2F2000ECFE6016C49451B
:103F800004D9D0F8001B00293FF557AF0021C0F835
:103F9000101BD0F8101B41F40021C0F8101BD0F802
:103FA000101B41F01801C0F8101BD0F8101B41F095
:103FB000C041C0F8101B0EF29C41C0F8141BD0F891
:103FC000001B41F08021C0F8001B36E7DEF800003E
:103FD000DDF81090416982691140490340F1F08198
:103FE000D0F81818D0F81C2811401FFA81FBBBF13B
:103FF000000F00F0E58106984FF0000900F5106011
:1040000003900DE0D5F83408059A012191408843CA
:10401000C5F834085FEA5B0B09F1010900F0CC81B7
:104020005FEACB70F6D0DEF8000009F00F06D0F89A
:104030001018D0F8342800EB4913F240D201D2B264
:10404000D3F80839114301EA0304039DE1074FEA5D
:104050004918059600F0DD80049B0127596B07FA8B
:1040600006F29143596305EB08018F609EF8061034
:1040700001290AD109EBC9010EEB8101D1E907231E
:10408000B9F1000F1A440A621BD0DEF8E0645FEA5F
:10409000096045D096F89C02032840F0BA80D6F813
:1040A000B8024269002A00F0B4800020C6F8D402A9
:1040B0005FFA89F13046904741F6287EC2F2000E41
:1040C000A7E0DEF8241049BB016C43F20A02C4F6F3
:1040D0005472914203D9D0F8001B00291ED400214C
:1040E000C0F8101BD0F8101B41F40021C0F8101BC1
:1040F000D0F8101B41F01801C0F8101BD0F8101BAD
:1041000041F0C041C0F8101B0EF29C41C0F8141BD6
:10411000D0F8001B41F08021C0F8001BDEF8E064FD
:10412000D6F8940202286DD1B069318C884218D932
:10413000421A706AB2614318D6F8C8024FF4807709
:10414000014642628279736221F8147F002703627C
:10415000012A876204BF03630122006802F0FAFEAD
:1041600036E04FF000031ED1716981421BD3D6F8AF
:104170009802814217D2D6F8C8024FF480720146E5
:1041800021F8142F827903624362012A836204BFFB
:1041900003630122006802F0DDFED6F8C832002772
:1041A000C6F8987217E096F89C020022032807D1FF
:1041B000D6F8B802C16819B13046C6F8D42288478B
:1041C000D6F8C802802102F043FE0520C6F894020A
:1041D000D6F8C832002703F51571C3F86072C3F82A
:1041E00064729A79C3F86872A3F854721868012A45
:1041F00004BFC3F87072012202F0ACFE41F6287EC3
:10420000C2F2000E96F8A00200281CBF002086F81B
:10421000A002200742BF05EB080008218160E006EC
:1042200042BF05EB080010218160600642BF05EB2C
:10423000080040218160A0072CD50698494603F06C
:104240000DF841F6287EC2F2000E09EBC9000EEB14
:10425000800111F8170F012818D1DEF8E0040023BF
:10426000D0F8D4220B7000EB8202D2F8B8226AB1E7
:1042700090F89C12032909D1126A3AB15FFA89F1C8
:10428000904741F6287EC2F2000E00BF05EB080001
:104290000221816020067FF5BDAE09EBC9000EEB5F
:1042A0008005AC465CF8241FCDF81CC05CF8047F88
:1042B000B942FFF4AFAE2B4653F81C6FDEF800A0F6
:1042C0000893CB1BB34238BF1E4608EB0A03D3F852
:1042D00018490336A4B2B4EB960F04D25546B9423E
:1042E0003FF698AE8EE69EF80620DDF81C80CDF8ED
:1042F00004B003F5106005F1200B0AF580564FEA73
:104300000934CDF808A00EE0DCF800700AEB0301D8
:104310001F44CBF80010CCF800708169033389B2D8
:10432000B1EB930F40D3D8F80010B9423ED9089BA7
:10433000C91B1B68994238BF0B46DBF800A0002A56
:10434000E2D199B20029DFD003314FF0FF3707EBFC
:104350009107032F574612D38F0827F0030E5746B5
:10436000D7F80080BEF1040E44F806807D68A551A0
:10437000BD68A551FD6807F11007A551F0D1C1F343
:10438000810141F6287EDDF81C800029C2F2000E72
:10439000BAD03D6801293551B6D07D680229355122
:1043A0001CBFB9683151AFE7D8F80010DDE901B59D
:1043B000B9423FF62FAE25E6DEF80000DDF810909A
:1043C00041698269DDF818801140B1F1FF3F1BDCC3
:1043D000D9F8041021F00101C9F804109EF8CC149A
:1043E000012903D100218EF8CC1409E0DEF8E01495
:1043F00091F89C22042A04BF91F89D2281F89C2206
:10440000416901F00041416141698269114009053A
:1044100025D5D9F80810C9071DD0DEF8E01491F8A9
:104420009C22042A1CBF91F89C2281F89D22042220
:1044300081F89C22D0F8001E41F00101C0F8001E56
:104440009EF80B1039B14EF61051CEF200010A68F9
:1044500042F006020A60416901F40061416141696C
:1044600082691140C90440F11F81D9F8041021F07C
:104470000101C9F80410102102F0F0FE41F6287E77
:10448000C2F2000E9EF80400010600F0B480C1B232
:10449000042900F0030001D2002166E06FF0600201
:1044A00002EA411200234FF67F37002108EB030692
:1044B000C6F80879D6F80059803325F40015C6F8F7
:1044C0000059C6F8087BD6F8005B9A4225F400151F
:1044D000C6F8005BD6F8005B01F1040145F0006509
:1044E000C6F8005BC6F82879D6F8205925F40015DF
:1044F000C6F82059C6F8287BD6F8205B25F40015AD
:10450000C6F8205BD6F8205B45F00065C6F8205B56
:10451000C6F84879D6F8405925F40015C6F8405930
:10452000C6F8487BD6F8405B25F40015C6F8405B1A
:10453000D6F8405B45F00065C6F8405BC6F8687980
:10454000D6F8605925F40015C6F86059C6F8687B9E
:10455000D6F8605B25F40015C6F8605BD6F8605BA2
:1045600045F00065C6F8605BA0D1002843D008F58F
:10457000106202EB41134FF67F364F019E60D55912
:1045800008F5306325F4001503EB4111D5518E6019
:10459000D959012821F40011D951D95941F00061AC
:1045A000D95128D007F120015518AE60555802287E
:1045B00025F40015555003EB0105AE605E5826F456
:1045C00000165E505E5846F000665E5013D007F14C
:1045D000400011184FF67F378F60115821F40011F9
:1045E000115019188F60195821F4001119501958D9
:1045F00041F000611950D9F81C0040F00110C9F8D1
:104600001C009EF80F0040B1D9F8840040F00B0068
:10461000C9F8840009F1440008E0D9F8140042F216
:104620002B010843C9F8140009F11000016843F296
:104630000A0341F00B010160D9F80000C4F654737D
:1046400020F4FE60C9F80000DEF800009EF80610B5
:10465000026C9A4203D9D0F8002B002A20D4002201
:10466000C0F8102BD0F8102B012942F40022C0F81A
:10467000102BD0F8102B42F01802C0F8102BD0F8F5
:10468000102B42F0C042C0F8102B09D10EF29C4111
:10469000C0F8141BD0F8001B41F08021C0F8001BAB
:1046A000416901F480514161416982691140890485
:1046B00040F1E880D0F8001940F2FF729143C0F851
:1046C0000019D0F8041841F48071C0F80418D0F82B
:1046D000081801F0060289074FF0020158BF0F21A8
:1046E000002A08BF114602298EF8071012D140F2A5
:1046F0001C01C2F20001096845F24032CFF6277270
:1047000043F200530A44C0F20C039A420FD24FF412
:1047100070517AE0C268002922F47052C260C26807
:1047200042F41052C26078D072B600BFFEE741F684
:104730004062CFF61B7244F240230A44C0F20F03DA
:104740009A4202D24FF460515FE0A1F5740244F640
:104750008073A2F51052C0F212039A4202D24FF4B3
:10476000505152E0A1F183724DF22063A2F5E7426D
:10477000C0F213039A4202D24FF4405145E04BF28B
:104780006062CFF6E5624EF260330A44C0F216036F
:104790009A4202D24FF4305137E04DF20032CFF658
:1047A000CE6247F240730A44C0F21B039A4202D21F
:1047B0004FF4205129E045F6C032CFF6B36249F2FA
:1047C000C0130A44C0F221039A4202D24FF410519E
:1047D0001BE0A1F1B77247F22053A2F55852C0F284
:1047E00038039A4202D24FF400510EE045F2E04203
:1047F000CFF6596249F6E0430A44C0F241034FF450
:10480000C0519A4238BF4FF4E051C26822F470524E
:10481000C260C2681143C1600121DEF8E054012486
:104820002974002185F89C42C5F89412D5F8B80285
:104830006960C5F8A41285F8A01218B142680AB1DF
:1048400028469047D5F8C802002100224023402680
:1048500002F09CFAD5F8C80280210022402385F896
:104860006341A5F8606102F091FA41F6287EC2F238
:10487000000EDEF8000085F823402E84416901F423
:1048800000514161416982691140090716D5DEF87E
:10489000E01491F89C22032A0CD1D1F8B8224AB135
:1048A000D2693AB10846904741F6287EC2F2000E1E
:1048B000DEF80000416901F0080141614169826947
:1048C000114009062ED5D8F8181021F08001C8F83B
:1048D00018109EF80410022924D30EF27B2401251F
:1048E00003E000BF01358D421AD214F8240B0128D1
:1048F000F8D105F00F0000EBC0000EEB8002280697
:10490000DEF8000002F1140158BF02F5157102F043
:1049100029FC41F6287EC2F2000E9EF80410E1E761
:10492000DEF80000416982691140C90230D59EF865
:104930000410022928D30EF13B0408F51265012664
:10494000012705E0013724348F4205F1200519D2F3
:1049500028686278012AF5D1B0F1FF3FF2DC07F058
:104960000F0000EBC0000EEB8001DEF800001431F8
:10497000267002F0F7FB41F6287EC2F2000E9EF888
:104980000410DFE7DEF80000416901F480114161A5
:10499000416982691140890232D59EF80420022AB9
:1049A0002AD3DEF8D414013A0EF51F7308F53267E6
:1049B000012604E02433013A07F120071CD03D68AA
:1049C0001C78012CF6D1B5F1FF3FF3DC81EA1545E7
:1049D000ED07EFD103F8016CD8F8185045F08005C9
:1049E000C8F81850D8F814502D06E3D4D9F804109C
:1049F00041F40071C9F80410416901F400114161EA
:104A0000416982691140490003D5416901F0804143
:104A10004161416982691140490713D544686107C2
:104A20000DD5DEF8E024012182F89C12D2F8B812EC
:104A300029B14B6811791046754698472868416836
:104A40002143416009B0BDE8F08F000070470000CD
:104A50002DE9F04FEDB00446D0F8AC0111B90028B3
:104A600040F05386399438B100291CBFD4F898011E
:104A70005FEAD00B40F04C86D4F8A4110029084618
:104A8000019100F042863AA828300090A068D4E94D
:104A900000173590E068D4E92E9A3890E06A002338
:104AA0002E90A06A0E90606D1990206D2B90E06F93
:104AB0001690A06F1B90D4E928061590606B369075
:104AC000206B3290E06D2D90A06D2A90D4F8840078
:104AD0002390D4F880001190D4F8AC000C90D4F856
:104AE000A8000F906069379020693390E06B349094
:104AF000A06B3190606E2890206E2990D4F88C00C5
:104B00002190D4F888001F90D4F8B4001090D4F805
:104B1000B0000D90E0692790A0692490606C2C9003
:104B2000206C2290E06E2090A06E1E90D4E9240BA1
:104B30001A90606A2F90206A3090E06C2590A06CEB
:104B40002690606F1C90206F1D90D4F89C001790E9
:104B5000D4F898001890D4E93002CDE90A2000BFBB
:104B60002E98199A784050400E9A09932B9B0891E1
:104B700051401B9A59405140169A14965040464055
:104B80001598279A81EA000C2298249907974840A3
:104B90001E991A9F48402C9978405140209A80EAEB
:104BA0000907514081EA0B01700081EA0A0540EAD9
:104BB000DC714FEA4C0040EAD670A04687EA000458
:104BC00085EA01000A99029081EA00030B98CDE979
:104BD000045680EA0405C8E93053259A2F9B0394B4
:104BE00082EA03051C9A0D9C5540179ACDF848A0FF
:104BF000554085EA01082699309ACDF84CB081EAF3
:104C000002051D99DDF830B04D401899CDF8189087
:104C10004D4085EA0006319833991F9D80EA0102D4
:104C200029983799424034986A4080EA01032898CD
:104C300010994340219882EA040A434083EA010222
:104C40004FEA4A0444EAD27484EA0C0E54000599EF
:104C500044EADA7484EA0105049932984C0044EA83
:104C6000D7737F0047EAD17C3599369C41402A981A
:104C70004140389844402D9844402398444011982E
:104C800084EA0B0441400F986700414047EAD1791C
:104C90008CEA010C490041EAD47186EA01004FEA2E
:104CA000480183EA040788EA090441EAD6797600D4
:104CB00046EAD87686EA0A0389EA0201029E2F9A1A
:104CC000DDF818A072400A92259A8AEA030A724017
:104CD0000B921C9A72402592179A56402F96039E6B
:104CE000309A72400592269A724017921D9A72402D
:104CF0002692189A56403096079E84EA06022E9E07
:104D0000049284EA0602199E079284EA0602169E1D
:104D1000199284EA0602149E1D9266402E96089E01
:104D200080EA06020E9E149280EA06022B9E1692DC
:104D300080EA06021B9E189280EA0602159E1C92CB
:104D400070402B90389885EA000836986840159096
:104D50002D9868401B90239868402D9085EA0B00A1
:104D6000389035988EEA0005329880EA0E000E9051
:104D70002A9880EA0E002390119880EA0E00329063
:104D80000F9880EA0E003690379887EA000E349824
:104D900087EA000B289878402890219878402A903C
:104DA00010987840379033981E9F8CEA000931980C
:104DB0008CEA0006299880EA0C0021901F9880EA6E
:104DC0000C0033900D9880EA0C003590279883EA08
:104DD000070C81EA00022C981A9F81EA00042098AF
:104DE0005F4048402C901398299748403190129882
:104DF000149F484034902498229958405940399B38
:104E00001F60399B049F5F60399B9D60399BC3F88D
:104E10000C80DDF8E480C8E90602059808F1340248
:104E2000C8F820000A98C8E91014C8F82400169899
:104E3000A021C8F828000798C8E9049EC8F82C00EB
:104E40000E98C8F83000159882E841081798C8F8FD
:104E500048000B98C8F84C001898C8F850001998EA
:104E6000C8F854002398C8F858001B98C8F85C008C
:104E70002198C8F860002898C8E9190C2C98C8F83F
:104E80006C002698C8F870002598C8F874001C9823
:104E9000C8F878001D98C8F87C003298C8F88000DF
:104EA0002D98C8F884003398C8F888002A98C8F864
:104EB0008C002998C8F890003198C8F89400309870
:104EC000C8F898002F98C8F89C002B98C8F8A00044
:104ED0002E98C8F8A4003698C8F8A8003898C8F8E2
:104EE000AC003598C8F8B0003798C8E92D0A349856
:104EF000C8F8BC000098FCF706FC98E88F000DF19C
:104F0000E80CD8F81C408CE88F00D8E90801D8E9F3
:104F100005654EF2182BCDE94140439100204FF03A
:104F2000010E1821C0F6000BCDE93F65389181468E
:104F300000EB40004CF6CD4100EB4E00CCF6CC41EE
:104F4000A0FB013727F0030303EB9703C21A02EB20
:104F5000420000EB4900A0FB017626F0030707EBB7
:104F60009607C11B01EB41000B46369100EB420056
:104F7000342100FB01F73F0A07EB8707C01B74468B
:104F80009646C2B201463790500050FA81F043F283
:104F9000343100EB4300C3F23331A0FB017A09EB5B
:104FA00089070BEB870308EBC70153F8243015463C
:104FB000339201EBC40251F83410D2F8048003F0AC
:104FC0003F02C2F1200B08FA02F321FA0BF646EA7F
:104FD000030CB2F12006C2F1400358BF01FA06FCEF
:104FE00001FA02F6C3F1200221FA03F108FA02F2F3
:104FF00041EA020158BF0026BBF1000F58BF28FA52
:105000000BF141EA06023AA901EBC70646F8342043
:105010000AEB8A02A0EB020A0AEB4A0000EB450009
:105020004FF0340200FB02F24FEA122202EB82023E
:10503000A0EB020B5FFA8BF04FEA400252FA8BF2C0
:10504000329002EB4A0043F23432C3F233323590ED
:10505000A0FB022028FA03F2349058BF002206EB8E
:10506000C40142EA0C0239984A600EEB8E0100EB53
:10507000C1024EF21820C0F6000000EB810656F87F
:10508000296002EBC90352F839205B6806F03F063D
:10509000C6F1200703FA06F822FA07F040EA0800F2
:1050A000B6F12005DDF8E48058BF02FA05F002FAF7
:1050B00006F5C6F14006C6F1200422FA06F203FA0C
:1050C00004F442EA0402F446CE4658BF0025002FFD
:1050D00058BF23FA07F223FA06F30DF1E80958BF87
:1050E00000232A4309EBC101184301EBCE0341F829
:1050F0003E20DDF8D8E058604EF218230EEB8E000B
:10510000C0F6000303EB800308EBC00153F82C301A
:1051100001EBCC0251F83C10526803F03F03C3F19D
:10512000200602FA03F721FA06F52F43B3F1200512
:1051300058BF01FA05F701FA03F5C3F14003C3F1C3
:10514000200421FA03F102FA04F441EA040158BFF1
:105150000025002E58BF22FA06F122FA03F258BFAA
:105160000022294309EBC000DDF8CC903A4300EB64
:10517000CC0340F83C1037995A604FEA89004EF250
:10518000182350FA81F0C0F6000303EB800308EB0C
:10519000C00153F82E3001EBCE0251F83E10526898
:1051A00003F03F03C3F1200602FA03F721FA06F5E4
:1051B0002F43B3F1200558BF01FA05F701FA03F5B3
:1051C000C3F14003C3F1200421FA03F102FA04F40D
:1051D00041EA040158BF0025002E58BF22FA06F10B
:1051E00022FA03F20DF1E80C58BF00220CEBC000CC
:1051F0003A4300EBCE0329435A604EF2182340F89D
:105200003E100AEB8A00C0F6000303EB800308EBB4
:10521000C00153F8293001EBC90251F83910526826
:1052200003F03F03C3F1200602FA03F721FA06F563
:105230002F43B3F12005DDF8C8E04C4658BF01FA12
:1052400005F701FA03F5C3F14003C3F1200421FA85
:1052500003F102FA04F441EA040158BF0025002ECC
:1052600058BF22FA06F122FA03F241EA05010CEBDB
:10527000C00058BF002200EBC90340F839104FEAC4
:105280008E0050FA8BF04EF2182B3A43C0F6000B0A
:105290005A600BEB800308EBC00153F82A3001EB96
:1052A000CA0251F83A10526803F03F03C3F12006D6
:1052B00002FA03F721FA06F52F43B3F1200558BF90
:1052C00001FA05F701FA03F5C3F14003C3F1200425
:1052D00021FA03F102FA04F441EA040158BF00255F
:1052E000002E58BF22FA06F122FA03F258BF00221C
:1052F00029430CEBC0003A4340F83A1000EBCA00D7
:10530000426034983899359A00EB80000639A2EB58
:1053100000007FF40BAE40463AA9C822FCF79FF983
:10532000D8E92402D8E93034D8F81C70D8E90C59EF
:10533000D8E9181C3297D8F854E0D8E9007A23EA63
:10534000000821EA050620EA010B81EA08013391F1
:1053500027EA030148408BEA0501359125EA070158
:105360005940249022EA0C0030912AEA040151406D
:1053700080EA0900279124EA0201389029EA0A000C
:1053800081EA0C01604037912CEA09012F9039988D
:10539000069139990897D0F8B400329FD1F884105B
:1053A00027EA0002399B4A402C9221EA0E0220EAA9
:1053B0000101DB6C81EA0E0134912EEA0301794090
:1053C0002E9182EA0301369123EA0701399A399F27
:1053D0000596399E9269D7F8B070D6F8806022EAB7
:1053E0000704399B84EA06052295399D1B6DAD6C37
:1053F00026EA030427EA06065E40AB4383EA020E70
:1054000025EA02027A40484084EA05032692259064
:105410003998399A3293399BC0683999D2F8A420C7
:105420003196D3F89C30399EC96E20EA02075F405E
:10543000F66B209723EA010722EA03034B40B143AE
:105440004140199187EA06012D913999399F26EA41
:105450000000399E28938968399BD7F8A070D6F848
:105460009860399C9B6E21EA07057540A46B1E95D8
:1054700026EA030527EA06065E40A3434B40504058
:105480002B9385EA040324EA01011C903998399A88
:105490002A937940399B1D91406A3999D2F8BC20F2
:1054A0002996D3F88C30399EC96D20EA02075F40F7
:1054B000F66A139723EA010722EA03034B40B1433C
:1054C0004140169187EA060123913999399F26EACE
:1054D0000000399E2193096A399BD7F8B870D6F835
:1054E0008860399C9B6D21EA07057540A46A1A956E
:1054F00026EA030527EA06065E40A3435040399A90
:105500004B4024EA0101179039981B937940D2F857
:10551000AC30399A1891406939991F96D26F399EEB
:10552000496F20EA03075740766C129722EA010779
:1055300023EA020282EA0109B1434140149187EA59
:1055400006083999399F26EA0000399A399E85EA7A
:10555000040B0969D7F8A870399C126FB66F21EA5D
:105560000705246CCDF81CA085EA060A26EA020588
:1055700027EA060686EA020CA2434A4024EA010111
:1055800065404F40744683EA000EDDE938101592FD
:10559000C16039983599369A8160399837992D9B31
:1055A000416139983399CDF844B001613998279910
:1055B000149EC16139982499CDF840908161399841
:1055C0003099CDE90AE7016239982F990E9441622A
:1055D00039982E9984623998399CC16239983299E8
:1055E0000F95016339983199426339982C9A8163F8
:1055F00039983499CDF83080C16339982299CDF823
:1056000034C0016439982B9942643998269A82648F
:105610003998259AC2643998289A01653998199958
:10562000416539982A99816539982999C3653998CE
:10563000099B016639981E9942663998139A8166CA
:1056400039982099C16639981D99016739981C9934
:10565000416739981B99816739981699C1673998BC
:105660002399C0F880B039989346C0F884103998CF
:105670001F99C0F8881039982199C0F88C10399872
:105680001A99C0F8901039981599C0F89420399853
:10569000189AC0F898203998179AC0F89C20399821
:1056A000069AC0F8A01039981299C0F8A4603998E9
:1056B000C0F8A8503998C0F8AC803998C0F8B0C08C
:1056C0003998C0F8B4903998D146C0F8B8A0399844
:1056D0008A46C0F8BC1039984EF25811C0E9307EA5
:1056E000C0F6000101EBC30051F83310059F40687C
:1056F0007940089F50407940079F01334740019807
:105700006760834221607FF42BAA6DB0BDE8F08F03
:10571000D4F89C014FF6FC7CABF10108C1F6FF7C8C
:10572000C608B8F1030F0BF00309A64601D2002307
:1057300037E03AA80BEA0C0A00F1100401F110035B
:10574000002000BF0746B04207F1010032BF53E915
:10575000042500220025B04244E9042500F101009F
:1057600032BF53E9022500220025B04244E9022558
:1057700000F1010032BFD3E9002500220025B0422C
:10578000C4E9002500F1010032BFD3E9022500225F
:105790000025C4E902252034504503F12003D1D16E
:1057A0003B1DB9F1000F35D0B34205D201EBC30266
:1057B00051F83300526801E0002000223AAC04EBBB
:1057C000C305B9F1010F44F833006A6022D0581CB8
:1057D000B04205D201EBC00551F830206D6801E000
:1057E0000022002504EBC007B9F1020F44F8302075
:1057F0007D600FD0981CB04205D201EBC00251F879
:105800003010526801E00021002204EBC00344F88C
:1058100030105A60B8F1030FCDF8E09001D20021AA
:1058200032E03AA80CEA0B0CAEF12003A0F12007FD
:10583000002100BF57F8209F53F8206F07F1040E96
:105840009EE8204CD3E90104D3E90328684086EAA6
:105850000905C3E9005082EA0B0084EA0A029A6053
:105860007A695C69D86084EA020088EA0E02C3E9BA
:105870000420D7E90602D3E9065604317240684095
:105880008C459861DA61D5D1389A399C002A3FF469
:10589000F3A80DF1E80E0EEBC10004EBC1075EF8B2
:1058A000313040687E6854F8315070406B40012AB6
:1058B00044F8313078603FF4DFA8481C0EEBC00399
:1058C00004EBC0065EF830C05B68756854F8307051
:1058D0006B4087EA0C07022A44F8307073603FF48B
:1058E000CBA8881C0EEBC00104EBC0035EF830208F
:1058F00049685F6854F830607940724044F830205D
:105900005960FFF7B9B80000002808BF70472DE9BB
:10591000F041ECB08846002955D06D460646284631
:105920004FF4CC711746FBF7EEFEC82066901820A6
:10593000699001206B9004208DF89401F8082021D3
:105940006A90306868917168B26833901F20A8240B
:1059500034918DF8D80005F1D9009A21679405F1AA
:10596000CC073592FBF7ADFE80208DF873012846F9
:1059700039463294FFF76CF8679D6A9A0020AA4274
:1059800032906B9019D96E46404631462A46FBF755
:1059900021FE00BF30460021FFF75AF86A9C679F3E
:1059A000621BBA4208EB05000AD931463A46FBF7BA
:1059B00011FE3D44A542EDD305E06946404600E0B6
:1059C0006946FBF707FE6CB0BDE8F0417047000088
:1059D000B0B581B043F2104CC2F2000CDCF80030DC
:1059E00040F21C04C2F20004A2EB030EDCF800201B
:1059F00023680EF10104C3F3CB33634342F20C4E30
:105A00000093C2F2000EDEF8003002E0009D013D7E
:105A100000959D6805402D1AB5FA85F56D098D42F2
:105A200009D0DCF80050AD1AA54207D2009D002D28
:105A3000ECD10024EDE7002001B0B0BD586820F0A3
:105A4000E0005860DEF80400B0F5827F0BD1DEF88C
:105A50000800B0F5004F02D0B0F5806F03D1186890
:105A600020F040001860DEF82800B0F5005F07D194
:105A7000186820F400501860186840F4005018604E
:105A800001208EF8510000208EF85000032001B054
:105A9000B0BD00007047000043F21040C2F20000A9
:105AA00001680131016070474EF68850CEF2000067
:105AB000016841F4700101607047000042F26440E7
:105AC000C2F200000021FBF7DDBF000042F2AC4053
:105AD000C2F200000421FBF7D5BF000042F2F440FF
:105AE000C2F200000821FBF7CDBF000042F23C509B
:105AF000C2F200000C21FBF7C5BF000042F2845047
:105B0000C2F200001021FBF7BDBF000080B588B0D5
:105B100040F2EE010020C2F20001CDF80200ADF823
:105B20001E00CDF81A00CDF81600CDF81200CDF801
:105B30000E00CDF80A00CDF8060005200978ADF872
:105B4000000068468DF80210FDF7D0FF42F2CC50FD
:105B5000C2F20000FDF7C2FE08B080BD00000000E8
:105B600042F21460C2F20000006841F21112016AB0
:105B7000114208D1016A40F24442114203D1016846
:105B800021F0010101602DE9F04F81B02DED028B74
:105B90008AB0C1684CF2AE7621F0010141F6383C82
:105BA00042F6AC389FED4E8BC0F20106C1604FF05B
:105BB000010A4FF0000BC2F2000CC2F200080027ED
:105BC00000204FF0000E019024E0E018744607F02A
:105BD00016FF53EC182B07F0A1FF07F0E1FE41F28E
:105BE0005861C2F2000141F82900009841F6383CA2
:105BF0004CF2AE76A646C2F2000CC0F2010644EAB0
:105C0000000E00BF0BF1020BBBF1180F4FEA8A0A1E
:105C100000F0AE801CF80B00022814D341F2B864E7
:105C20000BEB4B02C2F2000404EB021112014B68B1
:105C3000A258019C9A1AE3B2022804F1010448F820
:105C4000232001944AD14BF001091CF809000228D5
:105C5000D8D341F2B86409EB4902C2F2000404EB64
:105C6000021112014B68A258019C9A1AE3B2022851
:105C700004F1010448F823200194C3D04FEA4A02FA
:105C8000009202220DE000BF013251F8223042F2B0
:105C900054541B1B0027B3F5EC6F98BF01278242B9
:105CA000B0D051F822303D0605D142F268041D1BE8
:105CB000B5F59D7FE8D346F23F441D1BB54202F186
:105CC0000102ECD251F82240E51A203DB5F5F67FED
:105CD0007FF67BAF8242E2D194E700BF022210E060
:105CE000000000000000E03F013251F8223042F293
:105CF00054541B1B0027B3F5EC6F98BF0127824259
:105D0000A1D051F822303C0605D142F268041C1B98
:105D100064089C2CE8D946F23F441C1BB44202F1B3
:105D20000102ECD251F82240E51A203DB5F5F67F8C
:105D300002D98242E3D186E7E018744607F05FFE9D
:105D400053EC182B07F0EAFE07F02AFE41F25861E7
:105D500041F6383C4CF2AE76A646C2F20001C2F2E1
:105D6000000CC0F2010641F82B0044EA0A0E6AE773
:105D7000019940F2EF040806C2F2000479D0A1F1C3
:105D800001095FFA89F009EBD01040B2F4464FEAFE
:105D9000600E4FF0000A5FFA8EFB00BF0AF10100AF
:105DA0004FFA8AF442B24FFA89F0824227465346AC
:105DB00017DC534604E000BF511C4AB282420FDC9C
:105DC00051B258F8217058F82450AF42F4DA5DB25D
:105DD00008EB85056E68013348F821606F60EBE7DA
:105DE0005FB258F8270058F8241048F82400D8B2B9
:105DF000584548F8271007D058B27045D4BF03F172
:105E0000010AA3F10109C9E758F82E004CF29D01DF
:105E1000A0F2EC40C9F6094151FB000040F2EF044A
:105E2000C11101EBD070C0F38001BCF1000FC2F2D0
:105E30000004217079D00121814341F2B86041F220
:105E40005863E6460122C2F20000C2F20003674630
:105E500005E000BF5200303003F1040357B1174290
:105E6000F8D01E6805689743761B06F6AB561E6091
:105E7000F0E70021BEF1000F57D041F6613200205B
:105E80002378C2F200029FED328B41F25868CDE9CF
:105E90000800CDE90600CDE90400107800244FF099
:105EA000010A4FF0000B0025C2F2000800298DF80E
:105EB0000A300FBF0421013010700321ADF8081023
:105EC0008DF80B0024A0075D0AFA07F616EA0E0FFC
:105ED0001DD058F827000AFA04F14BEA010BF146ED
:105EE00007F08DFD53EC182B07F018FE07F058FD56
:105EF00005EB450102AACE46114448F827008872F6
:105F0000020A000C29EA060E01354A720872152CA5
:105F100006D8BEF1000F03D0082D04F10104D1D33F
:105F200002A8CDF80CB0FDF7E1FD41F65031C2F208
:105F30000001002242F21460C2F200000A700AB0AE
:105F4000BDEC028B01B0BDE8F04FFDF7C7BC00BF50
:105F50007DC2ABF5AAF75740131211020C0D1704BE
:105F60000A050103140F0708160B0615090E000099
:105F700042F25C60C2F200001421FBF783BD000016
:105F800042F25C60C2F200000068C1680269D20798
:105F900018BF11F0010100D1704741F66431C2F21F
:105FA00000010A6802F580320A606FF001010161A8
:105FB00070470000B0B540F6FF3E0568C4F2000E21
:105FC00040F2004C7045C4F2010C0FDCB0F1804F80
:105FD00019D040F20043C4F20003984213D040F6B7
:105FE0000003C4F2000398420DD011E040F60043D4
:105FF000C4F20003984206D0604504D00023C4F2E6
:106000000103984204D14B6825F0700243EA02056F
:1060100041F6FF73C4F2000398420DDC70451FDCAB
:10602000B0F1804F41D040F20043C4F200039842E7
:106030003BD040F6000321E043F6FF73C4F20103B6
:10604000984220DC42F20003C4F2000398422CD0B4
:106050000023C4F20103984227D0604525D029E0EF
:1060600040F60043C4F2000398421ED041F60003FC
:10607000C4F20003984218D041F60043C4F2000372
:10608000984212D016E044F20003C4F20103984291
:106090000BD044F60003C4F20103984205D044F249
:1060A0000043C4F20103984204D1CB6825F4407246
:1060B00043EA02050A688C684B69C46240F4806454
:1060C0008262644504BF09690163026825F08001AA
:1060D00042F0040219430260012242610160B0BD36
:1060E000F0B581B0D0F8D42200EB8202D2F8C032F1
:1060F00023B301F00F058C4605EB850100EB810110
:1061000051F8144F64B1D0F8C86205EBC50006EB36
:10611000800EDEF81C00B4FBF0F707FB104078B1EE
:106120000024C3F81442D2F8C402056905B3D3F8B9
:10613000080203F504716246A84718E0032417E03B
:106140000024B2790C60714601F8145F0120012A25
:10615000CC6048700C614C6106D130680122CEF8E9
:10616000304000F0F7FE03E0306800F0F3FE00245A
:10617000204601B0F0BD0000D0F8D42200EB82032D
:10618000D3F8C022002A04BF0320704780B5D0F89E
:10619000C80201F00F0101EBC10100EB8100D0F852
:1061A0006802D3F8C412C2F80C02CB68D2F8040219
:1061B00002F503719847002080BD0000B0B5044689
:1061C000D0F8C80240F2011290F894140287012915
:1061D0000CD10021012284F83710A0F8782284F82D
:1061E00077114FF48171A0F85C1083E00268D2F857
:1061F0002019B1F1FF3F0BDCD2F8201941F000610A
:10620000C2F82019D2F8201941F08041C2F82019B3
:10621000D2F83C1847F6000C21F00201C2F83C18F5
:10622000D2F81C18CEF6334C21F00201C2F81C182B
:10623000D2F82039012503EA0C03C2F820390022E4
:10624000036880F8942484F83720A0F87852D3F8B3
:10625000205BB5F1FF3F0BDCD3F8205B45F0006518
:10626000C3F8205BD3F8205B45F08045C3F8205B82
:10627000D3F83C580CF1707125F40035C3F83C5844
:10628000D3F81C5825F40035C3F81C58D3F8205B0C
:106290002940C3F8201B80F8942484F877214FF418
:1062A00081710268A0F85C10D2F84019B1F1FF3F8B
:1062B0000BDCD2F8401941F00061C2F84019D2F865
:1062C000401941F08041C2F84019D2F83C1821F041
:1062D0000401C2F83C18D2F81C1821F00401C2F8DD
:1062E0001C18D2F8401901EA0C01C2F8401900212B
:1062F00080F89414D4F8D402002504EB8000D0F880
:10630000C01284F84B50656459B1D0F8C40240689B
:106310008047D4F8D40204EB8000C0F8C052C4F81F
:10632000BC520020B0BD000010B5D0F8D41200EB74
:106330008100D0F8C04284B1D0F8C41259B194F8A9
:106340000002FF2807D08B6894F801222146984765
:10635000FF2084F80002002010BD032010BD0000C3
:10636000014640F29C000A22C2F200000A807047F7
:10637000B0B540F25801C2F200014C8891F800E03B
:106380008446744540F2BE8040F25800C2F20000DC
:10639000714603E011448AB2A24264D202781044EA
:1063A0004378052B02D18378822B23D011448AB203
:1063B000A24258D2027810444378052B02D1837848
:1063C000822B17D011448AB2A2424CD202781044D8
:1063D0004378052B02D18378822B0BD011448AB2EB
:1063E000A24240D2027810444378052BD2D1837860
:1063F000822BCFD1744539D940F25801C2F2000145
:10640000734603E013449AB2A24231D20A7811448F
:106410004D78052D02D18D78012D2AD013449AB2E2
:10642000A24225D20A7811444D78052D02D18D78EB
:10643000012D1ED013449AB2A24219D20A781144F7
:106440004D78052D02D18D78012D12D013449AB2CA
:10645000A2420DD20A7811444D78052DD2D18D7803
:10646000012DCFD105E000207445C5D800213CE0C6
:106470000021744539D940F25803C2F2000304E008
:1064800096441FFA8EF2A2422FD21A7813445D78F6
:10649000052D02D19D78812D28D0724495B2A54258
:1064A00023D293F800E073445D78052D02D19D78E6
:1064B000812D1BD0724495B2A54216D293F800E00C
:1064C00073445D78052D02D19D78812D0ED07244E4
:1064D00095B2A54209D293F800E073445D78052D8A
:1064E000CED19D78812DCBD100E0002300281CBFA8
:1064F0001022827100291CBF40208880002B1CBF05
:106500004020988040F258004321C2F20000ACF8CD
:106510000010B0BDB0B540F25801C2F200014C8885
:1065200091F800E08446744540F2C08040F2580083
:10653000C2F20000714603E011448AB2A24264D262
:10654000027810444378052B02D18378822B23D024
:1065500011448AB2A24258D2027810444378052BE3
:1065600002D18378822B17D011448AB2A2424CD236
:10657000027810444378052B02D18378822B0BD00C
:1065800011448AB2A24240D2027810444378052BCB
:10659000D2D18378822BCFD1744539D940F25801BA
:1065A000C2F20001734603E013449AB2A24231D210
:1065B0000A7811444D78052D02D18D78012D2AD00D
:1065C00013449AB2A24225D20A7811444D78052D7F
:1065D00002D18D78012D1ED013449AB2A24219D255
:1065E0000A7811444D78052D02D18D78012D12D0F5
:1065F00013449AB2A2420DD20A7811444D78052D67
:10660000D2D18D78012DCFD105E000207445C5D8B9
:1066100000213CE00021744539D940F25803C2F210
:10662000000304E096441FFA8EF2A2422FD21A7899
:1066300013445D78052D02D19D78812D28D07244B8
:1066400095B2A54223D293F800E073445D78052DFE
:1066500002D19D78812D1BD0724495B2A54216D2ED
:1066600093F800E073445D78052D02D19D78812D6B
:106670000ED0724495B2A54209D293F800E073445B
:106680005D78052DCED19D78812DCBD100E0002302
:1066900000281CBF1022827100291CBF4FF400701B
:1066A0008880002B1CBF4FF40070988040F2580087
:1066B0004321C2F20000ACF80010B0BDB0B540F20A
:1066C0005801C2F200014C8891F800E084467445FC
:1066D00040F2BE8040F25800C2F20000714603E072
:1066E00011448AB2A24264D2027810444378052B46
:1066F00002D18378822B23D011448AB2A24258D28D
:10670000027810444378052B02D18378822B17D06E
:1067100011448AB2A2424CD2027810444378052B2D
:1067200002D18378822B0BD011448AB2A24240D28C
:10673000027810444378052BD2D18378822BCFD1B5
:10674000744539D940F25801C2F20001734603E0A2
:1067500013449AB2A24231D20A7811444D78052DE1
:1067600002D18D78012D2AD013449AB2A24225D2AB
:106770000A7811444D78052D02D18D78012D1ED057
:1067800013449AB2A24219D20A7811444D78052DC9
:1067900002D18D78012D12D013449AB2A2420DD2AB
:1067A0000A7811444D78052DD2D18D78012DCFD1A5
:1067B00005E000207445C5D800213CE00021744567
:1067C00039D940F25803C2F2000304E096441FFA9C
:1067D0008EF2A2422FD21A7813445D78052D02D191
:1067E0009D78812D28D0724495B2A54223D293F88A
:1067F00000E073445D78052D02D19D78812D1BD07A
:10680000724495B2A54216D293F800E073445D78C5
:10681000052D02D19D78812D0ED0724495B2A542EE
:1068200009D293F800E073445D78052DCED19D78B0
:10683000812DCBD100E0002300281CBF10228271E3
:1068400000291CBF40208880002B1CBF402098805E
:1068500040F258004321C2F20000ACF80010B0BD75
:106860002DE9F04140F23845C2F2000504462846C1
:106870004FF40771FAF747FFD4F8D402217C04EBF8
:106880008000C0F8C052D4F8C8024027C4F8BC52F7
:10689000002908BF4FF40077812102223B464FF0C8
:1068A000020800F073FAD4F8C8020126012102227E
:1068B0003B4684F8376000F069FA1021D4F8C8022A
:1068C000616482210322082384F8776100F05EFA74
:1068D000D4F8D4020027C5F8047204EB8000D0F885
:1068E000C40284F84B6000688047C5F81472C5F88C
:1068F0001872D5F80432E3B1D4F8C802227CC0F88B
:106900008432002A14BF40224FF400720027C0E9ED
:10691000A22782790127012AA0F8787204BFC0F863
:106920009432012200F51E71006800F013FB4FF055
:1069300000084046BDE8F08170B582B00446D0F84A
:10694000D4020E4604EB8000D0F8C0520021002D86
:106950008DF80710ADF8041000F09F80317811F029
:1069600060022DD0202A40F08E80F288002A3CD090
:1069700049B2B1F1FF3F41DD7078402A85F800024D
:106980004FF0030028BF402285F80122C4F894028A
:10699000D4F8C832C4F85421C4F85821C3E9985235
:1069A0009A7903F515710020012AC4F86451C3F8DF
:1069B0006802A3F8540242D11868C3F870525CE030
:1069C00070780B285FD80025DFE800F006685D5D71
:1069D0005D5D5D5D5D5D3B5994F89C02032852D17D
:1069E000022001ABC4F8940235E0D0F8C40231466D
:1069F000836870780022002598474FE0D0F8C402E1
:106A00002946836870789847F0880221072828BFB4
:106A10000720C4F89412D4F8C8324FF48072194693
:106A20006562C4E9050021F8142F9A790026012A2D
:106A300058621D629E6202D118681D631DE01868CD
:106A400030E094F89C0203281DD10220C4F894027F
:106A500001200DF10703D4F8C8624FF4807231466B
:106A600063626061A06121F8142FB2797062012A1B
:106A70003362B56215D130683363012212E094F8B5
:106A80009C0203280AD0D4F8C802802100F0E0F963
:106A9000D4F8C802002100F0DBF90325284602B033
:106AA00070BD306800F056FA0025F7E780B504A005
:106AB00000F002F940F23820C2F2000080BD00BFB1
:106AC00043444320436F6E666967000040F2A800AC
:106AD0001222C2F200000A807047000080B504A0B4
:106AE00000F0EAF840F23820C2F2000080BD00BF9A
:106AF00043444320496E746572666163650000001B
:106B000040F2D0000422C2F200000A807047000068
:106B100080B504A000F0D0F840F23820C2F20000A6
:106B200080BD00BF43796D706C65000080B504A026
:106B300000F0C2F840F23820C2F2000080BD00BF71
:106B4000547261636B65720047F61020C1F6FF70E6
:106B5000026883684FF01A0C9B18A1F800C000F07F
:106B6000A680B0B54FF0370C1A0F0CEB13714068CC
:106B7000B3F1204F38BF02F1300140F2D402C2F22B
:106B80000002917019014FF0000E0CEB117582F8A4
:106B900003E0C3F30364B1F1204F38BF04F13005C3
:106BA000190215710CEB117582F805E0C3F303545B
:106BB000B1F1204F38BF04F13005190395710CEB8A
:106BC000117582F807E0C3F30344B1F1204F38BFD9
:106BD00004F13005190415720CEB117582F809E007
:106BE000C3F30334B1F1204F38BF04F13005190568
:106BF00095720CEB117582F80BE0C3F30324B1F12D
:106C0000204F38BF04F1300519061573C3F3031480
:106C10000CEB1175B1F1204F4FEA037103F00F0334
:106C200082F80DE038BF04F1300503F137049573A5
:106C300082F80FE0B1F1204F38BF03F13004010FAB
:106C40000CEB1073147482F811E0B0F1204F38BFD0
:106C500001F1300301010CEB1174937482F813E01D
:106C6000C0F30363B1F1204F38BF03F130040102D8
:106C70001475C0F303530CEB1174B1F1204F4FEABC
:106C8000003182F815E038BF03F130040CEB1173CA
:106C9000947582F817E0C0F30340B1F1204F38BF7C
:106CA00000F13003137682F819E0BDE8B04040F2FD
:106CB000D400C2F200007047002808BF704780B5BA
:106CC000027892B1831C4FF0000C00BF13F8012C26
:106CD00072B11A787AB15A7882B19A780CF1040CB0
:106CE000002A03F10403F1D10AE04FF0000C07E0A1
:106CF0004CF0010C04E04CF0020C01E04CF0030CF1
:106D00005FFA8CF2022340F2382E03EB4202C2F209
:106D1000000E0A808EF8002003228EF801200378EE
:106D200083B3023002224FF0000C00BFD1B20EF844
:106D3000013041F001010EF801C010F8013C0BB325
:106D4000911CC9B20EF8013041F001010EF801C0EA
:106D50000378BBB1111DC9B20EF8013041F0010139
:106D60000EF801C043786BB1911DC9B20EF8013025
:106D700041F001010EF801C083780832002B00F1C8
:106D80000400D3D1BDE8804070470000B0B501F0E9
:106D90000F0C4CB20CEBCC01B4F1FF3F00EB810EB9
:106DA00005DD0EF5157100248EF8554204E001242E
:106DB0000EF114018EF8154091F801E06FF3DF2316
:106DC000BEF1000F81F800C08B600A7118BFA1F8F6
:106DD0001AC0022A04BF00244C7190F894140129AF
:106DE00008BFB0BD0168BEF1010FD1F81C484FEAE1
:106DF0004C1E11D1012505FA0CF52C43C1F81C4895
:106E00007144D1F800592D041DD401F5106143EAF5
:106E100082434FEA8C520EE04FF4803505FA0CF5B0
:106E20002543C1F81C587144D1F8005B2D040AD4E5
:106E300001F5306192040D682A431A4342F08052F2
:106E400042F400420A60002180F89414B0BD0000B2
:106E500080B5037901F00F0E9E4501D9082172E03B
:106E60004BB2B3F1FF3F09DD01EBC10100EB810340
:106E700003F51571002283F8552208E00EEBCE01D0
:106E800000EB810C01230CF114018CF8153090F803
:106E900094240123012A8B7081F800E001D1102194
:106EA00051E0497880F89434036801294FEA4E1183
:106EB000194406D1D1F8002901F51061002A06D540
:106EC00012E0D1F8002B01F53061002A0CD4BEF19C
:106ED000000F09D00A6822F080420A604FF40012C5
:106EE0000B681A430A602BE00A68BEF1000F42F4F7
:106EF00000120A6024D190F806C0196C43F20B020C
:106F0000C4F65472914203F5306102D30A68002A34
:106F100016D400220A610A69BCF1010F42F4002272
:106F20000A610A6942F018020A610A6942F0C04225
:106F30000A6105D100F29C424A614FF08022CFE7FE
:106F4000002180F8941440F20030C0F20130C840B3
:106F5000C0B280BD70B54B7891F800C0012B2ED126
:106F6000D1F810E000EB4C14D4F81039BEF1000F4A
:106F700004F510644CD06FF3120323612369BCF154
:106F8000000F6FF3DC4323618D6871D00EEB0503B6
:106F9000013BB3FBF5F30025C1F6F875266905EA58
:106FA000C345354325610D79012D6DD1256925F046
:106FB000C04525614FF0C04505EA437361E000EB31
:106FC0004C16D6F8103BBCF1000F6FF31203C6F855
:106FD000103BD6F8103B06F530646FF3DC43C6F87F
:106FE000103B8B680D6920D01DB3EE18013EB6FB37
:106FF000F3F640F2000CB5B26B430B62C1F6F87CBD
:1070000025690CEAC6462E436FF3DF43266117E07D
:107010006FF3DC43236123694FF0000E43F4002338
:10702000236123696FF3120333E0002D18BF0B6156
:107030000B6226696FF3DF43334323614FF4002370
:107040002669012A43EA0603236103D1CA68002A9C
:1070500018BF6261097901292FD1D0F80808216889
:10706000C0054FF0805058BF4FF00050084323E058
:10707000AE4504D90D614FF40023AE4601E04FF454
:10708000002325692B432361734625696FF3DF4392
:107090002B43012A236116D1CA69002A18BF6261F5
:1070A0000979012909D1D0F808182068C9054CBF11
:1070B00040F0805040F0005020604FF004412068C4
:1070C0000843206070BD236843F0044323600B79BC
:1070D000012B3BD1D0F808382568DB054FF08053F1
:1070E00058BF4FF000532B43002A2360EAD11FFA08
:1070F0008EF2002AE6D0D51C4FF0FF33C96803EBAF
:10710000950300F580504FEA0C32032BC5F3810341
:107110000ED3AE0826F003040E68043C16504E68E9
:1071200016508E681650CE6801F110011650F3D13A
:10713000002BC7D00E68012B8650C3D04E68022B9F
:10714000865008BF70BD8968815070BDBEF1000FC8
:10715000B8D00CF00F01012202FA01F100F634045C
:10716000ADE7000081B0002200924A780978012A38
:107170004FEA411138D100F510604258B2F1FF3F9B
:1071800038DC0A5842F000620A500A5842F0804245
:107190000A5042F21072009B01330093009B93420D
:1071A00028D84358B3F1FF3F24DC009B0133009300
:1071B000009B93421ED84358B3F1FF3F1ADC009B5B
:1071C00001330093009B934214D84358B3F1FF3F1F
:1071D00010DC009B01330093009B93420AD8435874
:1071E000B3F1FF3FD7DD05E000F530604258B2F162
:1071F000FF3F01DD01B070470A5842F000620A50BB
:107200000A5842F080420A5042F21072009B013349
:107210000093009B9342EDD84358B3F1FF3FE9DC64
:10722000009B01330093009B9342E3D84358B3F192
:10723000FF3FDFDC009B01330093009B9342D9D8D2
:107240004358B3F1FF3FD5DC009B01330093009B13
:107250009342CFD84358002BD8D4CBE781B000223B
:107260000092009A01320092009AB2F1706F4ED8EB
:107270000269002A1ED4009A01320092009AB2F1EB
:10728000706F44D80269002A14D4009A0132009227
:10729000009AB2F1706F3AD80269002A0AD4009AB3
:1072A00001320092009AB2F1706F30D80269B2F1E7
:1072B000FF3FD6DC89010022203100920161009954
:1072C000013100910099B1F1706F20D801698906F0
:1072D0001DD50099013100910099B1F1706F16D858
:1072E0000169890613D50099013100910099B1F126
:1072F000706F0CD80169890609D500990131009198
:107300000099B1F1706F02D801698906D7D401B034
:1073100070470000FEE7000083B070B5C1B045A81B
:1073200001AC0EC020464FF48071FAF7ECF945AA83
:1073300015A120460092F9F71FF82046F9F74CF8FE
:1073400043F20C45C2F200052E88044616FA80F07E
:107350000021B1EBD02F0AD142F60C40C2F200005E
:10736000A2B2304401A9FAF735F926442E80B0B212
:10737000FAF73EFB002804BF0020288041B0BDE89A
:10738000704003B0704700BF0A0A62757379200A23
:1073900000000000000000002DE9F04381B02DED59
:1073A000028B82B0002041F644680190C2F20008CE
:1073B00098F83C00D8F8007001284FF0010900F05F
:1073C000998088F83C90384650F8081FC90726D1A4
:1073D00001684DF6836241F00101016040F21C0139
:1073E000C2F200010968C4F21B32A1FB0212910C27
:1073F00001EB41010191019989B101990139019193
:10740000019961B1019901390191019939B101994C
:1074100001390191019911B101990139EAE7026835
:10742000D8F84010D2070CD141F01000C8F8400045
:1074300008F144004FF00109012102681143016085
:1074400058E040F20172914301F58071C8F8401094
:107450007968490506D5D8F84010012262F30D314C
:10746000C8F84010D8F8401000230022C90444BFD7
:10747000D8F8441021F0060342F20431C8F8443031
:1074800088F83C206FF02202C4F201013A600A68D9
:10749000D20606D0A1F54172974220D04FF00009E4
:1074A00028E042F20002C4F20102974215D042F2F3
:1074B0000022C4F2010297420CD042F20012C4F240
:1074C00001029742EAD10A68D20606D0A1F582727B
:1074D0009742E3D10968C906E0D4016804E04FF699
:1074E0000452CFF6FF7289584FF0000911F0405F47
:1074F00000F0B080B868400544BFB8685FEAC0508B
:1075000066D443F21040C2F2000001683A68920764
:1075100008D40268521A332AF8D33A689207F5D48D
:10752000042056E06FF012003860D8F8400040F4B4
:107530000070C8F84000B86810F0405F19D198F8A2
:107540001800B0B9F86A10F4700F02D0B86840059E
:107550000FD4D8F8400020F48070C8F84000D8F864
:107560004000C00405D4D8F8400040F00100C8F83D
:107570004000F86C9FED8C1A80B200EE100AB8EE55
:10758000C00A20EE010A10EE100A06F0B3FC9FEDCF
:107590006C0B53EC102B06F0C1FA06F0DFF8044632
:1075A00006F0A8FC9FED680B054653EC102B0E4629
:1075B00006F0D9FC08B1642023E09FED650B284656
:1075C00053EC102B314606F0E3FC00B3002018E02A
:1075D0002020D8F840100843C8F840000020B968BF
:1075E00021F00101B960B968C90707D1D8F8401086
:1075F00041F2011291430131C8F84010002188F88E
:107600003C1002B0BDEC028B01B0BDE8F0839FEDF1
:10761000671A00EE104AB4EE410AF1EE10FA03DAEE
:107620009FED4D8B002064E09FED611AB4EE410A9E
:10763000F1EE10FA03DA9FED4A8B012059E09FED3D
:107640005D1AB4EE410AF1EE10FA06DA9FED468BB0
:1076500002204EE04FF08041EFE69FED571AB4EE66
:10766000410AF1EE10FA03DA9FED418B032040E06E
:107670009FED521AB4EE410AF1EE10FA03DA9FEDD3
:107680003E8B042035E09FED4E1AB4EE410AF1EE38
:1076900010FA03DA9FED3A8B05202AE09FED491A94
:1076A000B4EE410AF1EE10FA03DA9FED378B0620B3
:1076B0001FE09FED451AB4EE410AF1EE10FA03DA2D
:1076C0009FED338B072014E09FED401AB4EE410A82
:1076D000F1EE10FA03DA9FED308B082009E09FED00
:1076E0003C1AB4EE410AF1EE10FA22DA9FED2C8B2F
:1076F000092038A101EB800090ED002A30EE420A0B
:1077000031EE421A80EE010A10EE100A06F0F2FB8A
:107710009FED130B53EC102B06F000FA53EC182BD3
:1077200006F04EF806F03CF9B9F1000F3FF457AF00
:1077300067E76420B9F1000F3FF451AF61E700BF84
:10774000CDCCCCCCCCCC16409A9999999999104033
:107750006666666666660A4000000000000000007B
:107760000000000000002440000000000000344041
:107770000000000000003E40000000000000444007
:1077800000000000000049400000000000004E40E2
:107790000000000000805140000000000000544044
:1077A00000000000008056403333533AC3F5684070
:1077B000295C6F40AE4771405C8F7240E17A744043
:1077C00014AE774048E17A4052B87E4085EB814064
:1077D000CDCC844033335340C3F56840295C6F40BF
:1077E000AE4771405C8F7240E17A744014AE7740CE
:1077F00048E17A4052B87E4085EB8140CDCC844050
:1078000083B070B5C1B0044645A801AD0EC0281DB7
:10781000FC21F9F778FF0320ADF808004FF6FC6073
:10782000CFF6FC600835019045AA28462146009213
:10783000F8F7A2FD2846F8F7CFFD43F20C44C2F258
:10784000000400F1090125880E1815FA86F00022BF
:10785000B2EBD02FADF80A100AD142F60C40C2F2BA
:107860000000B2B2284401A9F9F7B4FE35442580DE
:10787000A8B2FAF7BDF8002804BF0020208041B06C
:10788000BDE8704003B07047A2B043F6300AC4F2BE
:10789000020ADAF8D0034EF60C5B40F40070CAF826
:1078A000D003DAF8D003CEF2000B40F48060CAF8BF
:1078B000D003DAF8D01340F2003041F48071CAF8F6
:1078C000D013DBF800104FF6FF02C0F2FA5011405F
:1078D000014340F21C04CBF80010C2F200042168FE
:1078E00044F6D358C1F26208A1FB08174FF0FF33EA
:1078F00003EB97170021B1EB176F26D14EF200165C
:10790000CEF2000646F8EC7CF0278BF817700727BC
:1079100046F8E81C46F8F07CDBF80060C6F3022667
:1079200086F00705042D28BF0425AB40033E27EA57
:10793000030338BF0E46B3401B018BF8173043F2E8
:107940001443C2F2000301271F700991DAF81430C2
:1079500000F5807043F48043CAF81430DAF814302C
:1079600043F2104903F480430993099B0991DAF823
:107970001030C2F2000943F08053CAF81030DAF830
:10798000103003F080530993099BDBF800301A4054
:107990001043CBF800000991DAF81000002240F003
:1079A0008050CAF81000DAF81000C4F2020200F0A9
:1079B00080500990099847F200000991CFF6FE70B7
:1079C000115841F480411150105800F48040099042
:1079D00009985AF8280C00F00C00042831D15AF804
:1079E000300C6020C4F247200121C0F8201ED9F8D5
:1079F0000010DAF8442092075DD4D9F80020521A1A
:107A0000022A00F2ED80DAF84420920753D4D9F824
:107A10000020521A022A00F2E380DAF8442092078A
:107A200049D4D9F80020521A022A00F2D980DAF893
:107A3000442092073FD4D9F80020521A022AD8D9FC
:107A4000CEE05AF8280C00F00C00082803D15AF8B0
:107A50002C0C4002C3D45AF8300C40F480304AF861
:107A6000300CD9F800005AF8301C8903B9D4D9F881
:107A70000010091A642900F2B3805AF8301C8903F7
:107A8000AFD4D9F80010091A642900F2A9805AF875
:107A9000301C8903A5D4D9F80010091A642900F212
:107AA0009F805AF8301C89039BD4D9F80010091A1A
:107AB0006429D8D994E05AF8281C01F00C0108294F
:107AC00035D15AF82C0C47F6FF71C0F643710840C7
:107AD00042F60821C0F24071884240F08180DAF815
:107AE000D00300F00700042808D805208AF8D00346
:107AF000DAF8D00300F00700052815D15AF8280C51
:107B000040F4E0504AF8280C5AF8280C40F4604041
:107B10004AF8280C5AF8280C20F0F0004AF8280CF3
:107B20005AF8300C80015ED472B600BFFEE7002127
:107B30000160D9F800105AF8302C920120D5D9F8FC
:107B40000020521A022A4BD85AF8302C920117D52D
:107B5000D9F80020521A022A42D85AF8302C920141
:107B60000ED5D9F80020521A022A39D85AF8302CEA
:107B7000920105D5D9F80020521A022ADBD92FE04C
:107B800042F60821C0F240714AF82C1C0121016024
:107B9000D9F800005AF8301C8901A0D4D9F8001097
:107BA000091A02291CD85AF8301C890197D4D9F82F
:107BB0000010091A022913D85AF8301C89013FF520
:107BC0008EAFD9F80010091A022909D85AF8301CCA
:107BD00089013FF584AFD9F80010091A0229D9D9D3
:107BE00072B600BFFEE75AF8280C022161F30100CB
:107BF0004AF8280CD9F8000041F288315AF8282CAC
:107C000002F00C02082A29D0D9F80020121A8A4260
:107C10003FF68AAF5AF8282C02F00C02082A1DD031
:107C2000D9F80020121A8A423FF67EAF5AF8282C63
:107C300002F00C02082A11D0D9F80020121A8A4248
:107C40003FF672AF5AF8282C02F00C02082A05D031
:107C5000D9F80020121A8A42D0D965E7DAF8D003A1
:107C600000F00600062809D105208AF8D003DAF8CA
:107C7000D00300F0070005287FF456AF5AF8280C0F
:107C8000052161F38C204AF8280C5AF8280C0421AD
:107C900061F34F304AF8280C5AF8280C00F00C0019
:107CA000082842F20040C0F2F40017D15AF82C1C08
:107CB0005AF82C2C5AF82C3C01F03F02C3F38811DF
:107CC000A1FB00010023F9F70DFC5AF82C1C02223D
:107CD000C1F3014102EB4101B0FBF1F05AF8281C5D
:107CE0000FF61862C1F30311515C4FF0FF3720FA11
:107CF00001F1A1FB080343F21440C2F20000027834
:107D00002160002A114607EB93134FF000084EF252
:107D1000001718BF0721B8EB136FCEF2000722D16E
:107D200047F8EC3CF0238BF81730072347F8E88C32
:107D300047F8F03CBAB1DBF800204FF0FF37C2F350
:107D4000022282F00703042B28BF042307FA03F35F
:107D5000033A21EA030138BF0022914009018BF860
:107D6000171001210170CDE90C88CDF87480DAF884
:107D7000000040F6184740F01000CAF80000DAF89A
:107D800000004FF6000100F010001D901D98CDF886
:107D90007480DAF80000C4F2020740F00400CAF868
:107DA0000000DAF80000CFF6FF7100F004001D902B
:107DB0001D98CDF87480DAF800003C4640F0800051
:107DC000CAF80000DAF8000009AE00F080001D904B
:107DD0001D98CDF87480DAF80000032540F001000A
:107DE000CAF80000DAF8000000F001001D901D98AC
:107DF000CDF87480DAF8000040F00200CAF8000004
:107E0000DAF8000000F002001D901D98CDF8748093
:107E1000DAF8000040F00800CAF80000DAF80000C4
:107E200000F008001D901D984FF0805078501120F0
:107E300038604FF4003044F8180949F2FF500990B7
:107E400003200A9041F20000C4F202003146CDF84E
:107E50002C80FAF7ADF94EF2100009A981E8210152
:107E6000A7F5836031460790FAF7A2F942F21010A5
:107E700009A981E821010020C4F202003146074629
:107E8000FAF796F94FF480500990012007F58065C4
:107E9000CDE90A0828463146CDF83080FAF788F94E
:107EA0004EF2303009900320CDE90A0828463146C9
:107EB0000895FAF77DF94FF4786009900320CDE931
:107EC0000A0820463146FAF773F94FF480400990CA
:107ED0004FF404100A9001200B9038463146FAF70F
:107EE00067F94FF4004009904FF48810CDE90A0873
:107EF00038463146FAF75CF90320099001204EF22A
:107F00000015CDE90A080C9020463146CEF2000556
:107F10000127FAF74DF96C2009904FF40410CDE9D0
:107F20000A0720463146FAF743F9102009A981E8EB
:107F3000810120463146CDF83080FAF739F9DBF877
:107F400000000422C0F3022080F00701042928BFAA
:107F500011464FF0FF36033806FA01F14FF00203E5
:107F600038BF404623EA010101FA00F0000185F81C
:107F700008034FF480702860DBF80010C1F3022181
:107F800081F00707042F38BF3A46033906FA02F298
:107F900038BF414623EA020202FA01F1090185F8DD
:107FA000281368600025C4F2020542F26440A5F57A
:107FB0008031C2F200004FF6FF73CDF88080CDE92A
:107FC0001E88CDF83480CDE90B88072280E80601B1
:107FD000C0E90338C0E90588FBF792F808B172B62A
:107FE000FEE742F264444FF48050C2F200041D9058
:107FF0001DA92046FBF7A4FB08B172B6FEE794F872
:108000003D00211D002804BF002084F83C00022010
:1080100084F83D002068FDF7CDFF012084F846007C
:1080200084F83E0084F83F0084F8400084F8410062
:1080300084F8420084F8430084F8440084F8450042
:1080400084F83D000620099000200A9009A92046E6
:10805000FBF796FC08B172B6FEE794F83C000128E5
:1080600001D172B6FEE7022084F83D00206841F29B
:10807000FF7342688168C4F2000322F070029842E4
:1080800042600DDC40F2FF72C4F20002904215DC47
:10809000B0F1804F29D040F20042C4F2000222E049
:1080A00040F2FF32C4F20102904212DC41F60002BB
:1080B000C4F20002904218D0002212E040F6000202
:1080C000C4F20002904210D040F60042C4F2000216
:1080D00009E044F20002C4F20102904205D040F2ED
:1080E0000042C4F20102904202D121F0800181607D
:1080F000012184F83D10002184F83C10016A026AD5
:10810000984222F00102026282690DDC40F2FF73A4
:10811000C4F20003984215DCB0F1804F2CD040F23D
:108120000043C4F2000322E040F2FF33C4F2010333
:10813000984212DC41F60003C4F2000398421BD0BF
:10814000002312E040F60003C4F20003984213D06B
:1081500040F60043C4F2000309E044F20003C4F215
:108160000103984208D040F20043C4F20103984250
:1081700008BF22F0030201E022F0030242F00102F4
:1081800022F0F00241F00A0182610162816942F24B
:10819000A46621F00C0181618169C2F2000681614F
:1081A000016A026A41F0A00122F0100202628269B3
:1081B00022F4734202F5807282610162816921F4C6
:1081C0004061816181698161016A026A41F42061D3
:1081D00022F480720262C26942F0010222F0F202CD
:1081E000C2610162C16921F00C01C161C169C16153
:1081F000016A026A41F4204122F480520262C2699B
:1082000022F4734202F58072C2610162C1690C22DC
:1082100021F44061C161C169C161002084F83C0062
:10822000A5F570444FF4E131C6E90041C6E902000A
:10823000C6E90402C6E9060096F8411021B1002102
:1082400000220023A0462FE086F840000990DAF8CB
:10825000141041F01001CAF81410DAF8141001F0EB
:108260001001099109990990DAF8001041F0010113
:10827000CAF80010DAF8001001F00101099109991B
:108280004FF4C06109910221CDE90A1003200C903E
:1082900007200D9009A92846F9F78AFFD6F8008033
:1082A000D6E90223D6E90601242786F84170D8F8DA
:1082B0000C7027F40057C8F80C70D8F8107027F429
:1082C00040573B43C8F81030D6E904371A43D8F872
:1082D0000C303A4349F20C67BB431A430A43C8F8CF
:1082E0000C20D8F8142022F440721043C8F814006F
:1082F00028F48060A04240F21C00C2F200004FF05F
:108300000A0200685AF8283C08BF0D2223FA02F23C
:108310004EF27C2302F00702C0F600039A5C7368F9
:10832000D0401922B1F5004FA0FB020120D15A0024
:10833000DB0FF9F7D7F848F21F51C5F2EB11A0FB9C
:1083400001235A094FF69C73C0F6FF7303F1805363
:1083500002FB0300322303EBC000A0FB01014FF43A
:10836000F87000EA111000EB0210C1F342111CE09A
:108370009A009B0FF9F7B6F848F21F51C5F2EB11BE
:10838000A0FB01235A094FF69C73C0F6FF7302FB52
:108390000300322303EB0010A0FB0101F02000EAF0
:1083A000511000EB0210C1F343110844C8F8080053
:1083B000D8F81000002120F49040C8F81000D8F838
:1083C00014004FF0804220F02A00C8F81400D8F8BA
:1083D0000C00032340F40050C8F80C002020716406
:1083E00086F8410086F8420042F2AC40C2F200003A
:1083F0004FF6FF7771632091CDE91E110D91CDE904
:108400000B11C0E90023C0E9021701618161FAF78D
:1084100077FE10B172B600BFFEE742F2AC444FF4F3
:108420008050C2F200041D901DA92046FBF788F978
:1084300008B172B6FEE794F83D00211D002804BF84
:10844000002084F83C00022084F83D002068FDF7FD
:10845000B1FD012084F8460084F83E0084F83F0016
:1084600084F8400084F8410084F8420084F8430016
:1084700084F8440084F8450084F83D000620099003
:1084800010200A9009A92046A046FBF779FA10B1FE
:1084900072B600BFFEE798F83C00012801D172B621
:1084A000FEE7022088F83D00D8F80000012342686A
:1084B000414663F3061241F2FF738168C4F2000380
:1084C000984242600DDC40F2FF72C4F2000290421A
:1084D00015DCB0F1804F29D040F20042C4F2000216
:1084E00022E040F2FF32C4F20102904212DC41F677
:1084F0000002C4F20002904218D0002212E040F6BE
:108500000002C4F20002904210D040F60042C4F2D1
:10851000000209E044F20002C4F20102904205D0D8
:1085200040F20042C4F20102904202D121F08001E7
:108530008160012188F83D100021424688F83C10F6
:10854000016A026A984222F00102026282690DDC2D
:1085500040F2FF73C4F20003984215DCB0F1804F83
:108560002CD040F20043C4F2000322E040F2FF337B
:10857000C4F20103984212DC41F60003C4F2000386
:1085800098421BD0002312E040F60003C4F200031F
:10859000984213D040F60043C4F2000309E044F2CD
:1085A0000003C4F20103984208D040F20043C4F231
:1085B0000103984208BF22F0030201E022F0030207
:1085C00042F0010222F0F00241F00A0182610162F0
:1085D0008169032321F00C01816181694FF6FF77E6
:1085E0008161016A026A41F0A00122F01002026278
:1085F000826922F4734202F58072826101628169AC
:1086000021F44061816181698161016A026A41F4FA
:10861000206122F480720262C26942F0010222F0FB
:10862000F202C2610162C16921F00C01C161C1693C
:10863000C161016A026A41F4204122F4805202625F
:10864000C26922F4734202F58072C2610162C1699B
:10865000042221F44061C161C169C4F20002C16118
:1086600042F2F440002102F57F72C2F2000088F865
:108670003C102091CDE91E110D91CDE90B11C0E9FF
:108680000023C0E9021701618161FAF739FD08B1E1
:1086900072B6FEE74FF480501D9042F2F440C2F2F1
:1086A00000001DA9FBF74CF808B172B6FEE742F2D4
:1086B000F440C2F2000090F83D0030B942F2F441BB
:1086C0000020C2F2000181F83C0042F2F444022092
:1086D000C2F2000484F83D002068211DFDF76AFC09
:1086E000012084F8460084F83E0084F83F0084F8B6
:1086F000400084F8410084F8420084F8430084F884
:10870000440084F8450084F83D00062009902020AC
:108710000A9009A92046FBF733F908B172B6FEE7C3
:1087200042F2F440C2F2000090F83C00012801D16E
:1087300072B6FEE742F2F4410220C2F2000181F873
:108740003D00086801234268816863F3061241F224
:10875000FF73C4F20003984242600DDC40F2FF72E6
:10876000C4F20002904215DCB0F1804F29D040F2F3
:108770000042C4F2000222E040F2FF32C4F20102E1
:10878000904212DC41F60002C4F20002904218D07E
:10879000002212E040F60002C4F20002904210D023
:1087A00040F60042C4F2000209E044F20002C4F2C2
:1087B0000102904205D040F20042C4F20102904210
:1087C00002D121F08001816042F2F4420121C2F223
:1087D000000282F83D10002182F83C10016A026A12
:1087E000984222F00102026282690DDC40F2FF73BE
:1087F000C4F20003984215DCB0F1804F2CD040F257
:108800000043C4F2000322E040F2FF33C4F201034C
:10881000984212DC41F60003C4F2000398421BD0D8
:10882000002312E040F60003C4F20003984213D084
:1088300040F60043C4F2000309E044F20003C4F22E
:108840000103984208D040F20043C4F20103984269
:1088500008BF22F0030201E022F0030242F001020D
:1088600022F0F00241F00A01826101628169032372
:1088700021F00C01816181694FF6FF778161016A06
:10888000026A41F0A00122F010020262826922F421
:10889000734202F5807282610162816921F4406154
:1088A000816181698161016A026A41F4206122F477
:1088B00080720262C26942F0010222F0F202C261D9
:1088C0000162C16921F00C01C161C169C161016A24
:1088D000026A41F4204122F480520262C26922F409
:1088E000734202F58072C2610162C16943F60042BF
:1088F00021F44061C161C169C4F20002C16142F268
:10890000F4400021C2F2000080F83C1042F23C50DA
:10891000A2F55052C2F200002091CDE91E110D9136
:10892000CDE90B11C0E90023C0E9021701618161A3
:10893000FAF7E6FB08B172B6FEE74FF480501D90DF
:1089400042F23C50C2F200001DA9FAF7F9FE08B14C
:1089500072B6FEE742F23C50C2F2000090F83D00D1
:1089600030B942F23C510020C2F2000181F83C00D3
:1089700042F23C540220C2F2000484F83D00206818
:10898000211DFDF717FB012084F8460084F83E0006
:1089900084F83F0084F8400084F8410084F84200E5
:1089A00084F8430084F8440084F8450084F83D00CE
:1089B0000620099030200A9009A92046FAF7E0FF26
:1089C00008B172B6FEE742F23C50C2F2000090F8E5
:1089D0003C00012801D172B6FEE742F23C51022070
:1089E000C2F2000181F83D00086841F2FF7342685D
:1089F0008168C4F2000322F07002984242600DDCEC
:108A000040F2FF72C4F20002904215DCB0F1804FD8
:108A100029D040F20042C4F2000222E040F2FF32CC
:108A2000C4F20102904212DC41F60002C4F20002DC
:108A3000904218D0002212E040F60002C4F2000278
:108A4000904210D040F60042C4F2000209E044F225
:108A50000002C4F20102904205D040F20042C4F28A
:108A60000102904202D121F08001816042F23C5229
:108A70000121C2F2000282F83D10002182F83C1070
:108A8000016A026A984222F00102026282690DDCE8
:108A900040F2FF73C4F20003984215DCB0F1804F3E
:108AA00034D040F20043C4F2000322E040F2FF332E
:108AB000C4F20103984212DC41F60003C4F2000341
:108AC000984223D0002312E040F60003C4F20003D2
:108AD00098421BD040F60043C4F2000309E044F280
:108AE0000003C4F20103984210D040F20043C4F2E4
:108AF0000103984208BF22F0030209E000000000D1
:108B000000000000010203040607080922F0030226
:108B100042F0010222F0F00241F00A01826101629A
:108B20008169032321F00C01816181694FF6FF7790
:108B30008161016A026A41F0A00122F01002026222
:108B4000826922F4734202F5807282610162816956
:108B500021F44061816181698161016A026A41F4A5
:108B6000206122F480720262C26942F0010222F0A6
:108B7000F202C2610162C16921F00C01C161C169E7
:108B8000C161016A026A41F4204122F4805202620A
:108B9000C26922F4734202F58072C2610162C16946
:108BA00021F44061C161C169C16142F23C500021C0
:108BB000C2F2000080F83C1043F60040C4F200000E
:108BC000A0F5405242F28450C2F200002091CDE95B
:108BD0001E110D91CDE90B11C0E90023C0E9021768
:108BE00001618161FAF78CFA08B172B6FEE74FF4C1
:108BF00080501D9042F28450C2F200001DA9FAF785
:108C00009FFD08B172B6FEE742F28450C2F2000046
:108C100090F83D0030B942F284510020C2F20001C8
:108C200081F83C0042F284540220C2F2000484F82D
:108C30003D002068211DFDF7BDF9012084F84600A4
:108C400084F83E0084F83F0084F8400084F8410036
:108C500084F8420084F8430084F8440084F8450016
:108C600084F83D000620099030200A9009A920468A
:108C7000FAF786FE08B172B6FEE742F28450C2F2FD
:108C8000000090F83C00012801D172B6FEE742F2E4
:108C900084510220C2F2000181F83D0008680123DE
:108CA0004268816863F3061241F2FF73C4F2000365
:108CB000984242600DDC40F2FF72C4F20002904222
:108CC00015DCB0F1804F29D040F20042C4F200021E
:108CD00022E040F2FF32C4F20102904212DC41F67F
:108CE0000002C4F20002904218D0002212E040F6C6
:108CF0000002C4F20002904210D040F60042C4F2DA
:108D0000000209E044F20002C4F20102904205D0E0
:108D100040F20042C4F20102904202D121F08001EF
:108D2000816042F284520121C2F2000282F83D10B9
:108D3000002182F83C10016A026A984222F0010286
:108D4000026282690DDC40F2FF73C4F200039842B4
:108D500015DCB0F1804F2CD040F20043C4F2000388
:108D600022E040F2FF33C4F20103984212DC41F6E4
:108D70000003C4F2000398421BD0002312E040F627
:108D80000003C4F20003984213D040F60043C4F23B
:108D9000000309E044F20003C4F20103984208D042
:108DA00040F20043C4F20103984208BF22F00302DC
:108DB00001E022F0030242F0010222F0F00241F051
:108DC0000A01826101628169072321F00C0181613E
:108DD00081694FF6FF778161016A026A41F0A00163
:108DE00022F010020262826922F4734202F580725C
:108DF00082610162816921F44061816181698161DF
:108E0000016A026A41F4206122F480720262C2693E
:108E100042F0010222F0F202C2610162C16921F056
:108E20000C01C161C169C161016A026A41F420415A
:108E300022F480520262C26922F4734202F5807207
:108E4000C2610162C16921F44061C161C169C1614E
:108E500042F284500021C2F2000080F83C10002051
:108E6000C4F20200A0F57C4242F25C60C2F2000053
:108E70000C91CDE90A11C0E90023C0E90217C0E94D
:108E800004118161FAF73CF908B172B6FEE74FF4BC
:108E90008050099042F25C60C2F2000009A9FAF722
:108EA0004FFC08B172B6FEE742F25C60C2F200000D
:108EB00090F83D0030B942F25C610020C2F200013E
:108EC00081F83C0042F25C650224C2F2000585F89C
:108ED0003D402868291DFDF76DF8012285F84620E0
:108EE00085F83E2085F83F2085F8402085F8412010
:108EF00085F8422085F8432085F8442085F84520F0
:108F000085F83D2095F83C00012801D172B6FEE7B6
:108F100042F25C60C2F2000080F83D4000684368A5
:108F2000816862F3061341F2FF72C4F200029042BC
:108F300043600DDC40F2FF72C4F20002904215DC87
:108F4000B0F1804F29D040F20042C4F2000222E08A
:108F500040F2FF32C4F20102904212DC41F60002FC
:108F6000C4F20002904218D0002212E040F6000243
:108F7000C4F20002904210D040F60042C4F2000257
:108F800009E044F20002C4F20102904205D040F22E
:108F90000042C4F20102904202D121F080018160BE
:108FA00042F25C620121C2F2000282F83D1000210F
:108FB00082F83C10016A026A41F2FF7322F001025A
:108FC00002628269C4F2000398420DDC40F2FF7332
:108FD000C4F20003984215DCB0F1804F2CD040F26F
:108FE0000043C4F2000322E040F2FF33C4F2010365
:108FF000984212DC41F60003C4F2000398421BD0F1
:10900000002312E040F60003C4F20003984213D09C
:1090100040F60043C4F2000309E044F20003C4F246
:109020000103984208D040F20043C4F20103984281
:1090300008BF22F0030201E022F0030242F0010225
:1090400022F0F00241F00A0182610162816942F27C
:109050000C4621F00C018161816943F60043816176
:10906000016A026A41F0A00122F0100202628269E4
:10907000002722F4734202F58072826101628169E5
:10908000C2F2000621F4406181618169C4F20003EB
:109090008161016A026A41F4206122F480720262F5
:1090A000C26942F0010222F0F202C2610162C169AA
:1090B00021F00C01C161C169C161016A026A41F418
:1090C000204122F480520262C26922F4734202F506
:1090D0008072C2610162C1694FF4827221F4406101
:1090E000C161C169C16142F25C60C2F2000080F8F6
:1090F0003C704FF400701021C6E900320A23C6E923
:109100000277C6E90477C6E90601C6E90877C6E929
:109110000A7396F8513063B10023CDE90633CDE9E7
:10912000043343F6004300244FF0000CC4F2000364
:1091300038E0002186F850100991DAF8100040F468
:109140000040CAF81000DAF8100000F4004009905E
:1091500009980991DAF8000040F00400CAF800000C
:10916000DAF8000000F00400099009984FF4E0508C
:1091700009900220CDE90A010C9006200D90079875
:1091800009A9F9F715F8D6E9047006F11805049055
:1091900023CD0595756AD6E90032D6E902C4079554
:1091A000B56A06954FF0020E86F851E01D6802F48C
:1091B000827225F040051D600CF404452A4404F435
:1091C00000652A4407F002073A44049F01F0380181
:1091D00007F001073A4400F400773A441144059A35
:1091E000012402F080021143069A02F40052114356
:1091F0001960042101EA10400799002201F01001D2
:1092000008445860D86920F40060D8610020C4F296
:109210000200A0F5604141F64460C2F200007265B0
:1092200086F8514001604FF4803141600121C0F661
:1092300000710C92027680F82020C0E90A1280F8B2
:109240003020C0E90222C461C0E90424F8F710FD0F
:1092500008B172B6FEE70A20CDE9090441F6446080
:109260000024C2F2000009A90B94F8F763FC08B1CE
:1092700072B6FEE741F6683140F20000C2F200012A
:10928000C2F20000C1E9AD04012041F62872C1F824
:10929000C442C1F8D04281F89C02C2F200024FF0F1
:1092A000A0401060042010714FF40070D0800220A4
:1092B0000C70C2F8E014C1F8C822C2F80900D481C9
:1092C00092F89514002942D141F628710024C2F287
:1092D000000181F894440994DAF8001041F001018A
:1092E000CAF80010DAF8001001F00101099109999B
:1092F0004FF4C051CDE9091003200C900A200D90C5
:10930000002009A9C4F202000B94F8F751FFDAF823
:1093100004004EF2001140F08000CAF804001D94D1
:10932000DAF81400CEF2000140F48040CAF81400CC
:10933000DAF8140000F480401D901D98DBF800005E
:109340004EF24340CEF2000004700820886041F6DF
:1093500028730320C2F20003002183F89504997159
:10936000D3E9000E826822F0010282605A7A4FF43B
:109370008073B3EB022F63D141F62871C2F2000172
:10938000097C826B002322F480328263C268CFF6AC
:10939000FF73A3F141131A40C260C268012922F48D
:1093A0004012C26003D1C16841F48011C160002144
:1093B00009910999013109910999B1F1706F00F290
:1093C000BA800169002921D40999013109910999CB
:1093D000B1F1706F00F2AF800169002916D40999CC
:1093E000013109910999B1F1706F00F2A48001690E
:1093F00000290BD40999013109910999B1F1706FD4
:1094000000F299800169B1F1FF3FD2DC0A21099194
:109410000999002961D0099901390991099900290F
:109420005BD00999013909910999002955D0099909
:1094300001390991099900294FD009990139E6E7C5
:1094400041F62872C2F20002D268C36843F04003BA
:10945000C36009910999013109910999B1F1706FBE
:1094600000F299800169002920D4099901310991FC
:109470000999B1F1706F00F28E800169002915D44D
:109480000999013109910999B1F1706F00F2838056
:10949000016900290AD40999013109910999B1F1A9
:1094A000706F78D80169B1F1FF3FD3DC0A210991CF
:1094B0000999002941D00999013909910999E1B324
:1094C0000999013909910999B9B3099901390991A2
:1094D000099991B309990139E9E7016941F001015D
:1094E00001610999013109910999B1F1706F22D88F
:1094F0000169C9071DD00999013109910999B1F193
:10950000706F18D80169C90713D009990131099101
:109510000999B1F1706F0ED80169C90709D009998D
:10952000013109910999B1F1706F04D80169C90736
:10953000D7D1002339E0032337E0016941F001016D
:1095400001610999013109910999B1F1706F22D82E
:109550000169C9071DD00999013109910999B1F132
:10956000706F18D80169C90713D0099901310991A1
:109570000999B1F1706F0ED80169C90709D009992D
:10958000013109910999B1F1706F04D80169C907D6
:10959000D7D1002300E00323816B12F47F4F14BF67
:1095A00021F4803141F4803181630EF47F01B1F503
:1095B000803F07D1816841F006018160816841F0F8
:1095C00020018160002B40F03685C1685FFA8EFC77
:1095D00021F0C041C160C16841F08041C160D9F84B
:1095E0000010D9F80020521A0A2A0ED8D9F8002003
:1095F000521A0A2A09D8D9F80020521A0A2A04D87D
:10960000D9F80020521A0B2AEBD34169C90700F0A0
:10961000CF81D9F80010D9F80020521A0A2A0ED8A2
:10962000D9F80020521A0A2A09D8D9F80020521A6B
:109630000A2A04D8D9F80020521A0B2AEBD3416920
:10964000C90700F0B581D9F80010D9F80020521AE6
:109650000A2A0ED8D9F80020521A0A2A09D8D9F8AD
:109660000020521A0A2A04D8D9F80020521A0B2ACC
:10967000EBD34169C90700F09B81D9F80010D9F8F4
:109680000020521A0A2A0ED8D9F80020521A0A2AA3
:1096900009D8D9F80020521A0A2A04D8D9F800208B
:1096A000521A0B2AEBD34169C90700F08181D9F81E
:1096B0000010D9F80020521A0A2A0ED8D9F8002032
:1096C000521A0A2A09D8D9F80020521A0A2A04D8AC
:1096D000D9F80020521A0B2AEBD34169C90700F0D0
:1096E0006781D9F80010D9F80020521A0A2A0ED83A
:1096F000D9F80020521A0A2A09D8D9F80020521A9B
:109700000A2A04D8D9F80020521A0B2AEBD341694F
:10971000C90700F04D81D9F80010D9F80020521A7D
:109720000A2A0ED8D9F80020521A0A2A09D8D9F8DC
:109730000020521A0A2A04D8D9F80020521A0B2AFB
:10974000EBD34169C90700F03381D9F80010D9F88B
:109750000020521A0A2A0ED8D9F80020521A0A2AD2
:1097600009D8D9F80020521A0A2A04D8D9F80020BA
:10977000521A0B2AEBD34169C90700F01981D9F8B5
:109780000010D9F80020521A0A2A0ED8D9F8002061
:10979000521A0A2A09D8D9F80020521A0A2A04D8DB
:1097A000D9F80020521A0B2AEBD34169C90700F0FF
:1097B000FF80D9F80010D9F80020521A0A2A0ED8D2
:1097C000D9F80020521A0A2A09D8D9F80020521ACA
:1097D0000A2A04D8D9F80020521A0B2AEBD341697F
:1097E000C90700F0E580D9F80010D9F80020521A16
:1097F0000A2A0ED8D9F80020521A0A2A09D8D9F80C
:109800000020521A0A2A04D8D9F80020521A0B2A2A
:10981000EBD34169C90700F0CB80D9F80010D9F823
:109820000020521A0A2A0ED8D9F80020521A0A2A01
:1098300009D8D9F80020521A0A2A04D8D9F80020E9
:10984000521A0B2AEBD34169C90700F0B180D9F84D
:109850000010D9F80020521A0A2A0ED8D9F8002090
:10986000521A0A2A09D8D9F80020521A0A2A04D80A
:10987000D9F80020521A0B2AEBD34169C90700F02E
:109880009780D9F80010D9F80020521A0A2A0ED869
:10989000D9F80020521A0A2A09D8D9F80020521AF9
:1098A0000A2A04D8D9F80020521A0B2AEBD34169AE
:1098B000C9077DD0D9F80010D9F80020521A0A2A19
:1098C0000ED8D9F80020521A0A2A09D8D9F800204F
:1098D000521A0A2A04D8D9F80020521A0B2AEBD3BC
:1098E0004169C90764D0D9F80010D9F80020521A8C
:1098F0000A2A0ED8D9F80020521A0A2A09D8D9F80B
:109900000020521A0A2A04D8D9F80020521A0B2A29
:10991000EBD34169C9074BD0D9F80010D9F8002022
:10992000521A0A2A0ED8D9F80020521A0A2A09D83F
:10993000D9F80020521A0A2A04D8D9F80020521A5D
:109940000B2AEBD34169C90732D0D9F80010D9F8F6
:109950000020521A0A2A0ED8D9F80020521A0A2AD0
:1099600009D8D9F80020521A0A2A04D8D9F80020B8
:10997000521A0B2AEBD34169C90719D0D9F8001044
:10998000D9F80020521A0A2A0ED8D9F80020521A03
:109990000A2A09D8D9F80020521A0A2A04D8D9F874
:1099A0000020521A0B2AEBD34169C90740F079868F
:1099B000BCF1000F00F0FE800EF00303BCF1040FB9
:1099C0004FF0000242D341F62871C2F20001A1F12A
:1099D00090070EF0FC04012100256E1C87F8C8607A
:1099E000A7F8E260AE1C87F8A450A7F8BE5087F82D
:1099F000EC60A7F80661EE1C043587F8A51087F81F
:109A0000A820C7E92B22C7F8B42087F8C91087F827
:109A1000CC20C7E93422C7F8D82087F8ED1087F8A2
:109A2000F020C7E93D22C7F8FC2087F8111187F81C
:109A30001061A7F82A6187F81421C7E94622C7F800
:109A40002021A54207F19007C7D12A46B3B341F6BA
:109A5000287402EBC201C2F2000404EB8105012468
:109A60000021012B6C752A75EA852976C5E9071155
:109A7000696223D0551C41F6287605EBC507C2F272
:109A8000000606EB8707022B7C753D75FD85397650
:109A9000C7E90711796211D0911C41F6287401EBD6
:109AA000C102C2F2000404EB820201241175D185C7
:109AB000002154751176C2E907115162BCF1040FFF
:109AC0004FF0000237D341F628770EF0FC01C2F2C6
:109AD000000700256E1C87F87862AE1C87F8545288
:109AE00087F89C62EE1C043587F8552287F85822C7
:109AF000C7E99722C7F8642287F8792287F87C2281
:109B0000C7E9A022C7F8882287F89D2287F8A022FB
:109B1000C7E9A922C7F8AC2287F8C12287F8C0623A
:109B200087F8C422C7E9B222C7F8D0228D4207F1D4
:109B30009007CFD12A46EBB341F6287702EBC2015A
:109B4000C2F2000707EB81070021012B87F85512AD
:109B500087F8542287F85812C7E99711C7F864129A
:109B600028D0571C41F6287507EBC706C2F200053E
:109B700005EB8606022B86F8551286F8547286F895
:109B80005812C6E99711C6F8641213D0911C41F619
:109B9000287301EBC102C2F2000303EB820200232F
:109BA00082F8553282F8541282F85832C2E997335B
:109BB000C2F8643241F62871C2F200014A68079285
:109BC0008A68C9680692C1F307410022C0F80421DF
:109BD000C0F80821C0F80C21C0F81021C0F81421E9
:109BE000C0F81821C0F81C21C0F82021C0F8242199
:109BF000C0F82821C0F82C21C0F83021C0F8342149
:109C0000C0F838210491C0F83C2139B1816B21F4AE
:109C100000118163816B41F4002110E0D0F8041839
:109C200041F00201C0F80418816B41F40011816316
:109C3000816B21F400218163816B21F48021816398
:109C4000069A002102F47F42B2F5807FC0F8001E20
:109C500008D1D0F80028079BB1EB136F07D1C0F8EB
:109C6000002808E0D0F8001841F0030101E042F0BC
:109C70000101C0F8001800210991099901310991E9
:109C80000999B1F1706F50D8016900291ED4099962
:109C9000013109910999B1F1706F46D80169002924
:109CA00014D40999013109910999B1F1706F3CD827
:109CB000016900290AD40999013109910999B1F181
:109CC000706F32D80169B1F1FF3FD6DC00210991F4
:109CD0004FF4846101610999013109910999B1F148
:109CE000706F22D8016989061DD509990131099142
:109CF0000999B1F1706F18D80169890613D50999CE
:109D0000013109910999B1F1706F0ED80169890685
:109D100009D50999013109910999B1F1706F04D8F8
:109D200001698906D7D4002100E0012105910021B5
:109D300009910999013109910999B1F1706F4ED8D2
:109D4000016900291ED40999013109910999B1F1DC
:109D5000706F44D80169002914D40999013109911F
:109D60000999B1F1706F3AD8016900290AD40999AB
:109D7000013109910999B1F1706F30D80169B1F1E0
:109D8000FF3FD6DC002109911021016109990131C1
:109D900009910999B1F1706F21D80169C90620D5DF
:109DA0000999013109910999B1F1706F17D80169C9
:109DB000C90616D50999013109910999B1F1706F58
:109DC0000DD80169C9060CD5099901310991099984
:109DD000B1F1706F03D80169C906D7D401E0012140
:109DE00005914FF0000BC0F810B8C0F814B80799EF
:109DF000C0F81CB8C9B2002900F0F080D0F80039D2
:109E00004FF0006202EA1313C0F800394FF67F37B3
:109E10004B1EC0F810B9C0F8087909D0A1F1020CA6
:109E2000BCF1030F03F0030103910FD2012241E0C3
:109E3000D0F8003B00F5306102EA1312C0F8002BA5
:109E400000220A614FF67F328A60C7E023F00304E4
:109E500000F5186700254FF0904E4FF67F36002230
:109E600057F8601C04320EEAE17147F8601C47F8AD
:109E7000505C47F8586C57F8401C94420EEAE17168
:109E800047F8401C47F8305C47F8386C57F8201CFE
:109E90000EEAE17147F8201C47F8105C47F8186C8F
:109EA00039680EEAE17139603D61BE6007F18007F3
:109EB000D6D10132039939B300F510615701CD595C
:109EC0004FF0904E01EB42160EEAE5750024CD519D
:109ED0003461039A4FF67F35012AB56014D03944B6
:109EE0000F6A0EEAE7720A620C63039A8D62022A15
:109EF0000AD00A6C4FF0904707EAE2720A64002227
:109F00000A654FF67F328A64D0F8001B4FF000627A
:109F100002EA1111C0F8001B0021C0F8101B4FF617
:109F20007F31002BC0F8081B58D0BCF1030F01D2C1
:109F3000012233E023F0030300F5386700254FF0DA
:109F400090444FF67F32002157F8606C043104EAE8
:109F5000E67647F8606C47F8505C47F8582C57F89D
:109F6000406C8B4204EAE67647F8406C47F8305C78
:109F700047F8382C57F8206C04EAE67647F8206C4E
:109F800047F8105C47F8182C3E6804EAE6763E6015
:109F90003D61BA6007F18007D6D14A1C0399E9B147
:109FA00000F530615301CF5801EB42164FF090425B
:109FB00002EAE7770025CF503561039C4FF67F37E3
:109FC000012CB7600AD019440B6A02EAE3720A62F4
:109FD0000D63039A8F62022A40F0FA80D0F81018BD
:109FE00021F48071C0F81018C0F818B0079A6FF00B
:109FF000804112F47F0F416103D1816941F010016A
:10A000008161816943F60002C8F23C021143069A5D
:10A01000816112F47F0F03D0816941F008018161F1
:10A020000499012905D181690422C4F20002114377
:10A030008161059840B141F628710220C2F2000109
:10A0400081F8950472B6FEE741F628720020C2F24C
:10A0500000020121507482F895141168D1F8002E85
:10A0600022F00302C1F8002ED1F8042842F00202C7
:10A07000C1F8042880224A624A6A42F480028A6255
:10A080004A6A8B6A02EB134242F40002C1F80421CF
:10A0900040F2200141F66832C2F20001C2F2000231
:10A0A000C2F8B812D2F8D41202F52E7252F821205A
:10A0B000ADF82400D26A4AB109A8904741F6683247
:10A0C000C2F20002D2F8D412C2F8D00241F66833CC
:10A0D000C2F2000303EB810040F2BC01C2F20001B6
:10A0E000C0F8C412D3F8C802D3F8D82290F8941458
:10A0F000012902F10101C3F8D81201D110211DE09C
:10A100000168CA68520606D5427B012A03D18A6BD0
:10A1100042F480328A638A6842F001028A60D1F890
:10A12000002E22F00302C1F8002ED1F8042822F0FC
:10A130000202C1F80428002180F8941440F2003093
:10A14000C0F20130C840C00716D143F60040C4F247
:10A15000000042F21465A0F52050C2F20005002173
:10A160000122C5E900012846C5E90212A961F8F7F4
:10A17000C7FF18B172B6FEE772B6FEE795F83D006C
:10A180000224002804BF002085F83C0085F83D40EB
:10A190002868291DFBF70EFF2868016821F00801D7
:10A1A0000160016841F008010160012185F8461055
:10A1B00085F83E1085F83F1085F8421085F8431069
:10A1C00085F83D1095F83C10012909D172B6FEE7DB
:10A1D00051F8402F4FF0904303EAE2720A602FE6F5
:10A1E00085F83D40426841F2FF738168C4F2000384
:10A1F00022F07002984242600DDC40F2FF72C4F21D
:10A200000002904215DCB0F1804F29D040F20042AC
:10A21000C4F2000222E040F2FF32C4F20102904296
:10A2200012DC41F60002C4F20002904218D0002273
:10A2300012E040F60002C4F20002904210D040F654
:10A240000042C4F2000209E044F20002C4F201023A
:10A25000904205D040F20042C4F20102904202D185
:10A2600021F080018160012043F6004142F2CC5B85
:10A2700085F83D000020C4F20001C2F2000B42F656
:10A28000E06385F83C00A1F530514FF6FF72CBE951
:10A290000203CBF818005846CBE90012F8F730FF5C
:10A2A00008B172B6FEE79BF83C00012801D172B6F6
:10A2B000FEE702208BF83D00DBF8000041F2FF735F
:10A2C00042688168C4F2000322F070029842426042
:10A2D0000DDC40F2FF72C4F20002904215DCB0F1D6
:10A2E000804F29D040F20042C4F2000222E040F246
:10A2F000FF32C4F20102904212DC41F60002C4F2C5
:10A300000002904218D0002212E040F60002C4F28F
:10A310000002904210D040F60042C4F2000209E070
:10A3200044F20002C4F20102904205D040F2004221
:10A33000C4F20102904202D121F08001816001202B
:10A340008BF83D0043F60040C4F2000041F6D462B1
:10A3500048F2A064002500F5C050C2F200024FF49C
:10A360008041C0F201048BF83C5082E83100C2E920
:10A370000351C2E90555C2E9075592F83D1009B1EC
:10A3800021462EE041F6D466C2F2000686F83C5023
:10A390000995DAF8000009A940F00200CAF80000A7
:10A3A000DAF8000000F0020009900998C020099036
:10A3B0001220CDE90A0503200C9004200D90089886
:10A3C000F7F7F6FE1D95DAF8100040F40010CAF811
:10A3D0001000DAF8100000F400101D901D98D6E966
:10A3E000000141F6D4632422C2F2000383F83D2029
:10A3F00002684EF27C2722F0010202600268C0F679
:10A40000000742F400420260026822F40042026047
:10A4100040F21C02C2F2000212685AF8283CC3F350
:10A420008223FB5C671C22FA03F340F60012C0F2A1
:10A430003D02B9423CBF48F28042C0F21E029A423D
:10A4400001D972B6FEE74DF68362C4F21B32A3FB5C
:10A4500002264268B50C22F03F0242EA96424FF4CF
:10A4600096744260654348F63814026AC0F24104AB
:10A47000A5FB045422F03F02B94238BFB40C661C5D
:10A4800032430262C2694CF6FF76B243B942A3F18D
:10A49000010309D24900B3FBF1F101316FF31F3120
:10A4A000042998BF04211CE041F6D467C2F20007DA
:10A4B000BF6857B119277943B3FBF1F101316FF34D
:10A4C0001F3169B101F5804107E001EB4101B3FBA8
:10A4D000F1F101316FF31F3111B101F5004100E0DD
:10A4E00001211143C16141F6D4650168C2F2000542
:10A4F000D5E9072321F0C0011143194301608168A8
:10A5000048F2FF3205F10C0791438CCF19431143F8
:10A51000AE698160C168002421F0FF0139433143F5
:10A52000C1600168012341F00101016020202C6419
:10A5300085F83D000020C4F20200A0F55F4141F61D
:10A540008C602C6385F83E40C2F200000125C0F605
:10A5500000730C944FF48032047680F82040C0E9F8
:10A560000A34C56180F8304080E81600C0E9034530
:10A570004561F7F77DFB08B172B6FEE70B20CDE928
:10A58000090541F68C600DF1240AC2F20000514623
:10A590000B94F7F7CFFA08B172B6FEE740F6184110
:10A5A0004FF600024FF48050C4F20201CFF6FF7262
:10A5B0008850D9F8000040F6B83140F6B932D9F8E1
:10A5C00000301B1A8B420ED8D9F800301B1A8B4270
:10A5D00009D8D9F800301B1A8B4204D8D9F80030BA
:10A5E0001B1A9342EBD34EF28420C0F60000FDF715
:10A5F00007F94EF29830C0F60000FDF701F94EF26F
:10A60000AB20C0F60000FDF7FBF84EF27230C0F64A
:10A610000000FDF7F5F80FF67860FDF7F1F80FF69A
:10A62000BC60FDF7EDF80FF6906000900FF69060BB
:10A630000121002200230024FDF7E2F841F6583002
:10A64000C2F20000C0E9004441F6D460C2F200004A
:10A65000D9F8001090F83D00202840F0F88041F62D
:10A66000D460C2F2000000688269920731D5D9F83F
:10A670000020521A1A2AF7D382699207F4D541F6BC
:10A68000D4620020C2F200022021106382F83D1043
:10A6900082F83E00106C022440F02000106400F0AC
:10A6A0001DBCD9F80010D9F80020521A0A2A0ED879
:10A6B000D9F80020521A0A2A09D8D9F80020521ACB
:10A6C0000A2A04D8D9F80020521A0A2AEBD940697C
:10A6D000B1E441F6D461C2F2000191F83C100129C5
:10A6E00000F0B58041F6D4620121C2F2000282F886
:10A6F0003C100168C90703D1016841F00101016004
:10A70000016821F400610160222182F83D1040219E
:10A7100082F83E100021116441F65831C2F2000166
:10A72000516208215185518D11850021CFF6FF71AD
:10A73000D162016841F480610160016841F4807177
:10A7400001604169C90709D14169C90704BF41696D
:10A750005FEAC17102D14169C907F2D0A02101614C
:10A76000F9F78AF9002872D1002141F6D4600991E5
:10A77000C2F2000000684269099282690992099A4E
:10A780004269120615D4426952052BD44269120659
:10A790000FD44269520525D44269120609D4426990
:10A7A00052051FD44269120603D442695205E7D507
:10A7B00018E001614169090631D44169490511D4A4
:10A7C000416909062BD4416949050BD44169090641
:10A7D00025D44169490505D4416909061FD4416959
:10A7E0004905E7D56FF4806141F6D46341610021EA
:10A7F000C2F200032022196383F83D2083F83E1043
:10A800001A6C42F004021A6483F83C10196C042993
:10A810001DD10168022441F40071016018E0016853
:10A8200041F4807101604169C90709D14169C907D3
:10A8300004BF41695FEAC17102D14169C907F2D021
:10A84000A1210161F9F718F9002800F0E181022443
:10A850004EF208304EF2E921C0F60000002C18BF7D
:10A860000124C0F6000108BF0846FCF7C9FF41F605
:10A870006032C2F20002107840EAC4000106107093
:10A8800041F07B8540F618414FF40030C4F20201DC
:10A890000860D9F80000D9F80010091A01290ED86B
:10A8A000D9F80010091A012909D8D9F80010091A95
:10A8B000012904D8D9F80010091A0229EBD3F5F7B9
:10A8C00021FD8DF82400F5F71DFD8DF82500F5F725
:10A8D00019FD8DF82600F5F715FD8DF82700F5F721
:10A8E00011FD8DF82800002040F618478DF87800FB
:10A8F0001D9010254FF48036C4F202070DF1870039
:10A9000001218DF887503E600124F8F723FB1DA834
:10A910000521F8F785F930203C608DF887000DF1AE
:10A92000870001213E60F8F715FB09A80521F8F71B
:10A9300011FB0DF1870001213C608DF887503E60CE
:10A94000F8F708FB1DA80521F8F76AF93C609DF8A7
:10A9500074009DF82410884240F079819DF87500BC
:10A960009DF82510884240F072819DF876009DF890
:10A970002610884240F06B819DF877009DF82710E3
:10A98000884240F064819DF878009DF82810884244
:10A9900040F05D810FF69430FCF732FF40F6184727
:10A9A0004FF40030C4F202073860E2208DF8240032
:10A9B0004FF4803609A801213E600125F8F7CAFA54
:10A9C000E1203D608DF8240009A801213E60F8F7E0
:10A9D000C1FA07203D608DF8240009A801213E60DE
:10A9E000F8F7B8FA1DA80121F8F71AF93D609DF8AB
:10A9F0007400272100F070008DF824108DF8740089
:10AA000009A801213E60F8F7A5FA1DA80121F8F771
:10AA1000A1FA23203D608DF8240003208DF87400F6
:10AA200009A801213E60F8F795FA1DA80121F8F761
:10AA300091FA21203D608DF8240009A801218DF8AC
:10AA400074503E60F8F786FA1DA80121F8F782FAE3
:10AA500022203D608DF8240009A801218DF8745052
:10AA60003E60F8F777FA1DA80121F8F773FA302055
:10AA70003D608DF8240009A801213E60F8F76AFACC
:10AA800041F65834C2F2000420460521F8F762FA74
:10AA90002A203D608DF8240009A801213E60F8F7C6
:10AAA00059FA20460521F8F755FA24203D608DF823
:10AAB000240048208DF8740009A801213E60F8F7B1
:10AAC00049FA1DA80121F8F745FA26203D608DF8C6
:10AAD0002400062409A801218DF874403E60F8F78F
:10AAE00039FA1DA80121F8F735FA3C203D608DF8B0
:10AAF000240009A801218DF874503E60F8F72AFA65
:10AB00001DA80121F8F726FA1D203D608DF82400CC
:10AB100009A801213E60F8F71DFA1DA80121F8F7E8
:10AB20007FF83D609DF87400800722D450208DF896
:10AB30002400732040F618478DF87400C4F2020711
:10AB400009A801213E60F8F705FA1DA80121F8F7D0
:10AB500001FA3D203D608DF8240009A801218DF8FF
:10AB600074403E60F8F7F6F91DA80121F8F7F2F9F4
:10AB70003D6041F65830C2F2000046797D2E1AD869
:10AB8000252040F618458DF824004FF48030C4F29B
:10AB900002058DF87460286009A801210124F8F7E6
:10ABA000D9F91DA80121F8F7D5F941F658302C60E4
:10ABB000C2F20000467941F65837C2F200073978F0
:10ABC0007A78BB78F8783F790296CDE900074EF2A3
:10ABD000BD30C0F60000FCF713FE20208DF82400E5
:10ABE0002E2040F618458DF874004FF48030C4F2E2
:10ABF0000205286009A801210124F8F7ABF91DA876
:10AC00000121F8F7A7F902202C60286000201FE03E
:10AC100041F6D460C2F20000028D002A00F04481A7
:10AC2000022A00F06381012A40F06C81006801680B
:10AC300021F48061016000210991416909918169D4
:10AC400009910999016841F40071016066E10220EF
:10AC500041F66032C2F20002117840F6184708430C
:10AC600010704FF48014C4F2020776203C608DF817
:10AC7000240000208DF8740009A801213C60012601
:10AC8000F8F768F91DA80121F8F764F91025F520F7
:10AC90003D603C608DF8240009A80121F8F75AF9BD
:10ACA0001DA80121F7F7BCFF3D609DF874004728FF
:10ACB00040F0148211208DF8746040F618468DF82B
:10ACC0002400C4F2020609A801213460F8F742F911
:10ACD0001DA80121F8F73EF93560D9F80000D9F830
:10ACE0000010091A0A290ED8D9F80010091A0A29E1
:10ACF00009D8D9F80010091A0A2904D8D9F800107F
:10AD0000091A0B29EBD376208DF82400002040F699
:10AD100018478DF874004FF48015C4F2020709A893
:10AD200001213D60F8F716F91DA80121F8F712F985
:10AD3000102614203E608DF8240002208DF8740047
:10AD400009A801213D60F8F705F91DA80121F8F7D0
:10AD500001F9E4203E603D608DF8240009A801213E
:10AD6000F8F7F8F81DA80121F7F75AFF3E609DF8A3
:10AD70007400642100F0EF008DF824108DF8740049
:10AD800009A801213D60F8F7E5F81DA80121F8F7B1
:10AD9000E1F865203E608DF8240008208DF87400ED
:10ADA00009A801213D60F8F7D5F81DA80121F8F7A1
:10ADB000D1F850203E608DF82400482409A80121D4
:10ADC0008DF874403D60F8F7C5F81DA80121F8F72B
:10ADD000C1F84F203E608DF8240009A801218DF8AC
:10ADE00074403D60F8F7B6F81DA80121F8F7B2F8F5
:10ADF0003E60D9F80000D9F80010091A01290ED8D0
:10AE0000D9F80010091A012909D8D9F80010091A2F
:10AE1000012904D8D9F80010091A0229EBD37620A9
:10AE20008DF82400002040F618468DF874004FF489
:10AE30008014C4F2020609A801213460F8F78AF8E8
:10AE40001DA80121F8F786F810254E2035608DF8F1
:10AE500024000F208DF8740009A801213460F8F750
:10AE600079F81DA80121F8F775F83560D9F80000C8
:10AE7000D9F80010091A0A290ED8D9F80010091AB1
:10AE80000A2909D8D9F80010091A0A2904D8D9F8CA
:10AE90000010091A0B29EBD34EF23930C0F600002E
:10AEA000FCF7AEFC00201AE10020099041F6D460C6
:10AEB000C2F200000068416909918169099109990C
:10AEC000016841F40071016041F6D4612020C2F2B2
:10AED0000001002481F83D0081F83E4041F6D46134
:10AEE0000020C2F2000181F83C00B1E40068016872
:10AEF00021F480610160016841F40061016000217A
:10AF0000099106E00020099041F6D460C2F20000E9
:10AF100000684169099181690991099941F6D461F3
:10AF2000C2F200014F6A93B2032B21D8012B44D007
:10AF3000022B7BD14269520709D4426952075CBF98
:10AF400042695FEA427202D442695207F2D502684E
:10AF500041F6D46142F4007202600269C2F200015B
:10AF600007F8012B4A8D013A4A8550E0D9F80010C4
:10AF70004169490600F196804169C90600F11181D5
:10AF8000D9F800104169490600F18C804169C90671
:10AF900000F10781D9F800104169490600F182806B
:10AFA0004169C90600F1FD80D9F8001041694906E0
:10AFB00078D44169C906D9D5F3E04269520626D44E
:10AFC0004269D20600F1ED80D9F8002042695206AC
:10AFD0001DD44269D20600F1E480D9F8002042690C
:10AFE000520614D44269D20600F1DB80D9F8002061
:10AFF000426952060BD44269D20600F1D280D9F8D8
:10B000000020426952064FF00102D9D500E001222A
:10B01000016941F6D46307F8011BC2F20003013A4B
:10B020005F621A85598D013959854BE043695B0789
:10B0300009D443695B075CBF43695FEA437302D489
:10B0400043695B07F2D50368394623F480630360E4
:10B05000036901F8013B41F6D463C2F2000359626F
:10B06000511E1985598D013959854169490709D4FE
:10B07000416949075CBF41695FEA417102D4416996
:10B080004907F2D5016841F6D46341F400710160CB
:10B090000169C2F200037970598D02370139023A11
:10B0A0005985B5E7016941F6D46307F8011BC2F27F
:10B0B0000003013A5F621A85598D0139598541694A
:10B0C000490703D411047FF42EAFFDE691B20329A2
:10B0D0009ED1016821F48061016099E7042041F666
:10B0E0006032C2F2000211780843107041F04581CD
:10B0F00042F2644072B6C2F20000066841F21111D9
:10B10000306A084208D1306A40F24441084203D113
:10B11000306820F00100306000207062F06842F278
:10B12000644120F00100F060C2F2000191F83E009D
:10B1300091F8427040F2FF7340F6000240F6004C76
:10B1400040F200410128C4F20003C4F20002C4F23C
:10B15000000CC4F2000108BF012F5FD142F264402D
:10B160000227C2F2000080F83E7080F84270F76853
:10B1700041F2FF7047F00207F760376AC4F200003F
:10B1800027F001073762376A864247F001073762C6
:10B190001CDC9E4228DCB6F1804F36D08E4234D083
:10B1A00038E06FF0100141F6D46241610020C2F234
:10B1B00000022021106382F83D1082F83E00116CDD
:10B1C0000224116482F83C00FFF742BB40F2FF37D3
:10B1D000C4F20107BE420CDC41F60007C4F20007CE
:10B1E000BE4212D000270CE096420ED066450CD02D
:10B1F00010E044F20007C4F20107BE4205D040F25D
:10B200000047C4F20107BE4204D1B76807F0070740
:10B21000062F03D0376847F00107376042F26440D9
:10B22000C2F2000090F83F5090F84370012D08BF23
:10B23000012F46D1022780F83F7080F84370F768ED
:10B2400041F2FF7047F00407F760376AC4F200006C
:10B2500027F010073762376A864247F010073762D7
:10B2600007DC9E4213DCB6F1804F21D08E421FD006
:10B2700023E040F2FF37C4F20107BE420CDC41F686
:10B280000007C4F20007BE4212D000270CE096422D
:10B290000ED066450CD010E044F20007C4F201075E
:10B2A000BE4205D040F20047C4F20107BE4204D1BD
:10B2B000B76807F00707062F03D0376847F0010784
:10B2C000376042F26440C2F2000090F8405090F8BB
:10B2D0004470012D08BF012F46D1022780F840702D
:10B2E00080F84470F76841F2FF7047F00807F76094
:10B2F000376AC4F2000027F480773762376A8642E3
:10B3000047F48077376207DC9E4213DCB6F1804F4A
:10B3100021D08E421FD023E040F2FF37C4F2010754
:10B32000BE420CDC41F60007C4F20007BE4212D058
:10B3300000270CE096420ED066450CD010E044F297
:10B340000007C4F20107BE4205D040F20047C4F234
:10B350000107BE4204D1B76807F00707062F03D0E4
:10B36000376847F00107376042F26440C2F20000DC
:10B3700090F8415090F84570012D08BF012F46D13B
:10B38000022780F8417080F84570F76841F2FF703D
:10B3900047F01007F760376AC4F2000027F48057BF
:10B3A0003762376A864247F48057376207DC9E422D
:10B3B00013DCB6F1804F21D08E421FD023E040F243
:10B3C000FF37C4F20107BE420CDC41F60007C4F2AD
:10B3D0000007BE4212D000270CE096420ED0664510
:10B3E0000CD010E044F20007C4F20107BE4205D0C1
:10B3F00040F20047C4F20107BE4204D1B76807F02B
:10B400000707062F03D0376847F001073760D8F8E1
:10B41000005041F211142F6A274208D12F6A40F2DE
:10B420004444274203D12F6827F001072F600027EB
:10B430006F62EF68404627F00107EF6098F83E40E2
:10B4400098F84270012C08BF012F40F08C80022731
:10B4500088F83E7088F84270EF68404647F002076F
:10B46000EF602F6A41F2FF7027F001072F622F6A09
:10B47000C4F2000047F0010785422F6242DC9D4282
:10B480004EDCB5F1804F65D08D4263D067E000BFE0
:10B490005C5F5F5F5F2F5C5F5F2C202F5F2F202F33
:10B4A0005F2F202F5F2F202E5F5F5F2F5F2F5C5F4E
:10B4B0005F5F2F200A0000002D416C706861000062
:10B4C000547261636B65722056657273696F6E3A70
:10B4D00025752E25752E257525730A002020202020
:10B4E000202F5F5F5F5F2F20202020202020202042
:10B4F0002F5F2F2020202020202020202020200A05
:10B500000A00000040F2FF37C4F20107BD4215DC1B
:10B5100041F60007C4F20007BD421BD0002715E02A
:10B52000954217D0654515D019E000BF574C414EE4
:10B5300020436865636B6564210A000044F20007DC
:10B54000C4F20107BD4205D040F20047C4F2010732
:10B55000BD4204D1AF6807F00707062F03D02F685C
:10B5600047F001072F6098F83F404046012C98F8BB
:10B57000437008BF012F47D1022788F83F7088F831
:10B580004370EF68404647F00407EF602F6A41F2CE
:10B59000FF7027F010072F622F6AC4F2000047F0F7
:10B5A000100785422F6207DC9D4213DCB5F1804F06
:10B5B00021D08D421FD023E040F2FF37C4F20107B3
:10B5C000BD420CDC41F60007C4F20007BD4212D0B8
:10B5D00000270CE095420ED065450CD010E044F2F7
:10B5E0000007C4F20107BD4205D040F20047C4F293
:10B5F0000107BD4204D1AF6807F00707062F03D04B
:10B600002F6847F001072F6098F840404046012C12
:10B6100098F8447008BF012F47D1022788F840707E
:10B6200088F84470EF68404647F00807EF602F6ADB
:10B6300041F2FF7027F480772F622F6AC4F2000076
:10B6400047F4807785422F6207DC9D4213DCB5F119
:10B65000804F21D08D421FD023E040F2FF37C4F24B
:10B660000107BD420CDC41F60007C4F20007BD42F1
:10B6700012D000270CE095420ED065450CD010E0AA
:10B6800044F20007C4F20107BD4205D040F2004772
:10B69000C4F20107BD4204D1AF6807F00707062FC7
:10B6A00003D02F6847F001072F6098F841404046CB
:10B6B000012C98F8457008BF012F46D1022788F861
:10B6C000417088F84570EF6841F2FF7047F010074D
:10B6D000EF602F6AC4F2000027F480572F622F6AB0
:10B6E000854247F480572F6207DC9D4213DCB5F199
:10B6F000804F21D08D421FD023E040F2FF37C4F2AB
:10B700000107BD420CDC41F60007C4F20007BD4250
:10B7100012D000270CE095420ED065450CD010E009
:10B7200044F20007C4F20107BD4205D040F20047D1
:10B73000C4F20107BD4204D1AF6807F00707062F26
:10B7400003D02F6847F001072F6042F2F440C2F2A5
:10B750000000056841F211142F6A274208D12F6AB0
:10B7600040F24444274203D12F6827F001072F609D
:10B7700000276F62EF6827F00107EF6090F83E4006
:10B7800090F84270012C08BF012F46D1022780F8A3
:10B790003E7080F84270EF6841F2FF7047F0020798
:10B7A000EF602F6AC4F2000027F001072F622F6AB2
:10B7B000854247F001072F6207DC9D4213DCB5F19B
:10B7C000804F21D08D421FD023E040F2FF37C4F2DA
:10B7D0000107BD420CDC41F60007C4F20007BD4280
:10B7E00012D000270CE095420ED065450CD010E039
:10B7F00044F20007C4F20107BD4205D040F2004701
:10B80000C4F20107BD4204D1AF6807F00707062F55
:10B8100003D02F6847F001072F6042F2F440C2F2D4
:10B82000000090F83F4090F84370012C08BF012FB2
:10B8300046D1022780F83F7080F84370EF6841F2EC
:10B84000FF7047F00407EF602F6AC4F2000027F092
:10B8500010072F622F6A854247F010072F6207DC1E
:10B860009D4213DCB5F1804F21D08D421FD023E0E3
:10B8700040F2FF37C4F20107BD420CDC41F600077D
:10B88000C4F20007BD4212D000270CE095420ED052
:10B8900065450CD010E044F20007C4F20107BD4238
:10B8A00005D040F20047C4F20107BD4204D1AF68A1
:10B8B00007F00707062F03D02F6847F001072F6016
:10B8C00042F2F440C2F2000090F8404090F8447018
:10B8D000012C08BF012F46D1022780F8407080F864
:10B8E0004470EF6841F2FF7047F00807EF602F6A7D
:10B8F000C4F2000027F480772F622F6A854247F454
:10B9000080772F6207DC9D4213DCB5F1804F21D098
:10B910008D421FD023E040F2FF37C4F20107BD4241
:10B920000CDC41F60007C4F20007BD4212D000272C
:10B930000CE095420ED065450CD010E044F20007B3
:10B94000C4F20107BD4205D040F20047C4F201072E
:10B95000BD4204D1AF6807F00707062F03D02F6858
:10B9600047F001072F6042F2F440C2F2000090F865
:10B97000414090F84570012C08BF012F46D10227A5
:10B9800080F8417080F84570EF6841F2FF7047F031
:10B990001007EF602F6AC4F2000027F480572F626F
:10B9A0002F6A854247F480572F6207DC9D4213DCE3
:10B9B000B5F1804F21D08D421FD023E040F2FF37F8
:10B9C000C4F20107BD420CDC41F60007C4F20007D7
:10B9D000BD4212D000270CE095420ED065450CD038
:10B9E00010E044F20007C4F20107BD4205D040F266
:10B9F0000047C4F20107BD4204D1AF6807F0070752
:10BA0000062F03D02F6847F001072F6042F23C5009
:10BA1000C2F20000056841F211142F6A274208D1D2
:10BA20002F6A40F24444274203D12F6827F00107D0
:10BA30002F6000276F62EF6827F00107EF6090F832
:10BA40003E4090F84270012C08BF012F46D10227DA
:10BA500080F83E7080F84270EF6841F2FF7047F066
:10BA60000207EF602F6AC4F2000027F001072F627F
:10BA70002F6A854247F001072F6207DC9D4213DCE5
:10BA8000B5F1804F21D08D421FD023E040F2FF3727
:10BA9000C4F20107BD420CDC41F60007C4F2000706
:10BAA000BD4212D000270CE095420ED065450CD067
:10BAB00010E044F20007C4F20107BD4205D040F295
:10BAC0000047C4F20107BD4204D1AF6807F0070781
:10BAD000062F03D02F6847F001072F6042F23C5039
:10BAE000C2F2000090F83F4090F84370012C08BF6C
:10BAF000012F46D1022780F83F7080F84370EF682D
:10BB000041F2FF7047F00407EF602F6AC4F20000B3
:10BB100027F010072F622F6A854247F010072F6227
:10BB200007DC9D4213DCB5F1804F21D08D421FD040
:10BB300023E040F2FF37C4F20107BD420CDC41F6BE
:10BB40000007C4F20007BD4212D000270CE0954266
:10BB50000ED065450CD010E044F20007C4F2010796
:10BB6000BD4205D040F20047C4F20107BD4204D1F6
:10BB7000AF6807F00707062F03D02F6847F00107CB
:10BB80002F6042F23C50C2F2000090F8404090F822
:10BB90004470012C08BF012F46D1022780F8407065
:10BBA00080F84470EF6841F2FF7047F00807EF60DB
:10BBB0002F6AC4F2000027F480772F622F6A854233
:10BBC00047F480772F6207DC9D4213DCB5F1804F8C
:10BBD00021D08D421FD023E040F2FF37C4F201078D
:10BBE000BD420CDC41F60007C4F20007BD4212D092
:10BBF00000270CE095420ED065450CD010E044F2D1
:10BC00000007C4F20107BD4205D040F20047C4F26C
:10BC10000107BD4204D1AF6807F00707062F03D024
:10BC20002F6847F001072F6042F23C50C2F200003B
:10BC300090F8414090F84570012C08BF012F46D183
:10BC4000022780F8417080F84570EF6841F2FF707C
:10BC500047F01007EF602F6AC4F2000027F4805706
:10BC60002F622F6A854247F480572F6207DC9D427E
:10BC700013DCB5F1804F21D08D421FD023E040F27C
:10BC8000FF37C4F20107BD420CDC41F60007C4F2E5
:10BC90000007BD4212D000270CE095420ED065454A
:10BCA0000CD010E044F20007C4F20107BD4205D0F9
:10BCB00040F20047C4F20107BD4204D1AF6807F06B
:10BCC0000707062F03D02F6847F001072F6042F2C5
:10BCD0008450C2F20000056841F211142F6A274215
:10BCE00008D12F6A40F24444274203D12F6827F03D
:10BCF00001072F6000276F62EF6827F00107EF60F0
:10BD000090F83E4090F84270012C08BF012F46D1B8
:10BD1000022780F83E7080F84270EF6841F2FF70B1
:10BD200047F00207EF602F6AC4F2000027F0010716
:10BD30002F622F6A854247F001072F6207DC9D4280
:10BD400013DCB5F1804F21D08D421FD023E040F2AB
:10BD5000FF37C4F20107BD420CDC41F60007C4F214
:10BD60000007BD4212D000270CE095420ED0654579
:10BD70000CD010E044F20007C4F20107BD4205D028
:10BD800040F20047C4F20107BD4204D1AF6807F09A
:10BD90000707062F03D02F6847F001072F6042F2F4
:10BDA0008450C2F2000090F83F4090F84370012C9C
:10BDB00008BF012F46D1022780F83F7080F84370FA
:10BDC000EF6841F2FF7047F00407EF602F6AC4F29A
:10BDD000000027F010072F622F6A854247F01007F6
:10BDE0002F6207DC9D4213DCB5F1804F21D08D42DC
:10BDF0001FD023E040F2FF37C4F20107BD420CDC44
:10BE000041F60007C4F20007BD4212D000270CE043
:10BE100095420ED065450CD010E044F20007C4F204
:10BE20000107BD4205D040F20047C4F20107BD4200
:10BE300004D1AF6807F00707062F03D02F6847F03B
:10BE400001072F6042F28450C2F2000090F8404097
:10BE500090F84470012C08BF012F46D1022780F8CA
:10BE6000407080F84470EF6841F2FF7047F00807B7
:10BE7000EF602F6AC4F2000027F480772F622F6AE8
:10BE8000854247F480772F6207DC9D4213DCB5F1D1
:10BE9000804F21D08D421FD023E040F2FF37C4F203
:10BEA0000107BD420CDC41F60007C4F20007BD42A9
:10BEB00012D000270CE095420ED065450CD010E062
:10BEC00044F20007C4F20107BD4205D040F200472A
:10BED000C4F20107BD4204D1AF6807F00707062F7F
:10BEE00003D02F6847F001072F6042F28450C2F25E
:10BEF000000090F8414090F84570012C08BF012FD8
:10BF000046D1022780F8417080F84570EF6841F211
:10BF1000FF7047F01007EF602F6AC4F2000027F4AB
:10BF200080572F622F6A854247F480572F6207DCC3
:10BF30009D4213DCB5F1804F21D08D421FD023E00C
:10BF400040F2FF37C4F20107BD420CDC41F60007A6
:10BF5000C4F20007BD4212D000270CE095420ED07B
:10BF600065450CD010E044F20007C4F20107BD4261
:10BF700005D040F20047C4F20107BD4204D1AF68CA
:10BF800007F00707062F03D02F6847F001072F603F
:10BF900042F25C60C2F20000056841F211142F6A9F
:10BFA000274208D12F6A40F24444274203D12F6828
:10BFB00027F001072F6000276F62EF6827F0010765
:10BFC000EF6090F83E4090F84270012C08BF012FBE
:10BFD00046D1022780F83E7080F84270EF6841F247
:10BFE000FF7047F00207EF602F6AC4F2000027F0ED
:10BFF00001072F622F6A854247F001072F6207DC95
:10C000009D4213DCB5F1804F21D08D421FD023E03B
:10C0100040F2FF37C4F20107BD420CDC41F60007D5
:10C02000C4F20007BD4212D000270CE095420ED0AA
:10C0300065450CD010E044F20007C4F20107BD4290
:10C0400005D040F20047C4F20107BD4204D1AF68F9
:10C0500007F00707062F03D02F6847F001072F606E
:10C0600042F25C60C2F2000090F83F4090F84370EA
:10C07000012C08BF012F46D1022780F83F7080F8BD
:10C080004370EF6841F2FF7047F00407EF602F6ADA
:10C09000C4F2000027F010072F622F6A854247F094
:10C0A00010072F6207DC9D4213DCB5F1804F21D0D1
:10C0B0008D421FD023E040F2FF37C4F20107BD429A
:10C0C0000CDC41F60007C4F20007BD4212D0002785
:10C0D0000CE095420ED065450CD010E044F200070C
:10C0E000C4F20107BD4205D040F20047C4F2010787
:10C0F000BD4204D1AF6807F00707062F03D02F68B1
:10C1000047F001072F6042F25C60C2F2000090F835
:10C11000404090F84470012C08BF012F46D10227FF
:10C1200080F8407080F84470EF6841F2FF7047F08B
:10C130000807EF602F6AC4F2000027F480772F62AF
:10C140002F6A854247F480772F6207DC9D4213DC1B
:10C15000B5F1804F21D08D421FD023E040F2FF3750
:10C16000C4F20107BD420CDC41F60007C4F200072F
:10C17000BD4212D000270CE095420ED065450CD090
:10C1800010E044F20007C4F20107BD4205D040F2BE
:10C190000047C4F20107BD4204D1AF6807F00707AA
:10C1A000062F03D02F6847F001072F6042F25C6032
:10C1B000C2F2000090F8414090F84570012C08BF91
:10C1C000012F46D1022780F8417080F84570EF6852
:10C1D00041F2FF7047F01007EF602F6AC4F20000D1
:10C1E00027F480572F622F6A854247F480572F62C9
:10C1F00007DC9D4213DCB5F1804F21D08D421FD06A
:10C2000023E040F2FF37C4F20107BD420CDC41F6E7
:10C210000007C4F20007BD4212D000270CE095428F
:10C220000ED065450CD010E044F20007C4F20107BF
:10C23000BD4205D040F20047C4F20107BD4204D11F
:10C24000AF6807F00707062F03D02F6847F00107F4
:10C250002F60F76841F2111427F00807F760376A7A
:10C2600027F480773762376A3762376A274208D106
:10C27000376A40F24440074203D1306820F00100A1
:10C28000306042F264480126C2F2000888F840603B
:10C2900088F84460E86820F00800E860286A20F424
:10C2A00080702862286A2862286A204208D1286A99
:10C2B00040F24447384203D1286820F0010028604A
:10C2C00042F25C60C2F2000080F8406080F8446096
:10C2D000E8684EF2001740F00100E8604FF480601B
:10C2E000CEF2000738604FF4000038604FF48070E1
:10C2F00078609BF83D0001283ED102208BF83D007C
:10C30000DBF8006041F2FF77F068C4F2000740F00C
:10C310000100BE42F06007DC9E4213DCB6F1804FA4
:10C3200021D08E421FD023E040F2FF30C4F2010042
:10C3300086420CDC41F60000C4F20000864212D0B6
:10C3400000200CE096420ED066450CD010E044F27E
:10C350000000C4F20100864205D040F20040C4F261
:10C360000100864204D1B06800F00700062803D01F
:10C37000306840F00100306062B64FF0805840F203
:10C38000DC5B41F66030C2F200000178E1B1C80721
:10C390004EF24730C0F6000040F0928048070AD5C0
:10C3A0004EF26630C0F60000FBF72AFA41F6603024
:10C3B000C2F20000017888074EF25930C0F6000042
:10C3C00048BFFBF71DFA7DE0FAF7E6FF0990FAF7A0
:10C3D000E3FF0A90FAF7E0FF0B90FAF7DDFF0C900D
:10C3E000FAF7DAFF0D90FAF7D7FF0E90FAF7D4FFBD
:10C3F0000F90FAF7D1FF1090FAF7CEFF1190FAF7ED
:10C40000CBFF1290FAF7C8FF1390FAF7C5FF14900C
:10C41000FAF7C2FF1590FAF7BFFF1690FAF7BCFFC4
:10C420001790FAF7B9FF1890FAF7B6FF1990FAF7D4
:10C43000B3FF1A90FAF7B0FF1B90FAF7ADFF42F284
:10C44000EC61C2F2000109781C90012940F0CB8315
:10C4500042F2EC60C2F200000021017041F6D460AB
:10C46000C2F20000D9F8002090F83D0020284EF2DA
:10C47000D020C0F6000040F0B48341F6D460C2F290
:10C48000000001688869800740F1AA82D9F800009D
:10C49000801A1A28F6D388698007F3D541F6D4614B
:10C4A000C2F20001002220200A6381F83D0081F8D9
:10C4B0003E20086C40F02000086481F83C208CE3AA
:10C4C000FBF79EF940F618404FF60001C4F2020057
:10C4D000CFF6FF714FF480524250D9F80000D9F8DE
:10C4E0000010091A64290ED8D9F80010091A642915
:10C4F00009D8D9F80010091A642904D8D9F800100D
:10C50000091A6529EBD340F618404FF60001C4F232
:10C510000200CFF6FF7140F80180D9F80000D9F889
:10C520000010091A64290ED8D9F80010091A6429D4
:10C5300009D8D9F80010091A642904D8D9F80010CC
:10C54000091A6529EBD340F618404FF60001C4F2F2
:10C550000200CFF6FF714FF480524250D9F800002C
:10C56000D9F80010091A64290ED8D9F80010091A50
:10C57000642909D8D9F80010091A642904D8D9F80F
:10C580000010091A6529EBD340F618404FF6000158
:10C59000C4F20200CFF6FF7140F80180D9F8000024
:10C5A000D9F80010091A64290ED8D9F80010091A10
:10C5B000642909D8D9F80010091A642904D8D9F8CF
:10C5C0000010091A6529EBD340F618404FF6000118
:10C5D000C4F20200CFF6FF714FF480524250D9F8F6
:10C5E0000000D9F80010091A64290ED8D9F80010F3
:10C5F000091A642909D8D9F80010091A642904D83D
:10C60000D9F80010091A6529EBD340F618404FF607
:10C610000001C4F20200CFF6FF7140F80180D9F8A2
:10C620000000D9F80010091A64290ED8D9F80010B2
:10C63000091A642909D8D9F80010091A642904D8FC
:10C64000D9F80010091A6529EBD340F618404FF6C7
:10C650000001C4F20200CFF6FF714FF48052425045
:10C66000D9F80000D9F80010091A64290ED8D9F8B1
:10C670000010091A642909D8D9F80010091A642988
:10C6800004D8D9F80010091A6529EBD340F61840F0
:10C690004FF60001C4F20200CFF6FF7140F80180AE
:10C6A000D9F80000D9F80010091A64290ED8D9F871
:10C6B0000010091A642909D8D9F80010091A642948
:10C6C00004D8D9F80010091A6529EBD340F61840B0
:10C6D0004FF60001C4F20200CFF6FF714FF4805212
:10C6E0004250D9F80000D9F80010091A64290ED870
:10C6F000D9F80010091A642909D8D9F80010091AC4
:10C70000642904D8D9F80010091A6529EBD340F63A
:10C7100018404FF60001C4F20200CFF6FF7140F856
:10C720000180D9F80000D9F80010091A64290ED840
:10C73000D9F80010091A642909D8D9F80010091A83
:10C74000642904D8D9F80010091A6529EBD340F6FA
:10C7500018404FF60001C4F20200CFF6FF714FF40B
:10C7600080524250D9F80000D9F80010091A642903
:10C770000ED8D9F80010091A642909D8D9F8001080
:10C78000091A642904D8D9F80010091A6529EBD3CD
:10C7900040F618404FF60001C4F20200CFF6FF71D8
:10C7A00040F80180D9F80000D9F80010091A64296E
:10C7B0000ED8D9F80010091A642909D8D9F8001040
:10C7C000091A642904D8D9F80010091A6529EBD38D
:10C7D00040F618404FF60001C4F20200CFF6FF7198
:10C7E0004FF480524250D9F80000D9F80010091ACD
:10C7F00064290ED8D9F80010091A642909D8D9F883
:10C800000010091A642904D8D9F80010091A6529FA
:10C81000EBD340F618404FF60001C4F20200CFF609
:10C82000FF7140F80180D9F80000D9F80010091A0A
:10C8300064290ED8D9F80010091A642909D8D9F842
:10C840000010091A642904D8D9F80010091A6529BA
:10C85000EBD340F618404FF60001C4F20200CFF6C9
:10C86000FF714FF480524250D9F80000D9F80010FF
:10C87000091A64290ED8D9F80010091A642909D8B0
:10C88000D9F80010091A642904D8D9F80010091A37
:10C890006529EBD340F618404FF60001C4F20200C0
:10C8A000CFF6FF7140F80180D9F80000D9F80010E8
:10C8B000091A64290ED8D9F80010091A642909D870
:10C8C000D9F80010091A642904D8D9F80010091AF7
:10C8D0006529EBD340F618404FF60001C4F2020080
:10C8E000CFF6FF714FF480524250D9F80000D9F8CA
:10C8F0000010091A64290ED8D9F80010091A642901
:10C9000009D8D9F80010091A642904D8D9F80010F8
:10C91000091A6529EBD340F618404FF60001C4F21E
:10C920000200CFF6FF7140F80180D9F80000D9F875
:10C930000010091A64290ED8D9F80010091A6429C0
:10C9400009D8D9F80010091A642904D8D9F80010B8
:10C95000091A6529EBD340F618404FF60001C4F2DE
:10C960000200CFF6FF714FF480524250D9F8000018
:10C97000D9F80010091A64290ED8D9F80010091A3C
:10C98000642909D8D9F80010091A642904D8D9F8FB
:10C990000010091A6529EBD340F618404FF6000144
:10C9A000C4F20200CFF6FF7140F80180D9F8000010
:10C9B000D9F80010091A64293FF6E3ACD9F8001041
:10C9C000091A64293FF6DDACD9F80010091A642968
:10C9D0003FF6D7ACD9F80010091A6429E8D9D0E499
:10C9E00041F6D460C2F2000090F83C0001284EF2FB
:10C9F000D020C0F6000000F0F48041F6D460C2F20E
:10CA00000000012280F83C200868C00703D10868B4
:10CA100040F001000860086841F6D46220F400602C
:10CA20000860C2F20002212082F83D00402082F816
:10CA30003E000020106441F65830C2F200005062FF
:10CA400008205085508D10850020CFF6FF70D062F1
:10CA5000086840F4807008604869C00709D14869D7
:10CA6000C00704BF48695FEAC07002D14869C007C7
:10CA7000F2D0A0200861F6F7FFFF00284EF2D02088
:10CA8000C0F6000040F0AD8000201D9041F6D4605B
:10CA9000C2F20000016848691D9088691D901D98C8
:10CAA0004869000615D44869400577D448690006EE
:10CAB0000FD44869400571D44869000609D4486913
:10CAC00040056BD44869000603D448694005E7D5A2
:10CAD00064E00020086141F6D460C2F20000068DD7
:10CAE000002E3FD0426A03E0020406461A4639D0BF
:10CAF0004869000615D4486940054FD448690006C6
:10CB00000FD44869400549D44869000609D44869EA
:10CB1000400543D44869000603D448694005E7D579
:10CB20003CE0134613F8010B41F6D4650861C2F2EC
:10CB30000005701E6B6228856F8D013F6F854F6900
:10CB40007F07D1D50704CFD0507841F6D46708616C
:10CB5000931CC2F20007B01E7B6238857A8D013AC1
:10CB60007A85C1E74869400700F1C88048694005F7
:10CB700014D44869400700F1C180486940050DD4CC
:10CB80004869400700F1BA804869400506D4486901
:10CB9000400700F1B38048694005E3D56FF4806039
:10CBA00041F6D4624861C2F20002002320201363E0
:10CBB00082F83D0082F83E30106C40F004001064B2
:10CBC00082F83C30106C04284EF2D020C0F60000F1
:10CBD00007D1086840F4007008604EF2D020C0F61B
:10CBE0000000FAF70DFE4FF0140C4FF0000E0EF19E
:10CBF00001024FFA8EF354B24FFA8CF6B4421D463E
:10CC0000724616DC724603E0601C44B2B4420FDC8C
:10CC100067B25AF827505AF823008542F4DA50B226
:10CC20000AEB8000416801324AF827104560EBE7C3
:10CC300055B25AF825005AF823104AF82300D0B20A
:10CC40000A284AF8251007D050B20A28D4BF02F1AA
:10CC5000010EA2F1010CCAE7139840F2EE01C2F2F4
:10CC60000001087040F618404FF60001C4F20200BF
:10CC7000CFF6FF714FF480524250D9F80000D9F836
:10CC80000010091AB1F5FA7F11D8D9F80010091A65
:10CC9000B1F5FA7F0BD8D9F80010091AB1F5FA7F6F
:10CCA00005D8D9F80010091AB1F5FA7FE7D940F68E
:10CCB00018404FF60001C4F20200CFF6FF7140F8B1
:10CCC0000180D9F80000D9F80010091A59453FF63B
:10CCD00058ABD9F80010091A59453FF652ABD9F8AC
:10CCE0000010091A59453FF64CABD9F8001040F234
:10CCF000DD52091A9142E6D3FFF743BB086840F4BE
:10CD00000070086041F6D460C2F20000202180F873
:10CD10003D10002180F83E1080F83C10D9F800103A
:10CD2000D9F80000401A052813D8D9F80000401A95
:10CD300005280ED8D9F80000401A052809D8D9F8D6
:10CD40000000401A06284EF22630C0F60000E7D355
:10CD500047E74EF22630C0F6000042E72DE9F04FDB
:10CD600081B00C4642F25C61C2F2000142F690369C
:10CD70000A68C2F20006315D126941F6643AD207D0
:10CD800042F6A839074641F28832C2F2000AC2F2DE
:10CD9000000918BF07F580379042DAF80020D9F86B
:10CDA0000030A8BF0746D01AC01942F2EE6502460D
:10CDB000C2F2000548BF42422B78682A0ED8591C9F
:10CDC000297004EB440142F210720901C2F2000220
:10CDD00050500120305501B0BDE8F08F032B1DD815
:10CDE00000200121C6E90000C6E90200C6E90400EE
:10CDF0003155297042F2ED61C2F20001087004EB76
:10CE0000440142F210720901C2F20002C9F8007036
:10CE1000CAF80000505001B0BDE8F08F46F23D72F4
:10CE2000C0F20202904210DB42F2ED6BC2F2000B44
:10CE30009BF8000004285BD341F65030C2F200009A
:10CE4000007870B3FAF768FA52E00029C3D00129DC
:10CE500019D1A0F21B41B1F5EC6FBCD842F21072AF
:10CE600004EB4401C2F2000202EB0111486042F2FD
:10CE7000ED61C2F200010A7802203055501C0870A2
:10CE800001B0BDE8F08F0B29A5D842F2107304EB76
:10CE90004402C2F2000303EB021242F82100481CD4
:10CEA00098E741F2B86042F21071C2F20000C2F29B
:10CEB00000014FF49062F4F7D2FB96E80F5041F670
:10CEC0003838C2F2000888E80F5041F6503101208E
:10CED000C2F20001087042F21460C2F20000006861
:10CEE000016841F001010160C16841F00101C160C8
:10CEF00042F21078C2F2000840464FF49061F4F715
:10CF000002FC04EB4402002001211201C6E90000EA
:10CF1000C6E90200C6E904003155CAF8000048F825
:10CF2000020029708BF80000C9F8007001B0BDE85C
:10CF3000F08F5FEA400C08BF91F0000F4FEA8C239E
:10CF40004FEAC12243EA51514FEA1C5018BF00F585
:10CF5000F0404FEA300018BF41F000415FEA6C5CDE
:10CF600000F02980BCF1FF3F08BF40F080407047CF
:10CF7000130C06BF12044FF0100C4FF0000C130EF0
:10CF800004BF12020CF1080C130F04BF12010CF1C4
:10CF9000040C930F04BF92000CF1020CD30F04BFDA
:10CFA00052000CF1010C11464FF00002A0F11F00DD
:10CFB000A0EB0C00704711F0004F08BF704731F034
:10CFC00000413FF4D5AF0B0C06BF09044FF0100C25
:10CFD0004FF0000C0B0E04BF09020CF1080C0B0FF4
:10CFE00004BF09010CF1040C8B0F04BF89000CF184
:10CFF000020CCB0F04BF49000CF1010CCCF1200353
:10D0000022FA03F341EA030102FA0CF2A0EB0C004E
:10D0100000F101007047000023F07F4720F07F4CB3
:10D0200080EA030000F00040ACEB070303F57C53FB
:10D0300003F1FF032DE9804909B44FEA144324EAC0
:10D0400003484FEA154B25EA0B4E0FF2042606EB78
:10D0500013273E7803FB0667C7F5000707FB06F6B4
:10D060004FEAD64606F102064FEA543707FB066C34
:10D07000CCF1005C4FEA1C472CEA074C0CFB06F590
:10D0800007FB06F404EB15464FEA961649085FEADB
:10D09000320234BF00204FF000404FEAD13706FB88
:10D0A00007FC4FEA1C4C0CFB0BF7D21B03FB0CF7E5
:10D0B00061EB07010CFB0EF7B0EB074072EB174278
:10D0C0000CFB08F734BFA2EB0742B2EB074261EB5F
:10D0D00017414FEA0C444FEA910706FB07FC4FEA61
:10D0E0001C4C0CFB0BF7B0EBC74072EB573203FB49
:10D0F0000CF734BFA2EBC742B2EBC74261EB57312A
:10D100000CFB0EF7B0EBC70072EB57720CFB08F785
:10D1100034BFA2EBC702B2EBC70261EB57714FEA13
:10D12000816141EA92114FEA826242EA90124FEA2B
:10D13000806004EBCC04039F4FEAD13706FB07FC69
:10D140004FEA1C4C0CFB0BF7D21B03FB0CF761EBFB
:10D1500007010CFB0EF7B0EB074072EB17420CFB1C
:10D1600008F734BFA2EB0742B2EB074261EB17416D
:10D170004FEA8C5504EB9C244FEA910706FB07FC11
:10D180004FEA1C4C0CFB0BF7B0EBC74072EB57326D
:10D1900003FB0CF734BFA2EBC742B2EBC74261EB13
:10D1A00057310CFB0EF7B0EBC70072EB57720CFB5C
:10D1B00008F734BFA2EBC702B2EBC70261EB5771AD
:10D1C0004FEA816141EA92114FEA826242EA90128B
:10D1D0004FEA806015EB4C2544F100044FEAD1374B
:10D1E00006FB07FC4FEA1C4C0CFB0BF7D21B03FBA6
:10D1F0000CF761EB07010CFB0EF7B0EB074072EB8D
:10D2000017420CFB08F734BFA2EB0742B2EB074210
:10D2100061EB17414FEA813141EA92414FEA823294
:10D2200042EA90424FEA80304FEA0C7615EB1C152B
:10D2300044F1000448EA03434EEA0B484FF0000E65
:10D24000B2EB080C71EB030724BF624639464EEB84
:10D250000E0E4FF0000B0018524149414BEB0B0BE7
:10D26000B2EB080C71EB03077BF1000B24BF6246A5
:10D2700039464EEB0E0E4FF0000B0018524149415B
:10D280004BEB0B0BB2EB080C71EB03077BF1000BC4
:10D2900024BF624639464EEB0E0E51EA020718BF14
:10D2A00046F0010616EB0E7655F1000254F100012E
:10D2B00003D5BDE88901BDE80088BDE88901BDE866
:10D2C0000048B619524141EB0101A3F10103704737
:10D2D00080807F7E7D7C7B7A7978777676757473B3
:10D2E000727171706F6E6E6D6C6C6B6A6A69686872
:10D2F000676666656464636362616160605F5F5E08
:10D300005E5D5D5C5C5B5B5A5A595958585757567D
:10D3100056555555545453535252525151505050E2
:10D320004F4F4F4E4E4D4D4D4C4C4C4B4B4B4A4A34
:10D330004A49494948484847474747464646454578
:10D3400045444444444343434342424242414141B1
:10D350009C46002B30D477002BD04FEA37071CB502
:10D3600003B44FF010004FF01001BAF1000F06D0D7
:10D37000BCF1000FDCBF40F0080040F008014FF0A6
:10D3800000000FBCBDE810400BF1010BBBF1010F19
:10D3900008BF5FEA170722BF12F1010211F1010174
:10D3A0004FF0004143F1000300F0004043EA000069
:10D3B0007047F9D35708D0E746EA06464FEA1646C3
:10D3C00013F1400F1FDD13F1200FDFBF16430A4694
:10D3D000002120335B42BED0C3F1200746EA064657
:10D3E0004FEA164602FA07F746EA070622FA03F260
:10D3F000C3F1200701FA07F742EA070221FA03F115
:10D400004FF00003A7E746EA020646EA06464FEA5F
:10D41000164646EA0106BCBF46EA0646360C4FF001
:10D4200000034FF000024FF0000194E72DE9804C1B
:10D4300070B49A46934691E8380007C831EA400C28
:10D4400048BF34EA430C03D5FFF7E6FDFFF780FF42
:10D45000F0BCBDE8008C2DE9804C70B49A46934630
:10D4600091E8380007C810F0804F08BF13F0804FD4
:10D4700003D100F005F8FFF76BFFF0BCBDE8008CAE
:10D4800020F07F4723F07F4C80EA030000F000404B
:10D4900007EB0C03A3F57C53A3F1FE0392F0000FFE
:10D4A00000F0B38095F0000F00F077802DE901497E
:10D4B0004FEA114021EA00484FEA144624EA0647A1
:10D4C00000FB06FC08FB06F607FB08F818EB06480D
:10D4D0004CEB164C00FB07F718EB07484CEB1740DA
:10D4E0004FEA124B22EA0B4E4FEA154625EA064751
:10D4F0000BFB06FC0EFB06F607FB0EFE1EEB064EB4
:10D500004CEB164C0BFB07F71EEB074E4CEB174B87
:10D5100018EB0B0840F1000018EB0E0B58EB00085D
:10D5200040F100008F1A4FF000014FF000063CBFA1
:10D53000C943661B14BFB5EB040C00213CBFC943B3
:10D54000F61B4FEA174427EA04454FEA1C472CEA2A
:10D55000074C04FB076205FB07F70CFB05F616EB0F
:10D56000074642EB174204FB0CFC16EB0C4642EB61
:10D570001C421BEB060658EB020241414EEA8E0E9E
:10D5800046EA9E0601D5BDE80189B619524141EB34
:10D590000101A3F10103BDE801894FEA144524EA22
:10D5A00005464FEA114721EA074C05FB07F406FB45
:10D5B00007F70CFB06F111EB074144EB174405FBA1
:10D5C0000CFC11EB0C4144EB1C444FEA124722EADD
:10D5D000074C05FB07F206FB07F70CFB06F616EBFC
:10D5E000074642EB174205FB0CFC16EB0C4642EBE0
:10D5F0001C456A1854F1000148BF7047B6195241E2
:10D6000041EB0101A3F10103704795F0000F37D002
:10D610004FEA114221EA02464FEA144724EA074C36
:10D6200002FB07F106FB07F70CFB06F414EB0744BB
:10D6300041EB174102FB0CFC14EB0C4441EB1C4189
:10D640004FEA154725EA074C02FB07F506FB07F7EB
:10D650000CFB06F616EB074645EB174502FB0CFCE8
:10D6600016EB0C4645EB1C42121951F1000148BF64
:10D670007047B619524141EB0101A3F10103704714
:10D680004FEA144524EA05464FEA114721EA074CC0
:10D6900005FB07F106FB07F70CFB06F212EB07424E
:10D6A00041EB174105FB0CFC12EB0C4251EB1C410A
:10D6B0004FF0000648BF7047921841EB0101A3F1FB
:10D6C0000103704703B401984100009850EAC1205B
:10D6D00018BF04204A0D18BF40F0010040F2FF724D
:10D6E000B2EB515F08BF40F00200012808BF0520DF
:10D6F00002B0704730380A2801D20120704700205C
:10D700007047000010B500290AD00878002807D01B
:10D7100005487844F3F7A0FE002801D0002010BD92
:10D720000248784410BD0000F20C0000EA0C000032
:10D7300010B500290AD00878002807D00548784499
:10D74000F3F78AFE002801D0002010BD024878447B
:10D7500010BD0000E20C0000DA0C000021F00042D5
:10D7600001F00043A2F16052B2F5801F28BFD2F150
:10D770007F6C0BD95FEA001C43EAC20242EB507097
:10D7800018BF704728BF20F001007047B2F5801F16
:10D79000BCBF184670474FEA410C1CF5001F02D26F
:10D7A000084600F04FBC70B500F062FA0000008936
:10D7B000FFF7F6BF4FF00040A0F580007047000073
:10D7C00010B591EA030F48BF83F0004300F1AC822B
:10D7D000841A71EB030C05D2121943EB0C03001BE6
:10D7E00061EB0C014FEA1154A4EB135CDFF81CE170
:10D7F0001EEA430F18BF9EEA445F00F0748021EADE
:10D80000045123EA0E0343F48013DCF1200E32D3DB
:10D8100022FA0CFE10EB0E0023FA0CFE41EB0E0177
:10D82000CCF1200E03FA0EFE10EB0E00CCF1200E10
:10D8300051F10001B1F5801F32D201EB045112FA0F
:10D840000EF2BDE8104058BF7047401C38BF5FEA79
:10D85000420218BF7047002814BF20F0010041F1B8
:10D8600000014FEA410313F5001F38BF7047A1F1D3
:10D87000C04100F04BBA012A43EB0302ACF1200C8B
:10D88000DCF11F0E32BF4FF0000E23FA0CF310EB49
:10D89000030041EB0451B4EB115FD0D0A1EB045174
:10D8A00001F58011490801EB04515FEA30000ED305
:10D8B00050F1000038BF12FA0EFE08D1BDE810404A
:10D8C000C9E7401C38BF5FEA4202CAD1C3E7BDE8DE
:10D8D00010404FEA410313F5001F38BF7047A1F114
:10D8E000C04100F013BA9EEA445F08D011EA5E0F0F
:10D8F000BDE8104004BF01F0004100207047BDE8C2
:10D90000104070B500F0B4F964FBBE3E0000E0FFCB
:10D91000491058BFC1F140415B1058BFC3F14043AB
:10D920008B42EFF30080704751EA030C17D41CF5CB
:10D93000801F58BFBCF5801F00F10680994218BFB8
:10D94000704708BF9042704707D711F5801F58BF36
:10D9500013F5801F19D499427047894270471CF50E
:10D96000801F08D5BCF5801FF7D58B4218BF7047C4
:10D9700008BF824270474FF4001C1CEB410F38BFB8
:10D980001CEB430F01D28B42704770B500F070F969
:10D99000922449004FF000514FF08053FFF7B8BF79
:10D9A0004FEA41034FEA5353A3F58063D3F11E03BB
:10D9B000C8BFD3F1210C0CDD4FF0004242EAC12276
:10D9C00042EA505232FA03FC8CEAE17CACEBE170A3
:10D9D0007047102BC4BF0020704703F5787CBCF162
:10D9E000FF3F04D06FF0004282EA2100704770B51B
:10D9F00000F03EF94992248000207047F2E710F0D1
:10DA0000004248BF4042B0FA80F310FA03F10AD056
:10DA1000C3F11D0303F5806302EB03524FEA41504B
:10DA200002EBD12170474FF00000704751EA030C20
:10DA300017D41CF5801F58BFBCF5801F00F106806D
:10DA4000994218BF704708BF9042704707D711F539
:10DA5000801F58BF13F5801F19D49942704789421F
:10DA600070471CF5801F08D5BCF5801FF7D58B4289
:10DA700018BF704708BF824270474FF4001C1CEB70
:10DA8000410F38BF1CEB430F01D28B42704770B57A
:10DA900000F0EEF8922449004FF080514FF000530F
:10DAA000FFF736BF51EA030C17D41CF5801F58BF8F
:10DAB000BCF5801F00F10680994218BF704708BF6F
:10DAC0009042704707D711F5801F58BF13F5801F8C
:10DAD00019D499427047894270471CF5801F08D5B8
:10DAE000BCF5801FF7D58B4218BF704708BF824234
:10DAF00070474FF4001C1CEB410F38BF1CEB430F69
:10DB000001D28B42704770B500F0B2F89224490000
:10DB10004FF000514FF08053FFF7FABE70B5DFF8B9
:10DB200048C11CEA111E1EBF1CEA13159EEA0C0F09
:10DB300095EA0C0F00F06F8081EA03044EEAD47E70
:10DB4000AE4421EA4C1123EA4C1341F4801143F412
:10DB50008013AEF17F7EA1FB024CA0FB036536195A
:10DB600055EB0C05A1FB034C4CF10003A0FB021C80
:10DB700016EB0C06654153F10003094218BF46F04D
:10DB8000010613F4007F0BD14FEA03314FEA053051
:10DB900041EA155140EA165034036FF003020AE0DF
:10DBA0004FEAC3214FEAC52041EA555140EA565099
:10DBB000F4026FF0020202EB2E4201EB025585EAFD
:10DBC000CE710AD05FEA440C18BF24F0004450F133
:10DBD000000041F1000120EAD47040F2FE7C624571
:10DBE00000D270BDA84214BF4FF080444FF04044B3
:10DBF000002E08BF0024BEF1806FA8BFA1F1C04174
:10DC0000BDE8704080F2828001F1C04101F0004126
:10DC10004FF0000070470CEA13159EEA0C0F18BF76
:10DC200095EA0C0F06D081EA030E4FF000000EF0CB
:10DC3000004170BD00F01CF88900013E00F007B8FB
:10DC400000F009B84FEA430C5FEA5C5C08D081EA57
:10DC5000030100F05BB84FEA410C5FEA5C5CF6D16F
:10DC600002494FF0000070470000FF070000F87FF6
:10DC70000EF1020E2EF0030E5EF8046B364205D450
:10DC8000012A43EB030515F5001F12D8012841EBCB
:10DC9000010C1CF5001F0CD80ED14FEAD17C0CEB07
:10DCA0004C0C0CF1020C15F5001F08BF4CEBD37C9B
:10DCB00004E04FF0080C01E04FEAD37C0CEB4C057C
:10DCC00026FA05F606F00706B6F1040C06D20EEBAE
:10DCD000860CBDE870404CF0010C6047DFE80CF0AA
:10DCE000090B02024FF00041A1F500214FF00000A6
:10DCF00070BD19461046012851EB010418BFD4F538
:10DD0000001484BF002001F0004170BD0808A0F598
:10DD100000114FEA3101704710B591EA030F48BF77
:10DD200083F000433FF554AD841A71EB030C07D226
:10DD30008CF0004C121943EB0C03001B61EB0C013F
:10DD40004FEA1154A4EB135CDFF8A4E11EEA430F81
:10DD500018BF9EEA445F00F0B48021EA045123EA30
:10DD60006E035242C3EB6E0338BF5B1EDCF1200E24
:10DD700025D322FA0CFE10EB0E0043FA0CFE41EB09
:10DD80000E01CCF1200E03FA0EFE10EB0E00CCF1CA
:10DD9000200E51F1000129D401EB045112FA0EF2C8
:10DDA000BDE8104058BF7047401C1CBFB2F1004F87
:10DDB000704700280CBF491C20F00100704712EB8F
:10DDC000020E43EB030218BF4FF0010E4EEA42026F
:10DDD000ACF1200CDCF11E0E56D943FA0CFE10EB10
:10DDE0000E00CCF11E0E51F1FF31D5D50EF1010E12
:10DDF00012FA0EFE404141EB010101EB445C5FEA87
:10DE00005C5C10D901EB045110EBDE7038BFBEF141
:10DE1000004FBDE8104018BF704700280CBF491CD8
:10DE200020F00100704734D24FEAD42C24F400646F
:10DE300011F500111BD0B1FA81F20B3AA41AA41EFD
:10DE4000D2F12003914030FA03F31943904001EBE3
:10DE5000CC7101EB0451002CBDE81040A8BF704705
:10DE600001F1C04101F000414FF000007047B0FAED
:10DE700080F310FA03F102D1BDE810407047E41AB4
:10DE8000173C4805C90AE2E701EB0451BDE8104020
:10DE9000704749104FEA300001EB0451BDE81040D3
:10DEA00002E04FF0000170474A0008BF0042F8D07E
:10DEB000B2F5001F28BF704701F000414FF000008D
:10DEC00070479EEA445F07D011EA5E0FBDE810403C
:10DED00004BF002100207047BDE8104070B5FFF777
:10DEE000C7FE00BF40DFF63E104683F0004170479A
:10DEF0000000E0FF43004FEAD30C4FEA3C0C4340E4
:10DF00001FBF40070CF1605113F0FE4F70471CF02B
:10DF1000006F03D10CF00041002070470CF000436B
:10DF200043EA507040EACC0010B500F038F800BF6A
:10DF3000000000924FEA0001FFF7E8BE4FF00041F9
:10DF4000A1F500214FF00000704710B5FFF7ECFC81
:10DF50000CBF0120002010BD10B5FFF7E5FC14BF79
:10DF60000120002010BD10B5FFF760FD8CBF01201F
:10DF7000002010BD10B5FFF759FD2CBF0120002077
:10DF800010BD10B5FFF78EFD94BF0120002010BD1D
:10DF900010B5FFF787FD34BF0120002010BD0EF142
:10DFA000020E2EF0030E5EF8044B244204D44FEA16
:10DFB0004102B2F17F4F11D84FEA4003B3F17F4FD6
:10DFC0000CD80ED14FEAD07C0CEB4C0C0CF1020CAF
:10DFD000B2F17F4F08BF4CEBD17C04E04FF0080C4E
:10DFE00001E04FEAD17C0CEB4C0324FA03F404F07B
:10DFF0000704B4F1040C06D20EEB840CBDE810400B
:10E000004CF0010C6047DFE80CF0070802024FF00B
:10E010000040A0F5800010BD0846420018BFD2F1B4
:10E02000807288BF00F0004010BDF1EE100A4FF67C
:10E03000FF71C0F2C03120EA010040F04070E1EE13
:10E04000100A7047FF2141EAD050C0057047F2F72F
:10E050000DBEF2F741BF000000000000000000000C
:10E06000303132333435363738394142434445460E
:10E070004030580030313233343536373839616208
:10E08000636465664030780004000008000000000A
:10E090000000000200010000103031323334353608
:10E0A00037383961626364656678700030313233C5
:10E0B00034353637383941424344454658500000DC
:10E0C00002400000000000A0000000000540000029
:10E0D000000000C8000000000C4000000000409C50
:10E0E00000000000194000000020BCBE000000003D
:10E0F00034400000BFC91B8E00000004B540000082
:10E10000504BCFD06607E2CF010000006C41000009
:10E110003E8251AADFEEA73401000000D942000080
:10E12000DCB5A0E23A301F97FFFFFFFFB4450000C7
:10E13000FD25A0C8E9A3C14FFFFFFFFFFF3F00007F
:10E140000000008000000000FF3F00000000008091
:10E1500000000000000000000100000000000000BE
:10E1600082800000000000008A8000000000008023
:10E1700000800080000000808B8000000000000014
:10E18000010000800000000081800080000000800D
:10E1900009800000000000808A00000000000000EC
:10E1A00088000000000000000980008000000000DE
:10E1B0000A000080000000008B800080000000004A
:10E1C0008B000000000000808980000000000080BB
:10E1D000038000000000008002800000000000803A
:10E1E00080000000000000800A80000000000000A5
:10E1F0000A00008000000080818000800000008014
:10E20000808000000000008001000080000000000D
:10E210000880008000000080000000000100000075
:10E22000BE0000001C0000005B0000002400000095
:10E230002C0100000600000037000000140100005F
:10E24000030000000A000000AB000000990000007D
:10E25000E7000000690000002D0000000F00000032
:10E260001500000088000000D200000042000000FD
:10E27000FD000000780000004E00000000000000DB
:10E28000010203040A0A2020205F5F5F5F5F5F20B6
:10E29000202020202020202020202020202020207E
:10E2A00020202020205F5F20200A00202F202F2008
:10E2B00020202F202F202F202F205F5F20605F5FE6
:10E2C000205C2F205F5F205C2F202F205F200A0022
:10E2D0004661696C656420746F207772697465208B
:10E2E000454550524F4D210A00537563636565647F
:10E2F00020746F20696E697469616C697A65204564
:10E300004550524F4D210A004661696C6564207486
:10E310006F20696E697469616C697A652045455042
:10E32000524F4D210A00454550524F4D20526566CF
:10E33000726573686564210A00494D55204368651C
:10E34000636B6564210A00496E76616C6964206CB8
:10E350006963656E73652E0A00574C414E206572E5
:10E36000726F722E0A00494D55206572726F722EBF
:10E370000A002F202F5F5F5F2F202F5F2F202F207D
:10E380002F202F202F202F202F202F5F2F202F20D6
:10E390002F20205F5F2F0A0020202F205F5F5F5F0C
:10E3A0002F5F20205F5F5F5F5F5F205F5F5F2020E8
:10E3B0005F5F5F5F20202F202F5F5F0A00436F6E3B
:10E3C00066696720416464723A25582025582025E3
:10E3D00058202558202558206368616E6E656C3A78
:10E3E00025750A0030E5000800000020F00000005C
:10E3F000EC01000820E60008F0000020283F0000A3
:10E400000C0200081C00000043000000F8FFFFFFA2
:10E410000C0000000E0000000F0000002E000000A5
:10E420001001000043000000F8FFFFFF00404040E3
:10E4300040404040404041414141414040404040D7
:10E440004040404040404040404040404005020283
:10E450000202020202020202020202020220202042
:10E46000202020202020200202020202020290909E
:10E47000909090901010101010101010101010109C
:10E4800010101010101010100202020202028888F0
:10E4900088888888080808080808080808080808FC
:10E4A00008080808080808080202020240000000E4
:10E4B000000000000000000000000000000000005C
:10E4C000000000000000000000000000000000004C
:10E4D000000000000000000000000000000000003C
:10E4E000000000000000000000000000000000002C
:10E4F000000000000000000000000000000000001C
:10E50000000000000000000000000000000000000B
:10E5100000000000000000000000000000000000FB
:10E5200000000000000000000000000000000000EB
:10E53000CD6A0008016B0008116B00082D6B000804
:10E54000496B0008AD6A0008DD6A00080024F40089
:10E5500061680008BD61000839690008000000001A
:10E5600029630008E16000087961000800000000EC
:10E57000000000000000000015650008716300083D
:10E58000BD6600086163000809024300020100C083
:10E5900032090400000102020100052400100105F7
:10E5A000240100010424020205240600010705825B
:10E5B0000308001009040100020A00000007050119
:10E5C0000240000007058102400000000A06000228
:10E5D00000000040010000001201000202020040A1
:10E5E00079041D57000201020301000061170008B1
:10E5F0005D17000859170008A5170008ED19000855
:10E60000040309041A0300000000000000000000D9
:10E61000000000000000000000000000000064FF97
:040000050800018965
:00000001FF
